:100000000C94500E0C9458170C9489170C94BA1732
:100010000C94EB170C941C180C944D180C947E182F
:100020000C94AF180C947D0E0C947D0E0C947D0EE8
:100030000C947D0E0C9490930C947D0E0C947D0E7C
:100040000C947D0E0C94A5690C947D0E0C947D0E81
:100050000C947D0E0C947D0E0C946D720C944714D0
:100060000C947D0E0C944A3F0C947D0E0C947D0EE6
:100070000C947D0E0C947D0E0C947D0E0C947D0ED4
:100080000C947D0E0C947D0E0C947D0E0C947D0EC4
:100090000C947D0E0C947D0E0C947D0E0C947D0EB4
:1000A0000C947D0E0C947D0E0C947D0E0C947D0EA4
:1000B0000C947D0E0C947D0E0C947D0E0C947D0E94
:1000C0000C947D0E0C947D0E0C947D0E0C947D0E84
:1000D0000C947D0E0C947D0E0C947D0E0C947D0E74
:1000E0000C947D0E084AD73B3BCE016E84BCBFFD0D
:1000F000C12F3D6C74319ABD56833DDA3D00C77FF8
:1001000011BED9E4BB4C3E916BAAAABE0000008090
:100110003F05A84CCDB2D44EB93836A9020C50B91F
:10012000918688083CA6AAAA2ABE000000803F004B
:10013000002100240027002A002D00300033000198
:10014000010000040107010A010000220025002827
:10015000002B002E003100340002010000050108D0
:10016000010B01000020002300260029002C002F95
:100170000032000001000003010601090105050528
:1001800005070508080808020202020A0A0808040E
:10019000040404010101010101010103030303033C
:1001A000030303040707070C0C0C0C0C0C0C0C02CB
:1001B00002020206060606060606060B0B0B0B0BD2
:1001C0000B0B0B01021020200808102040102040CB
:1001D000800201020108040201010204081020400B
:1001E0008080402010080402018004020180402029
:1001F0001008040201080402010102040810204052
:100200008001020408102040800000090A02080B47
:100210000C0D0706030401000000000000000000B0
:1002200000000000000000000000000000000000CE
:10023000000000000011100F00000000000000008E
:100240000000000000000000000000000000006549
:1002500063686F3A004572726F723A0053544F50A0
:100260005045442E20005072696E7465722073747C
:100270006F707065642064756520746F206572729C
:100280006F72732E204669782074686520657272DB
:100290006F7220616E6420757365204D3939392085
:1002A000746F20726573746172742E202854656DAA
:1002B000706572617475726520697320726573650B
:1002C000742E2053657420697420616674657220F1
:1002D00072657374617274696E6729004B494C4C86
:1002E00045442E20005072696E7465722068616CFE
:1002F0007465642E206B696C6C28292063616C6CBA
:10030000656421006F6B00526573656E643A20006E
:100310002200556E6B6E6F776E20636F6D6D616E30
:10032000643A2022004368616E67652066696C61EB
:100330006D656E74005A204F6666736574203A20AE
:10034000007A5F6D61783A20007A5F6D696E3A20BD
:10035000005A204F6666736574005A204F666673B4
:100360006574206F6B007A5F6D696E3A2000795F6B
:100370006D696E3A2000785F6D696E3A2000205AF0
:100380003A0020593A0020436F756E7420583A2085
:100390000020453A00205A3A0020593A00583A00C5
:1003A0004649524D574152455F4E414D453A4D6188
:1003B000726C696E2056313B20537072696E7465A1
:1003C000722F6772626C206D617368757020666F42
:1003D000722067656E36204649524D574152455F3F
:1003E00055524C3A687474703A2F2F6669726D7763
:1003F0006172652E756C74696D616B65722E636FC9
:100400006D2050524F544F434F4C5F564552534905
:100410004F4E3A312E30204D414348494E455F54AE
:100420005950453A556C74696D616B657220455839
:100430005452554445525F434F554E543A3120551E
:100440005549443A30303030303030302D30303053
:10045000302D303030302D303030302D30303030A5
:1004600030303030303030300A00556C74696D6196
:100470006B6572204F66662E0042656420646F6E65
:10048000652E0020423A0020453A00543A00426569
:10049000642048656174696E672E004865617469FF
:1004A0006E6720646F6E652E0020573A0020453A33
:1004B00000543A0048656174696E672E2E2E002044
:1004C00042403A0020403A00202F003A00205400D9
:1004D000202F0020423A00202F006F6B20543A005A
:1004E0002569206D696E2C202569207365630045A0
:1004F0006E642066696C65206C6973740042656780
:10050000696E2066696C65206C697374004E6F209B
:100510006D6F76652E00526573756D696E6720701C
:1005200072696E74005761697420666F722075730A
:1005300065722E2E2E00536C6565702E2E2E00FFD8
:10054000FFFF0000524300005243000052430000EE
:10055000000000000000000000000000000000009B
:100560000000000000000000524300005243000061
:1005700052430000A0400000A04000000040256958
:1005800020686F757273202569206D696E757465BA
:100590007300446F6E65207072696E74696E6720B7
:1005A00066696C650053544F505045442E200050EE
:1005B00072696E7465722073746F70706564206404
:1005C000756520746F206572726F72732E20466994
:1005D0007820746865206572726F7220616E642085
:1005E000757365204D39393920746F2072657374C5
:1005F0006172742E202854656D7065726174757215
:10060000652069732072657365742E2053657420AC
:1006100069742061667465722072657374617274A6
:10062000696E6729006F6B004E6F204C696E652004
:100630004E756D62657220776974682063686563C2
:100640006B73756D2C204C617374204C696E653A28
:1006500020004E6F20436865636B73756D2077696A
:100660007468206C696E65206E756D6265722C20F1
:100670004C617374204C696E653A20006368656351
:100680006B73756D206D69736D617463682C204C9C
:10069000617374204C696E653A20004C696E652068
:1006A0004E756D626572206973206E6F74204C61A7
:1006B0007374204C696E65204E756D6265722B31C6
:1006C0002C204C617374204C696E653A20004D31CA
:1006D000313000446F6E6520736176696E67206605
:1006E000696C652E006F6B004D3239002020506C14
:1006F000616E6E6572427566666572427974657385
:100700003A20002046726565204D656D6F72793A1A
:100710002000536570203139203230313400436F6E
:100720006D70696C65643A200028446176696420C4
:10073000427261616D2900207C20417574686F727E
:100740003A20005365702031392032303134203165
:10075000303A32323A323900204C6173742055708D
:1007600064617465643A2000312E302E30004D6192
:10077000726C696E0020536F6674776172652052E7
:100780006573657400205761746368646F672052F5
:1007900065736574002042726F776E206F757420E8
:1007A0005265736574002045787465726E616C20C3
:1007B000526573657400506F77657255700073747D
:1007C000617274002200656E717565696E67202222
:1007D000002200656E717565696E672022007C3CA1
:1007E0003E5E2B3D3F2F5B5D3B2C2A225C00656308
:1007F000686F3A0020746F6F206C6F6E67206578A9
:1008000074727573696F6E2070726576656E74654B
:10081000640020636F6C6420657874727573696F0F
:100820006E2070726576656E7465640045303A209E
:10083000005A3A2000593A2000583A20004D5331CE
:100840002C4D53322050696E730A0024F404D920D1
:100850001BC40C5C0E9804C4095F0265077101F4A7
:1008600005F900FB04B30048048700C10369005880
:1008700003550003034500BE023A008402310053D1
:10088000022A002902250004022000E4011C00C8FD
:10089000011900AF011700980114008401130071C1
:1008A0000110006101100051010E0043010D0036DE
:1008B000010B002B010B0020010B00150109000C9E
:1008C00001090003010800FB000800F3000800EB29
:1008D000000700E4000600DE000600D8000600D293
:1008E000000600CC000500C7000500C2000500BDE1
:1008F000000400B9000400B5000400B1000400AD1C
:10090000000400A9000400A5000300A20003009F4A
:100910000004009B00030098000300950002009370
:10092000000300900003008D0002008B000300888C
:100930000002008600020084000300810002007FA4
:100940000002007D0002007B0002007900020077B7
:1009500000010076000200740002007200010071C4
:100960000002006F0002006D0001006C0002006ACE
:1009700000010069000200670001006600010065D7
:1009800000010064000200620001006100010060DB
:100990000001005F0002005D0001005C0001005BDF
:1009A0000001005A000100590001005800010057E1
:1009B00000010056000100550001005400010053E1
:1009C00000000053000100520001005100010050DE
:1009D0000001004F0001004E0000004E0001004DDC
:1009E0000001004C0001004B0000004B0001004AD8
:1009F00000010049000100480000004800010047D4
:100A000000010046000000460001004500000045CE
:100A100000010044000100430000004300010042C7
:100A200000000042000100410000004100010040C0
:100A30000001003F0000003F0001003E0000003EBA
:100A40000001003D0000003D0001003C0000003CB2
:100A50000000003C0001003B0000003B0001003AA8
:100A60000000003A000100390000003900010038A0
:100A70000000003800000038000100370000003797
:100A8000000100360000003600000036000100358D
:100A90000000003500000035000100340000003483
:100AA0000000003400010033000000330000003378
:100AB000000100320000003200000032000100316D
:100AC0000000003100000031000100300000003063
:100AD000000000300001002F0000002F0000002F58
:100AE0000000002F0001002E0000002E0000002E4C
:100AF0000001002D0000002D0000002D0000002D41
:100B00000001002C0000002C0000002C0000002C34
:100B10000001002B0000002B0000002B0000002B28
:100B20000001002A0000002A0000002A0000002A1C
:100B30000001002900000029000000290000002910
:100B40000000002900010028000000280000002803
:100B500000000028000000280001002700000027F6
:100B600000000027000000270000002700010026E9
:100B700000000026000000260000002600000026DD
:100B800000010025000000250000002500000025D0
:100B900000000025000000250001002400000024C2
:100BA00000000024000000240000002400010023B5
:100BB00000000023000000230000002300000023A9
:100BC000000000230000002300010022000000229A
:100BD000000000220000002200000022000000228D
:100BE0000001002100000021000000210000002180
:100BF0000000002100000021000000210001002071
:100C00000000002000000020000000200000002064
:100C10000000002000000020000000200001001F54
:100C20000000001F0000001F0000001F0000001F48
:100C30000000001F0000001F0001001E0000001E39
:100C40000000001E0000001E00000024F4D43050FC
:100C5000C38E20C2A24017828B7011127A910D812F
:100C60006CD90AA861E108C7586607615143061E9E
:100C70004B5D05C145A7041A411104093D98037154
:100C80003931034036DB0265339102D4305402809F
:100C90002E1D02632CEE01752AC501B028A001109B
:100CA0002781018F2564012B244B01E0223401AC04
:100CB000211F018D200D01801FFC00841EED009777
:100CC0001DDF00B81CD200E61BC600201BBC006460
:100CD0001AB200B219A8000A19A0006A189900D126
:100CE00017910040178B00B516840031167E00B3B3
:100CF0001579003A157300C7146F0058146A00EE96
:100D00001366008813630025135E00C7125B006C36
:100D100012570015125400C111510070114F0021DB
:100D2000114B00D61049008D1047004610440002B8
:100D3000104200C00F4000800F3E00420F3C0006F2
:100D40000F3B00CB0E3800930E37005C0E350027AA
:100D50000E3400F30D3200C10D3100900D300060F3
:100D60000D2E00320D2D00050D2C00D90C2B00AEE0
:100D70000C2900850C29005C0C2700350C27000E7F
:100D80000C2600E80B2400C40B2400A00B23007DDC
:100D90000B23005A0B2100390B2100180B2000F8FF
:100DA0000A1F00D90A1E00BB0A1E009D0A1D0080F2
:100DB0000A1D00630A1C00470A1B002C0A1B0011B5
:100DC0000A1A00F7091A00DD091900C4091900AB55
:100DD000091900920917007B091800630917004CD4
:100DE00009160036091600200916000A091500F533
:100DF000081500E0081400CC081400B8081400A47A
:100E0000081400900813007D0812006B08130058A6
:100E100008120046081200340811002308110012BD
:100E200008110001081100F0071000E0071000D0C1
:100E3000071000C0071000B0070F00A107100091B5
:100E4000070E0083070F0074070F0065070E005799
:100E5000070E0049070E003B070D002E070E00206D
:100E6000070D0013070D0006070D00F9060C00ED35
:100E7000060D00E0060C00D4060C00C8060C00BCF1
:100E8000060C00B0060C00A4060B0099060C008DA1
:100E9000060B0082060B0077060B006C060B006148
:100EA000060A0057060B004C060A0042060A0038E4
:100EB000060A002E060A0024060A001A060A001076
:100EC00006090007060A00FD050900F4050900EB04
:100ED000050900E2050900D9050900D0050900C788
:100EE000050900BE050900B5050800AD050800A507
:100EF0000509009C050800940508008C050800847D
:100F00000508007C050800740508006C05070065ED
:100F10000508005D050700560508004E0507004757
:100F20000507004005080038050700310507002ABD
:100F3000050700230507001C050600160507000F1E
:100F40000507000805060002050700FB040600F57A
:100F5000040700EE040600E8040600E2040700DBD4
:100F6000040600D5040600CF040600C9040600C329
:100F7000040600BD040600B7040600B1040500AC79
:100F8000040600A6040600A00405009B04060095C4
:100F9000040500900406008A04050085040500800D
:100FA0000406007A04050075040500700405006B52
:100FB00004050066040500610405005C0405005793
:100FC000040500520405004D0405004804050043D3
:100FD0000405003E0404003A040500350405003011
:100FE0000404002C04050027040400230405001E4B
:100FF0000404001A04040016040500110404000D82
:10100000040400090405000404040000040400FCB6
:10101000030400F8030400F4030400F0030400ECEC
:10102000030400E8030400E4030400E0030400DC1C
:10103000030400D8030400D4030400D0030400CC4C
:10104000030400C8030300C50303006563686F3A27
:1010500000656E6473746F7073206869743A205A07
:1010600000205A3A00656E6473746F70732068696B
:10107000743A20590020593A00656E6473746F7099
:1010800073206869743A20580020583A00656E64ED
:1010900073746F7073206869743A20004572726FC0
:1010A000723A004572723A204D415854454D5020D5
:1010B0004245440054656D706572617475726520B7
:1010C0006865617465642062656420737769746320
:1010D000686564206F66662E204D415854454D501A
:1010E000207472696767657265642021210045720A
:1010F000723A204D494E54454D50003A204578747F
:101100007275646572207377697463686564206FB3
:1011100066662E204D494E54454D502074726967C5
:1011200067657265642021004572723A204D41580E
:1011300054454D50003A20457874727564657220AC
:101140007377697463686564206F66662E204D410D
:101150005854454D50207472696767657265642004
:101160002100202D20496E76616C696420657874B9
:101170007275646572206E756D6265722021000063
:10118000000000300E0100C00E0A00500F1400D005
:101190000F1E0060102800E010320070113C00F0BB
:1011A0001146007012500000135A008013640000B2
:1011B000146E00901478001015820090158C0010A9
:1011C0001696009016A0001017AA009017B40010F1
:1011D00018BE009018C8001019D2009019DC001039
:1011E0001AE600801AF000001BFA00801B0401F0D0
:1011F0001B0E01701C1801F01C2201601D2C01E067
:101200001D3601501E4001D01E4A01401F5401B03E
:101210001F5E0130206801A020720110217C019026
:10122000218601002290016026F401902A58028054
:101230002EBC0250322003E03584035039E803808D
:101240003C4C046563686F3A0048656174696E6779
:10125000206661696C656400504944204175746F73
:1012600074756E652066696E6973686564212050C7
:10127000757420746865206C617374204B702C2029
:101280004B6920616E64204B6420636F6E737461E0
:101290006E74732066726F6D2061626F766520696F
:1012A0006E746F20436F6E66696775726174696FE3
:1012B0006E2E6800504944204175746F74756E65D8
:1012C000206661696C6564212074696D656F757451
:1012D0000020403A006F6B20543A006F6B20423A76
:1012E00000504944204175746F74756E65206661C5
:1012F000696C6564212054656D70657261747572E6
:101300006520746F6F206869676800204B643A201D
:1013100000204B693A2000204B703A200020436C9B
:1013200061737369632050494420002054753A204A
:1013300000204B753A2000206D61783A2000206D26
:10134000696E3A200020643A200020626961733A95
:1013500020004D383420582059205A20450065631C
:10136000686F3A0043616E6E6F7420656E746572CB
:10137000207375626469723A20004D3234004D3238
:1013800033202573006175746F25692E67004572DF
:10139000726F723A006572726F7220777269746947
:1013A0006E6720746F2066696C65004E6F74205301
:1013B00044207072696E74696E67002F0053442078
:1013C0007072696E74696E67206279746520002E90
:1013D0000044656C6574696F6E206661696C656454
:1013E0002C2046696C653A200046696C652064656E
:1013F0006C657465643A002E006F70656E206661DE
:10140000696C65642C2046696C653A2000577269E6
:1014100074696E6720746F2066696C653A20002ECF
:10142000006F70656E206661696C65642C2046698A
:101430006C653A20002E006F70656E206661696CE5
:1014400065642C2046696C653A200046696C65200D
:1014500073656C6563746564002053697A653A202E
:101460000046696C65206F70656E65643A20002ED9
:10147000006F70656E206661696C65642C2046693A
:101480006C653A20004E6F7720667265736820663F
:10149000696C653A20004E6F7720646F696E672033
:1014A00066696C653A20002220706F7300222070FC
:1014B0006172656E743A2200535542524F55544939
:1014C0004E452043414C4C207461726765743A224A
:1014D00000747279696E6720746F2063616C6C2090
:1014E0007375622D67636F64652066696C65732030
:1014F0007769746820746F6F206D616E79206C65F8
:1015000076656C732E204D4158206C6576656C2095
:1015100069733A0053442063617264206F6B006FFB
:1015200070656E526F6F74206661696C65640076D9
:101530006F6C756D652E696E6974206661696C6586
:101540006400534420696E6974206661696C0065AB
:1015500063686F3A0048617264636F646564204435
:10156000656661756C742053657474696E67732069
:101570004C6F616465640053746F726564207365B9
:101580007474696E677320726574726965766564D8
:10159000002044002049002020204D3330312050CD
:1015A000005049442073657474696E67733A002073
:1015B0005A0020590020204D323036205800486F04
:1015C0006D65206F666673657420286D6D293A001D
:1015D000204500205A0020580020420020540020BE
:1015E000204D323035205300416476616E6365646E
:1015F000207661726961626C65733A20533D4D6972
:101600006E20666565647261746520286D6D2F7348
:10161000292C20543D4D696E2074726176656C20D2
:10162000666565647261746520286D6D2F73292C61
:1016300020423D6D696E696D756D207365676D65DE
:101640006E742074696D6520286D73292C20583DB7
:101650006D6178696D756D205859206A65726B20CF
:10166000286D6D2F73292C20205A3D6D6178696D8E
:10167000756D205A206A65726B20286D6D2F732955
:101680002C2020453D6D6178696D756D2045206A7F
:1016900065726B20286D6D2F732900205400202067
:1016A0004D323034205300416363656C6572617460
:1016B000696F6E3A20533D616363656C6572617456
:1016C000696F6E2C20543D72657472616374206181
:1016D0006363656C65726174696F6E0020450020FC
:1016E0005A0020590020204D3230312058004D61E1
:1016F00078696D756D20416363656C6572617469AD
:101700006F6E20286D6D2F7332293A00204500201E
:101710005A0020590020204D3230332058004D61AE
:1017200078696D756D206665656472617465732096
:10173000286D6D2F73293A00204500205A0020594A
:101740000020204D3932205800537465707320708A
:10175000657220756E69743A0053657474696E67BA
:10176000732053746F72656400022D2D3A2D2D0085
:101770002D2D2D0053440020590001200001200090
:101780004E6F2053442063617264005072696E741E
:101790002066726F6D2053440053746F7020707216
:1017A000696E7400526573756D65207072696E7430
:1017B000005061757365207072696E7400436F6EBE
:1017C00074726F6C00507265706172650054756E52
:1017D0006500496E666F2073637265656E00052E45
:1017E0002E004D61696E004D3234004D323320259C
:1017F00073004D383420582059205A20450046693E
:10180000726D776172652076657273696F6E0052D2
:101810006573746F7265206661696C7361666500DB
:101820004C6F6164206D656D6F72790053746F72D7
:1018300065206D656D6F7279004D6F74696F6E0014
:1018400054656D7065726174757265004D61696E85
:101850000053657020313920323031342031303A34
:1018600032323A3335003235303030305F73696EA2
:10187000676C6500556C74696D616B65723A2031F7
:10188000342E3038004669726D7761726520766556
:101890007273696F6E004573746570732F6D6D00A0
:1018A0004573746570732F6D6D005A737465707332
:1018B0002F6D6D005A73746570732F6D6D005973C1
:1018C000746570732F6D6D005973746570732F6D2F
:1018D0006D005873746570732F6D6D005873746567
:1018E00070732F6D6D00412D7265747261637400A9
:1018F000412D7265747261637400416D6178206579
:1019000000416D6178206500416D6178207A004169
:101910006D6178207A00416D6178207900416D61B8
:1019200078207900416D6178207800416D617820E0
:1019300078005654726176206D696E00565472615B
:1019400076206D696E00566D696E00566D696E0089
:10195000566D6178206500566D6178206500566D82
:101960006178207A00566D6178207A00566D617832
:10197000207900566D6178207900566D6178207865
:1019800000566D617820780056652D6A65726B008F
:1019900056652D6A65726B00567A2D6A65726B000A
:1019A000567A2D6A65726B005678792D6A65726B6E
:1019B000005678792D6A65726B00416363656C002F
:1019C000416363656C00436F6E74726F6C0050729C
:1019D00065686561742041425320636F6E660050F4
:1019E00072656865617420504C4120636F6E6600BB
:1019F0005049442D43005049442D43005049442D43
:101A000044005049442D44005049442D4900504958
:101A1000442D49005049442D50005049442D500058
:101A200046616E2073706565640046616E20737058
:101A30006565640042656400426564004E6F7A7AB1
:101A40006C65004E6F7A7A6C6500436F6E74726FCE
:101A50006C0053746F7265206D656D6F7279004212
:101A6000656400426564004E6F7A7A6C65004E6F63
:101A70007A7A6C650046616E207370656564004615
:101A8000616E2073706565640054656D7065726188
:101A9000747572650053746F7265206D656D6F7239
:101AA000790042656400426564004E6F7A7A6C6525
:101AB000004E6F7A7A6C650046616E2073706565C2
:101AC000640046616E2073706565640054656D70D6
:101AD00065726174757265004D6F76652061786915
:101AE0007300436F6F6C646F776E0050726568654A
:101AF00061742041425300507265686561742050E2
:101B00004C41004D6F7665205A004175746F206816
:101B10006F6D65004D38340044697361626C6520F7
:101B20007374657070657273004D61696E004D6FFE
:101B3000766520302E316D6D004D6F766520316DEC
:101B40006D004D6F76652031306D6D00507265709F
:101B5000617265004578747275646572004D6F76C8
:101B600065205A004D6F76652059004D6F766520CF
:101B700058004D6F766520617869730045787472FE
:101B800075646572005A00590058005072656865A6
:101B9000617420414253204265640050726568655B
:101BA000617420414253203100507265706172654A
:101BB000005072656865617420504C412042656434
:101BC000005072656865617420504C4120310050AE
:101BD000726570617265005A004D383420583020AB
:101BE000593000473238004D363030004368616E5E
:101BF00067652066696C616D656E7400466C6F7711
:101C000000466C6F770046616E20737065656400F6
:101C100046616E20737065656400426564004265CC
:101C200064004E6F7A7A6C65004E6F7A7A6C65004C
:101C30005370656564005370656564004D61696E3D
:101C400000436172642072656D6F76656400436164
:101C5000726420696E73657274656400494E46490A
:101C60004E4954594E414ECDCCCC3D0AD7233C175A
:101C7000B7D13877CC2B329595E6241FB14F0A00A7
:101C80000020410000C84200401C4620BCBE4CCA97
:101C90001B0E5AAEC59D7400631ADE3F31CA5C1A32
:101CA00011241FBECFEFD1E2DEBFCDBF00E00CBFDD
:101CB00014E0A0E0B2E0E8E8F2EB01E00BBF02C004
:101CC00007900D92A83AB107D9F71BBE12E1A8EA16
:101CD000B4E001C01D92AB34B107E1F71CE1CEE9DD
:101CE000DCE104C02297FE010E94E9D8C839D1077F
:101CF000C9F70E94C9D30C9437D90C940000A0E016
:101D0000B0E0E5E8FEE00C9406D9EC015B0161155A
:101D1000710519F0FB0191838083F9908F2D90E07C
:101D20000E94EDD8892BC9F7FDE2FF1621F4F99046
:101D3000EE24E39405C02BE2F21609F4F990EE24A8
:101D40008E0101501040C8016CE57CE143E050E099
:101D50000E941511892B01F58E010E5F1F4FC801DE
:101D60006FE57CE145E050E00E941511892B19F4E4
:101D70008E01095F1F4FA114B10419F0F501118301
:101D80000083E0FC04C070E090E080E814C070E0E4
:101D900090E080E86FEF08C1C80164E67CE143E0B1
:101DA00050E00E941511892B69F4A114B10429F4A3
:101DB00070E090E080EC6FE7F7C02296F501D183E8
:101DC000C083F6CF8824992440E050E060E070E0C2
:101DD000EF2DE053EA30A0F5F2E0EF2A8E2D90E0EF
:101DE0009C0128703070E2FE06C0232B79F5089420
:101DF000811C911C2BC0232B19F008948108910899
:101E0000DB01CA0112E0880F991FAA1FBB1F1A9598
:101E1000D1F7480F591F6A1F7B1F440F551F661FBC
:101E2000771F4E0F511D611D711D483929E9520759
:101E300029E9620729E1720748F084E0E82A06C030
:101E4000EE3F31F4E3FC39C098E0E92AF990C0CFC5
:101E5000E53311F0E53189F529912D3219F4E0E1EE
:101E6000EE2A05C02B3219F081E090E003C02991E1
:101E700082E090E0E22FE053EA3018F0C81BD90B63
:101E80001CC020E030E0FCE020383F075CF4C901D2
:101E9000880F991F880F991F280F391F220F331F92
:101EA0002E0F311DE991E053EA3068F3E4FE03C0E0
:101EB000309521953F4F820E931ECE2CDD24E1FEFE
:101EC00007C0A114B10421F02197F501D183C0838B
:101ED000CB01BA010E9452D57B018C01F3E0CF22E5
:101EE000DD2423E0C216D10421F417FB109517F965
:101EF000109557016801C801B70120E030E040E0CB
:101F000050E00E94B2D4882309F44AC097FE0DC065
:101F10002BE7E22E2CE1F22E909481949108939479
:101F2000C0E2D0E000E010E012C093E9E92E9CE1AD
:101F3000F92EF6CFF7012591359145915491C601BF
:101F4000B5010E9492D75B016C018C1A9D0A8C1618
:101F50009D0684F7D595C7950F5F1F4F0630110575
:101F600029F08CEF9FEFE80EF91EF1CFC501D601E5
:101F70007C018D018C2D880F8D2D881F8F3F51F096
:101F8000C601B50120E030E040E050E00E94B2D44C
:101F9000882331F482E290E090934A1280934912B0
:101FA0007E2D9F2D802F612F272F392F482F562FC1
:101FB000B901CA01CDB7DEB7ECE00C9422D92F925B
:101FC0003F925F926F927F928F929F92AF92BF9259
:101FD000CF92DF92EF92FF920F931F93CF93DF93F5
:101FE0008C011B01EA016115710519F0FB01918358
:101FF0008083209749F0CE010297839728F020E054
:1020000030E040E050E0F6C0F801A1908F018A2D49
:1020100090E00E94EDD8892BB9F7FDE2AF1631F4BC
:10202000F801A1908F015524539407C0FBE2AF162D
:1020300019F4F801A1908F015524209719F0C031AF
:10204000D105C1F4F0E3AF1679F4F8018081883747
:1020500011F0883549F4F801A1800E5F1F4FF2E0BE
:102060005F2AC0E1D0E006C0209721F480E3A816E3
:10207000E9F427C0C830D10531F1C930D10524F4C5
:10208000C230D10531F50CC0CA30D10589F0C0315C
:10209000D105F9F4C12CD12CE12CB8E0FB2E28C0DD
:1020A000C12CD12CE12CA0E4FA2E22C0CAE0D0E051
:1020B000FCECCF2EFCECDF2EFCECEF2EFCE0FF2E38
:1020C00017C0C8E0D0E0C12CD12CE12CE0E1FE2EFD
:1020D0000FC09E01442737FD4095542F60E070E00B
:1020E00080E090E80E94AAD8C901DA016C017D0164
:1020F00020E030E040E050E060E03E01882477FCE2
:102100008094982C70EDB72EBA0CE9E0EB1570F4C2
:102110008A2D81548A3118F499ECB92E06C08A2D83
:1021200081568A3150F589EAB82EBA0C8B2D90E091
:102130008C179D0714F56F3FE1F0C216D306E40635
:10214000F506B0F0CA01B901A40193010E9464D858
:102150009B01AC012B0D311D411D511D2130F0E0C3
:102160003F07F0E04F07F0E85F0710F461E001C0BF
:102170006FEFF801A1908F01C5CF2114310481F0D8
:10218000662331F001501040F1011183008308C033
:1021900051FE1AC002501040F1011183008314C097
:1021A00067FF12C050FC05C02FEF3FEF4FEF5FE716
:1021B00004C020E030E040E050E882E290E09093FC
:1021C0004A128093491216C050FE08C0509540959F
:1021D000309521953F4F4F4F5F4F0CC057FF0AC0BE
:1021E00082E290E090934A12809349122FEF3FEFE2
:1021F0004FEF5FE7B901CA01DF91CF911F910F91B6
:10220000FF90EF90DF90CF90BF90AF909F908F9016
:102210007F906F905F903F902F900895FB01DC01BD
:1022200005900D920020E1F70895FB01DC0141507B
:10223000504088F08D9181341CF08B350CF4805E19
:10224000659161341CF06B350CF4605E861B611186
:1022500071F3990B0895881BFCCFFB01DC01415001
:10226000504048F005900D920020C9F701C01D9222
:1022700041505040E0F70895FB0155915523A9F0D6
:10228000BF01DC014D9145174111E1F759F4CD0132
:102290000590002049F04D9140154111C9F3FB0113
:1022A0004111EFCF81E090E001970895FB01DC013F
:1022B00004C08D910190801921F441505040C8F71D
:1022C000881B990B0895FB01DC0102C001900D925F
:1022D00041505040D8F70895FB01DC010D900020DB
:1022E000E9F7119701900D920020E1F70895FC01A4
:1022F0008191861721F08823D9F79927089531977E
:10230000CF010895FB01DC0101900D920020E1F75F
:102310000895FB01DC014150504030F08D91019057
:10232000801919F40020B9F7881B990B0895FB0157
:10233000DC014150504048F001900D920020C9F757
:1023400001C01D9241505040E0F70895AEE0B0E06A
:10235000ECEAF1E10C940ED90E891F898EE08C8392
:102360001A8309838FEF9FE79E838D839E01265EEC
:102370003F4FCE010196688D798DA9010E94CA1147
:102380002F813885020F131FF80110822E96E4E08A
:102390000C942AD9ABE0B0E0E0EDF1E10C9400D967
:1023A0003C012B015A01FC0117821682838181FDB9
:1023B00003C06FEF7FEFC6C19AE0892E1E0108941B
:1023C000211C311CF3012381F20123FD859123FFA0
:1023D00081912F01882309F4B2C1853239F423FD9C
:1023E000859123FF81912F01853229F490E0B3017B
:1023F0000E94BD13E7CF982FFF24EE249924FFE11C
:10240000FF15D0F09B3269F09C3228F4903259F0DD
:10241000933291F40EC09D3249F0903369F441E05B
:1024200024C052E0F52A84E0F82A28C098E0F92A6E
:1024300025C0E0E1FE2A22C0F7FC29C0892F805385
:102440008A3070F4F6FE05C0989C902C1124980EEA
:1024500015C0E89CE02C1124E80EF0E2FF2A0EC023
:102460009E3229F4F6FC6BC140E4F42A07C09C3686
:1024700019F450E8F52A02C0983649F4F20123FD18
:10248000959123FF91912F01992309F0B8CF892FBE
:102490008554833018F08052833038F444E050E0A3
:1024A000A40EB51E5FE359830FC0933631F0933706
:1024B00079F0933509F056C020C0F50180818983F9
:1024C00042E050E0A40EB51E610101E010E012C030
:1024D000F501C080D180F6FC03C06FEF7FEF02C032
:1024E000692D70E042E050E0A40EB51EC6010E94C6
:1024F000B2138C015FE7F52214C0F501C080D180D2
:10250000F6FC03C06FEF7FEF02C0692D70E042E080
:1025100050E0A40EB51EC6010E94A7138C0150E81E
:10252000F52AF3FE07C01AC080E290E0B3010E94D2
:10253000BD13EA948E2D90E008171907A8F30EC07A
:10254000F601F7FC8591F7FE81916F0190E0B301F0
:102550000E94BD13E110EA940150104001151105CD
:1025600079F7EAC0943611F0993669F5F7FE08C09C
:10257000F501208131814281538184E090E00AC0DD
:10258000F501808191819C01442737FD4095542FAE
:1025900082E090E0A80EB91E9FE6F92257FF09C01D
:1025A00050954095309521953F4F4F4F5F4FE0E854
:1025B000FE2ACA01B901A1012AE030E00E94E91314
:1025C000D82ED21840C0953729F41F2D1F7E2AE03F
:1025D00030E01DC01F2D197F9F3661F0903720F429
:1025E000983509F0ACC00FC0903739F0983709F032
:1025F000A6C004C028E030E00AC0106114FD1460D9
:1026000020E130E004C014FD166020E132E017FF45
:1026100008C0F501608171818281938144E050E0BE
:1026200008C0F50180819181BC0180E090E042E02A
:1026300050E0A40EB51EA1010E94E913D82ED218B5
:102640008FE7F82EF122F6FE0BC05EEFF522D914CB
:1026500038F4F4FE07C0F2FC05C08FEEF82202C089
:102660001D2D01C0192DF4FE0DC0FE01ED0DF11D53
:102670008081803319F499EEF92208C01F5FF2FEC1
:1026800005C003C08F2D867809F01F5F0F2DF3FC66
:1026900014C0F0FE0FC01E1510F09D2C0BC09D2C19
:1026A0009E0C911A1E2D06C080E290E0B3010E949C
:1026B000BD131F5F1E15C0F304C01E1510F4E11AF0
:1026C00001C0EE2404FF0FC080E390E0B3010E943C
:1026D000BD1302FF1DC001FD03C088E790E00EC0DE
:1026E00088E590E00BC0802F867891F001FF02C052
:1026F0008BE201C080E2F7FC8DE290E0B3010E9422
:10270000BD1306C080E390E0B3010E94BD139A940C
:10271000D914C0F3DA94F101ED0DF11D808190E040
:10272000B3010E94BD13DD20A9F706C080E290E04E
:10273000B3010E94BD13EA94EE20C1F743CEF3012A
:1027400066817781CB012B96E2E10C941CD9FC01C8
:102750000590615070400110D8F7809590958E0FCC
:102760009F1F0895FC016150704001900110D8F73F
:10277000809590958E0F9F1F08950F931F93CF9371
:10278000DF938C01EB018B8181FF1BC082FF0DC0A9
:102790002E813F818C819D812817390764F4E8815F
:1027A000F9810193F983E88306C0E885F985802FD4
:1027B0001995892B31F48E819F8101969F838E8399
:1027C00002C00FEF1FEFC801DF91CF911F910F9152
:1027D0000895FA01AA27283051F1203181F1E894B7
:1027E0006F936E7F6E5F7F4F8F4F9F4FAF4FB1E004
:1027F0003ED0B4E03CD0670F781F891F9A1FA11DFF
:10280000680F791F8A1F911DA11D6A0F711D811DFF
:10281000911DA11D20D009F468943F912AE0269FC4
:1028200011243019305D3193DEF6CF010895462F23
:102830004770405D4193B3E00FD0C9F7F6CF462F04
:102840004F70405D4A3318F0495D31FD405241936D
:1028500002D0A9F7EACFB4E0A6959795879577952A
:102860006795BA95C9F700976105710508959B01B1
:10287000AC010A2E06945795479537952795BA953A
:10288000C9F7620F731F841F951FA01D08951F9223
:102890000F920FB60F9211242F933F938F939F9314
:1028A000AF93BF938091AC049091AD04A091AE041E
:1028B000B091AF043091B0040196A11DB11D232F3A
:1028C0002D5F2D3720F02D570196A11DB11D2093AE
:1028D000B0048093AC049093AD04A093AE04B09385
:1028E000AF048091A8049091A904A091AA04B0918A
:1028F000AB040196A11DB11D8093A8049093A90477
:10290000A093AA04B093AB04BF91AF919F918F9114
:102910003F912F910F900FBE0F901F9018958FB77A
:10292000F8942091AC043091AD044091AE045091E4
:10293000AF048FBFB901CA0108959B01AC017FB7F5
:10294000F8948091A8049091A904A091AA04B09150
:10295000AB0466B5A89B05C06F3F19F00196A11D99
:10296000B11D7FBFBA2FA92F982F8827860F911DE1
:10297000A11DB11D62E0880F991FAA1FBB1F6A9598
:10298000D1F7BC012DC0FFB7F8948091A8049091B5
:10299000A904A091AA04B091AB04E6B5A89B05C018
:1029A000EF3F19F00196A11DB11DFFBFBA2FA92F4E
:1029B000982F88278E0F911DA11DB11DE2E0880F71
:1029C000991FAA1FBB1FEA95D1F7861B970B885E3C
:1029D0009340C8F2215030404040504068517C4FF5
:1029E000211531054105510571F60895019739F01A
:1029F000880F991F880F991F02970197F1F7089583
:102A0000789484B5826084BD84B5816084BD85B5C9
:102A1000826085BD85B5816085BDEEE6F0E0808190
:102A200081608083E1E8F0E01082808182608083B1
:102A3000808181608083E0E8F0E080818160808334
:102A4000E1EBF0E0808184608083E0EBF0E0808166
:102A500081608083E1E9F0E0808182608083808111
:102A600081608083E0E9F0E0808181608083E1EA39
:102A7000F0E0808182608083808181608083E0EAF1
:102A8000F0E0808181608083E1E2F1E0808182601A
:102A90008083808181608083E0E2F1E080818160D9
:102AA0008083EAE7F0E080818460808380818260B7
:102AB00080838081816080838081806880831092A0
:102AC000C10008951F93CF93DF93182FEB0161E0AE
:102AD0000E944216209709F4CAC0CF3FD10509F4DD
:102AE000C9C0E12FF0E0E75FFD4F8491893009F420
:102AF00066C08A30B0F48430F1F1853040F4823021
:102B000059F1833070F5813009F0AEC020C08730B4
:102B100009F443C0883008F048C0863009F0A4C0EA
:102B200034C08D3009F478C08E3038F48B3009F41D
:102B30005AC08C3008F066C04CC0803109F480C0A7
:102B4000813109F487C08F3009F08EC06FC084B521
:102B5000806884BDC7BD92C084B5806284BDC8BD95
:102B60008DC080918000806880938000D093890020
:102B7000C093880083C08091800080628093800031
:102B8000D0938B00C0938A0079C08091B000806898
:102B90008093B000C093B30071C08091B000806298
:102BA0008093B000C093B40069C0809190008068A9
:102BB00080939000D0939900C09398005FC080915B
:102BC0009000806280939000D0939B00C0939A0005
:102BD00055C080919000886080939000D0939D00B4
:102BE000C0939C004BC08091A00080688093A0009F
:102BF0008091A0008F7B8093A000D093A900C09308
:102C0000A8003CC08091A00080628093A000D09377
:102C1000AB00C093AA0032C08091A000886080936E
:102C2000A000D093AD00C093AC0028C080912001DB
:102C3000806880932001D0932901C09328011EC091
:102C400080912001806280932001D0932B01C0935A
:102C50002A0114C080912001886080932001D093C4
:102C60002D01C0932C010AC0C038D1051CF4812F5E
:102C700060E002C0812F61E00E94F516DF91CF91E4
:102C80001F910895CF93DF93482F50E0CA018D53D1
:102C90009E4FFC01349143585E4FFA018491882382
:102CA00069F190E0880F991FFC01E15DFE4FA5914D
:102CB000B491FC01E75BFE4FC591D491662351F4BA
:102CC0002FB7F8948C91932F909589238C938881BA
:102CD00089230BC0623061F42FB7F8948C91932F45
:102CE000909589238C938881832B88832FBF06C07E
:102CF0009FB7F8948C91832B8C939FBFDF91CF91DA
:102D00000895893009F449C08A30A0F4843051F123
:102D1000853040F4823079F1833000F5813009F05C
:102D200063C026C0873079F1883098F5863009F085
:102D30005BC025C08D3009F442C08E3028F48B3042
:102D4000B1F18C30C0F52DC0803109F442C0813121
:102D500009F445C08F3009F047C037C0809180002A
:102D60008F7703C0809180008F7D809380000895CD
:102D700084B58F7702C084B58F7D84BD089580911E
:102D8000B0008F7703C08091B0008F7D8093B0003A
:102D90000895809190008F7707C0809190008F7D7B
:102DA00003C080919000877F809390000895809168
:102DB000A0008F7707C08091A0008F7D03C0809115
:102DC000A000877F8093A0000895809120018F77D5
:102DD00003C0809120018F7D809320010895809110
:102DE0002001877F809320010895FF920F931F9306
:102DF000F62E482F50E0CA01875F9D4FFC012491B9
:102E0000CA018D539E4FFC01149143585E4FFA0145
:102E100004910023C9F0222319F0822F0E94811609
:102E2000E02FF0E0EE0FFF1FE75BFE4FA591B4919E
:102E30009FB7F894FF2021F48C911095812302C054
:102E40008C91812B8C939FBF1F910F91FF900895C0
:102E50000F931F93482F50E0CA01875F9D4FFC01DD
:102E60002491CA018D539E4FFC01049143585E4F3B
:102E7000FA011491112319F420E030E015C0222347
:102E800019F0822F0E948116812F90E0880F991FE0
:102E90008D599E4FFC01A591B4918C9120E030E0BA
:102EA000802311F021E030E0C9011F910F910895B6
:102EB0001F920F920FB60F920BB60F9211242F9301
:102EC0003F934F935F936F937F938F939F93AF93B2
:102ED000BF93EF93FF938091B5049091B604892B33
:102EE00029F0E091B504F091B6041995FF91EF91A6
:102EF000BF91AF919F918F917F916F915F914F9112
:102F00003F912F910F900BBE0F900FBE0F901F900F
:102F100018951F920F920FB60F920BB60F921124B5
:102F20002F933F934F935F936F937F938F939F93D1
:102F3000AF93BF93EF93FF938091B7049091B80440
:102F4000892B29F0E091B704F091B8041995FF910D
:102F5000EF91BF91AF919F918F917F916F915F9111
:102F60004F913F912F910F900BBE0F900FBE0F907E
:102F70001F9018951F920F920FB60F920BB60F92DB
:102F800011242F933F934F935F936F937F938F936E
:102F90009F93AF93BF93EF93FF938091B904909168
:102FA000BA04892B29F0E091B904F091BA0419957B
:102FB000FF91EF91BF91AF919F918F917F916F9111
:102FC0005F914F913F912F910F900BBE0F900FBECD
:102FD0000F901F9018951F920F920FB60F920BB67D
:102FE0000F9211242F933F934F935F936F937F938F
:102FF0008F939F93AF93BF93EF93FF938091BB0405
:103000009091BC04892B29F0E091BB04F091BC04A1
:103010001995FF91EF91BF91AF919F918F917F9102
:103020006F915F914F913F912F910F900BBE0F9039
:103030000FBE0F901F9018951F920F920FB60F9210
:103040000BB60F9211242F933F934F935F936F937F
:103050007F938F939F93AF93BF93EF93FF93809151
:10306000B1049091B204892B29F0E091B104F09160
:10307000B2041995FF91EF91BF91AF919F918F91FC
:103080007F916F915F914F913F912F910F900BBE68
:103090000F900FBE0F901F9018951F920F920FB6B2
:1030A0000F920BB60F9211242F933F934F935F9380
:1030B0006F937F938F939F93AF93BF93EF93FF9300
:1030C0008091B3049091B404892B29F0E091B3046A
:1030D000F091B4041995FF91EF91BF91AF919F9139
:1030E0008F917F916F915F914F913F912F910F90B1
:1030F0000BBE0F900FBE0F901F9018951F920F924E
:103100000FB60F920BB60F9211242F933F934F934C
:103110005F936F937F938F939F93AF93BF93EF933F
:10312000FF938091BD049091BE04892B29F0E0911A
:10313000BD04F091BE041995FF91EF91BF91AF913D
:103140009F918F917F916F915F914F913F912F91BF
:103150000F900BBE0F900FBE0F901F9018951F92EF
:103160000F920FB60F920BB60F9211242F933F932D
:103170004F935F936F937F938F939F93AF93BF937F
:10318000EF93FF938091BF049091C004892B29F0A5
:10319000E091BF04F091C0041995FF91EF91BF91A8
:1031A000AF919F918F917F916F915F914F913F91DF
:1031B0002F910F900BBE0F900FBE0F901F90189580
:1031C000CF92DF92EF92FF920F931F93CF93DF93F3
:1031D0007C016B018A01C0E0D0E00FC0D6016D9187
:1031E0006D01D701ED91FC910190F081E02DC701B7
:1031F0001995C80FD91F015010400115110571F71D
:10320000CE01DF91CF911F910F91FF90EF90DF9052
:10321000CF900895DC01ED91FC910190F081E02DBB
:1032200019950895CF93DF93EC016115710519F499
:1032300020E030E00FC0DB010D900020E9F711978E
:10324000A61BB70BE881F9810280F381E02DAD0167
:1032500019959C01C901DF91CF9108950E9412191F
:103260000895EF92FF920F931F93CF93DF93EC019A
:10327000E0907007F090710700917207109173074A
:10328000688179818A819B81A80197010E94B2D4CB
:10329000882324F4E882F9820A831B83E090740770
:1032A000F090750700917607109177076C817D810A
:1032B0008E819F81A80197010E94B2D4882324F4B3
:1032C000EC82FD820E831F83E0907807F0907907EF
:1032D00000917A0710917B07688579858A859B859F
:1032E000A80197010E94B2D4882324F4E886F986C5
:1032F0000A871B87E0908903F0908A0300918B0373
:1033000010918C03688179818A819B81A801970142
:103310000E94C0D6181624F4E882F9820A831B831F
:10332000E0908D03F0908E0300918F031091900335
:103330006C817D818E819F81A80197010E94C0D6FA
:10334000181624F4EC82FD820E831F83E090910313
:10335000F09092030091930310919403688579850E
:103360008A859B85A80197010E94C0D6181624F46F
:10337000E886F9860A871B87DF91CF911F910F910D
:10338000FF90EF90089580918E0708956770707098
:10339000E82FF0E0E75FFD4F84918B3028F4883010
:1033A000A0F4863090F106C08E30D0F08F5083307C
:1033B00060F521C08091B100887F8093B100809139
:1033C000B100862B8093B100089580919100887F91
:1033D0008093910080919100862B809391000895B5
:1033E0008091A100887F8093A1008091A100862B0D
:1033F0008093A100089580912101887F809321010D
:1034000080912101862B8093210108950F931F93B2
:10341000CF93DF938130910549F46F5F7F4F09F0BF
:1034200046C081EC94E00E947A8941C0892B09F062
:103430003EC06F5F7F4FD9F580E294E090938C0699
:1034400080938B0680919206882321F08FE896E086
:103450000E94C345C7E4D6E000E214E005C06F97C0
:1034600085E0C131D80751F0198308838F81882303
:10347000B1F3CE0104960E94C345F1CF80E294E0FF
:10348000998388838F81882321F0CE0104960E943E
:10349000C34580E294E09093F1048093F00480911E
:1034A000F704882321F084EF94E00E94C345DF9164
:1034B000CF911F910F91089580E090E06FEF7FEF23
:1034C0000E94061A089581E090E06FEF7FEF0E945E
:1034D000061A08950E94867180918E07882309F04C
:1034E0003AC081E080938E07809191079091920776
:1034F000A0919307B09194078093950790939607B6
:10350000A0939707B0939807E5E5F2E0949108C07F
:103510008091C00085FFFCCF9093C60031969491B6
:103520009923B1F7E6E6F2E0949108C08091C000DB
:1035300085FFFCCF9093C600319694919923B1F703
:103540008091C00085FFFCCF8AE08093C6008CE5A7
:1035500092E00E946ECA0895F8940E948671159AAE
:1035600010927C07469A10927D07439A10927E072C
:10357000409AE5E5F2E0949108C08091C00085FF93
:10358000FCCF9093C600319694919923B1F7E5EE64
:10359000F2E0949108C08091C00085FFFCCF909329
:1035A000C600319694919923B1F78091C00085FFB0
:1035B000FCCF8AE08093C6008CED92E00E947DCA29
:1035C000FFCF0E948F146093990770939A0780939E
:1035D0009B0790939C07E091C207F091C307EC53BF
:1035E000F84F80818823A9F4E4E0F3E0949108C0C7
:1035F0008091C00085FFFCCF9093C60031969491D6
:103600009923B1F78091C00085FFFCCF8AE08093B9
:10361000C60008950E948F146093990770939A07CB
:1036200080939B0790939C070895EF92FF920F93CE
:103630001F930E948F14E0909D07F0909E070091C9
:103640009F071091A0072091990730919A07409108
:103650009B0750919C07621B730B840B950BE6161E
:10366000F7060807190738F4E114F10401051105FC
:1036700011F00E94AC1A8091970390919803A09149
:103680009903B0919A030097A105B10559F10E94E1
:103690008F142091990730919A0740919B07509180
:1036A0009C07621B730B840B950B20919703309141
:1036B00098034091990350919A03261737074807BA
:1036C000590780F490912D1180912E11981751F483
:1036D000159A10927C07469A10927D07439A109291
:1036E0007E07409A0E94A4581F910F91FF90EF907F
:1036F00008956F927F928F929F92AF92BF92CF92D6
:10370000DF92EF92FF920F931F93F82E6091A10723
:103710007091A2078091A3079091A4072091A5071B
:103720003091A6074091A7075091A8070E94CDD6D7
:103730003B014C0100D000D00DB71EB70F5F1F4FEB
:1037400060917F0370918003882777FD8095982F83
:103750000E9454D520919B0330919C0340919D037E
:1037600050919E030E9492D720E030E040E752E45F
:103770000E94B9D420E030E048EC52E40E94B9D471
:103780005B016C01F8016082718282829382F48213
:1037900080918307858384E597E06DEA77E041EACD
:1037A00057E020E001E032E0E32E0E94A452809135
:1037B000AD079091AE07A091AF07B091B00780938D
:1037C000540790935507A0935607B09357078091DD
:1037D000B1079091B207A091B307B091B40780935D
:1037E000580790935907A0935A07B0935B078091AD
:1037F000B5079091B607A091B707B091B80780932D
:103800005C0790935D07A0935E07B0935F0780917C
:10381000B9079091BA07A091BB07B091BC078093FC
:10382000600790936107A0936207B09363078DB719
:103830009EB706960FB6F8949EBF0FBE8DBF0E942E
:103840008F146093990770939A0780939B079093C6
:103850009C071F910F91FF90EF90DF90CF90BF904A
:10386000AF909F908F907F906F900895CF92DF924E
:10387000EF92FF920F931F938DEA97E00E94311908
:103880000E948F146093990770939A0780939B0707
:1038900090939C076091540770915507809156074B
:1038A000909157072091AD073091AE074091AF0737
:1038B0005091B0070E94B2D4882309F07AC0609179
:1038C00058077091590780915A0790915B07209192
:1038D000B1073091B2074091B3075091B4070E94ED
:1038E000B2D4882309F065C060919B0370919C035A
:1038F00080919D0390919E0320E030E040E752E4E8
:103900000E94B9D47B018C018DEA97E061EB77E0EE
:1039100045EB57E029EB37E0E3E8CE2EE7E0DE2E7B
:103920000E948B5B8091AD079091AE07A091AF078D
:10393000B091B0078093540790935507A093560712
:10394000B09357078091B1079091B207A091B30748
:10395000B091B4078093580790935907A0935A07E2
:10396000B0935B078091B5079091B607A091B70718
:10397000B091B80780935C0790935D07A0935E07B2
:10398000B0935F078091B9079091BA07A091BB07E8
:10399000B091BC078093600790936107A093620782
:1039A000B09363071F910F91FF90EF90DF90CF903E
:1039B000089560917F0370918003882777FD80953B
:1039C000982F0E9454D520919B0330919C034091E5
:1039D0009D0350919E030E9492D720E030E040E783
:1039E00052E40E94B9D420E030E048EC52E488CFA1
:1039F0008FED99E00E94D53FE7E0F3E0949108C095
:103A00008091C00085FFFCCF9093C60031969491C1
:103A10009923B1F7409191075091920760919307D4
:103A2000709194074F5F5F4F6F4F7F4F8FED99E01D
:103A30002AE030E00E9496408091C00085FFFCCFD4
:103A40008AE08093C6000E94E11A08952F923F9267
:103A50004F925F926F927F928F929F92AF92BF929E
:103A6000CF92DF92EF92FF920F931F93DF93CF934A
:103A7000CDB7DEB728970FB6F894DEBF0FBECDBF27
:103A800098878F838330910508F056C1FC01E15C73
:103A9000FA4FD4903C01660C771C660C771C93019E
:103AA0002C5A384F3A83298380E090E0A0E0B0E0C0
:103AB000F90180839183A283B38384E597E068E56D
:103AC00077E04CE557E020E637E00E947C56F301B2
:103AD000EE5BFA4FE590F590059114916D2D7727E7
:103AE00067FD7095882777FD8095982F0E9454D5A3
:103AF0001B012C0193012355384F3C832B83C801B4
:103B0000B70120E030E040EC5FE30E9492D7A201D1
:103B100091010E9492D7AB81BC816D937D938D936F
:103B20009C931397F301E159FC4FFE83ED83608171
:103B300071818281938160939B0370939C03809336
:103B40009D0390939E0320E030E040E752E40E9402
:103B5000B9D47B018C018DEA97E061EB77E045EB0E
:103B600057E029EB37E0A3E8CA2EA7E0DA2E0E943F
:103B70008B5B0E948A6980E090E0A0E0B0E0E98180
:103B8000FA8180839183A283B38384E597E068E51B
:103B900077E04CE557E020E637E00E947C56F301E1
:103BA000EE58FA4F85909590A590B490C501B40158
:103BB0009058A20191010E9492D7AB81BC816D9374
:103BC0007D938D939C93139760919B0370919C03BD
:103BD00080919D0390919E0320E030E040E752E405
:103BE0000E94B9D47B018C018DEA97E061EB77E00C
:103BF00045EB57E029EB37E00E948B5B0E948A6916
:103C0000C501B401A50194010E94D9D3A20191017B
:103C10000E9492D7EB81FC816083718382839383BE
:103C2000AD81BE816D917D918D919C9120E030E0C0
:103C300040E05FE30E9492D760939B0370939C03E4
:103C400080939D0390939E0320E030E040E752E490
:103C50000E94B9D47B018C018DEA97E061EB77E09B
:103C600045EB57E029EB37E00E948B5B0E948A69A5
:103C7000F301E25BFA4F6591759185919491F3019F
:103C8000EC59F84FA080B180C280D380A601950185
:103C90000E94D9D37B018C01CB01D801E981FA8143
:103CA00080839183A283B383F301E65AFA4F65912F
:103CB000759185919491F0E78F2EF7E09F2E860CF9
:103CC000971CA60195010E94D9D3D4016D937D93D1
:103CD0008D939C931397F301EA59FA4F659175916F
:103CE00085919491E9E8F3E06E0E7F1EA60195019F
:103CF0000E94D9D3D3016D937D938D939C93139799
:103D0000C701D801EB81FC8180839183A283B383B7
:103D100080E090E0A0E0B0E080939B0390939C0350
:103D2000A0939D03B0939E030E940E68AF81B88557
:103D3000A458B84F81E08C9328960FB6F894DEBF54
:103D40000FBECDBFCF91DF911F910F91FF90EF90EC
:103D5000DF90CF90BF90AF909F908F907F906F90AB
:103D60005F904F903F902F900895682F2091C20749
:103D70003091C30780E690E0AC01249FC001259FED
:103D8000900D349F900D11248253984F70E00E9443
:103D900077119C019093CD078093CC0780E0232B73
:103DA00009F081E00895FC01949108C08091C00061
:103DB00085FFFCCF9093C600319694919923B1F77B
:103DC0008FED99E022E030E00E94A6410895FC01C9
:103DD000949108C08091C00085FFFCCF9093C600ED
:103DE000319694919923B1F78FED99E02AE030E074
:103DF0000E94774008958091CC079091CD0701965D
:103E000060E070E04AE050E00E94DF0F089580918A
:103E1000CC079091CD07019660E070E00E947F0E84
:103E20000895CF93DF93EC018091830780939007EF
:103E300084E50E94B51E882309F482C00E94071FF2
:103E40000E9426D5262F60939007662309F478C038
:103E5000EFE4F2E0949108C08091C00085FFFCCFB0
:103E60009093C600319694919923B1F7CD36D10540
:103E7000C1F0CE36D10544F4C836D105C1F0C936FB
:103E8000D10509F04DC010C0CA3DD10539F0CD3D76
:103E9000D10509F045C0E0E0F2E03FC0E7E1F2E023
:103EA00031C0EEE2F2E023C0E5E4F2E015C0ECE55B
:103EB000F2E007C08091C00085FFFCCF319690935F
:103EC000C60090819923B1F72BC08091C00085FF77
:103ED000FCCF31969093C60090819923B1F720C012
:103EE0008091C00085FFFCCF31969093C6009081F1
:103EF0009923B1F715C08091C00085FFFCCF3196A2
:103F00009093C60090819923B1F70AC08091C000B8
:103F100085FFFCCF31969093C60090819923B1F72D
:103F20008FED99E0622F40E050E00E948440809144
:103F3000C00085FFFCCF8AE08093C60081E001C00D
:103F400080E0DF91CF910895AF92BF92CF92DF9240
:103F5000EF92FF920F931F93CF93DF9314E5E12E1F
:103F600017E0F12ECDEAD7E000E010E0F801E052D2
:103F7000FC4F80810E94B51E882339F10E94071FE3
:103F80005B016C01F801E25BF84F8081882311F03E
:103F900061E002C06091BD0770E0882777FD8095E1
:103FA000982F0E9454D5F70120813181428153819D
:103FB0000E9492D79B01AC01C601B5010E94D9D3E2
:103FC000688379838A839B8309C0F701808191810B
:103FD000A281B38188839983AA83BB830F5F1F4F1C
:103FE00084E090E0E80EF91E24960430110509F0F3
:103FF000BDCF86E40E94B51E8823E1F00E94071F12
:104000007B018C016093BE077093BF078093C0074C
:104010009093C10720E030E040E050E00E94C0D61D
:10402000181644F4E0929B03F0929C0300939D03C6
:1040300010939E03DF91CF911F910F91FF90EF900E
:10404000DF90CF90BF90AF9008950E94A41F89E4A5
:104050000E94B51E882359F00E94071F6093A10794
:104060007093A2078093A3079093A4070CC080E0ED
:1040700090E0A0E0B0E08093A1079093A207A09306
:10408000A307B093A4078AE40E94B51E882359F0C1
:104090000E94071F6093A5077093A6078093A70748
:1040A0009093A807089580E090E0A0E0B0E08093AE
:1040B000A5079093A607A093A707B093A807089514
:1040C0002F923F924F925F926F927F928F929F9228
:1040D000AF92BF92CF92DF92EF92FF920F931F9316
:1040E000DF93CF93CDB7DEB7EE970FB6F894DEBF70
:1040F0000FBECDBF87E40E94B51E882309F44EC4CD
:104100000E94071F0E9421D56430710509F441C047
:104110006530710554F46230710541F16330710509
:104120006CF57723CCF40C94BA376A35710509F431
:10413000E0C36B35710534F46C31710511F00C94EA
:10414000BA376FC06B35710509F4D7C36C3571058B
:1041500011F00C94BA37D6C380918E07882331F4BE
:104160000E94A41F0E94361C0C94E13780918E0798
:10417000882321F40E94252081E007C080918E07CA
:10418000882339F40E94252080E00E94791B0C943A
:10419000E13786E395E00E946ECA80E50E94B51E75
:1041A000882321F4EE24FF24870106C00E94071F04
:1041B0000E9426D57B018C0183E50E94B51E8823D1
:1041C00061F00E94071F20E030E04AE754E40E94BB
:1041D00092D70E9426D57B018C010E948A690E9499
:1041E0008F145B016C01AE0CBF1CC01ED11E0E945F
:1041F0008F146093990770939A0780939B0790930D
:104200009C0706C00E940C760E94151B0E94A0CA43
:104210000E948F146A157B058C059D0598F30C94FC
:10422000BA3780919B0390919C03A0919D03B0911C
:104230009E038093C8079093C907A093CA07B093C1
:10424000CB0780917F0390918003909353078093D5
:10425000520784E690E09093800380937F030E944E
:104260008F146093990770939A0780939B0790939C
:104270009C0781E00E941568809154079091550732
:10428000A0915607B09157078093AD079093AE0762
:10429000A093AF07B093B00780915807909159074A
:1042A000A0915A07B0915B078093B1079093B20732
:1042B000A093B307B093B40780915C0790915D071A
:1042C000A0915E07B0915F078093B5079093B60702
:1042D000A093B707B093B8078091600790916107EA
:1042E000A0916207B09163078093B9079093BA07D2
:1042F000A093BB07B093BC0780E090E0A0E0B0E0E3
:1043000080939B0390939C03A0939D03B0939E0383
:1043100088E50E94B51E882361F489E50E94B51ED8
:10432000882339F48AE50E94B51E882311F481E0C0
:1043300001C080E080939F03882361F488E50E9498
:10434000B51E882309F41BC289E50E94B51E882387
:1043500009F415C280E090E0A0E0B0E0809354073B
:1043600090935507A0935607B0935707809358072B
:1043700090935907A0935A07B0935B07BFE38B2E26
:10438000B5E09B2EF401E49084E597E068E577E0E2
:104390004CE557E020E637E00E947C56A2E46A2E06
:1043A000A5E07A2EF301659175918591949120E0B5
:1043B00030E040EC5FE30E9492D75B016C01FF2488
:1043C000E7FCF0940027F7FC0095102FC801B70117
:1043D0000E9454D59B01AC01C601B5010E9492D741
:1043E0006093AD077093AE078093AF079093B007CB
:1043F000F4E04F2E512C460C571CF201659175913B
:10440000859194910894811C911CF401D49020E032
:1044100030E040EC5FE30E9492D77B018C016D2D70
:10442000772767FD7095872F972F0E9454D59B01A2
:10443000AC01C801B7010E9492D76093B107709395
:10444000B2078093B3079093B40720916F03309124
:104450007003409171035091720320939B0330933A
:104460009C0340939D0350939E03E0907303F09050
:1044700074030091750310917603C801B7010E947F
:10448000B2D4882344F4E0929B03F0929C030093FF
:104490009D0310939E03F301A590B590C590D49011
:1044A000F201E590F59005911491C601B501A801BE
:1044B00097010E94C0D618162CF4C801B701A601B6
:1044C000950104C0C601B501A80197010E94B9D4A5
:1044D0009B01AC010E9492D79B01AC01CA0120E074
:1044E00030E040E85FE30E94D9D30E94FFD79B01F0
:1044F000AC0160919B0370919C0380919D0390910E
:104500009E030E9492D760939B0370939C038093B9
:104510009D0390939E0360919B0370919C038091F7
:104520009D0390919E0320E030E040E752E40E941A
:10453000B9D47B018C018DEA97E061EB77E045EB24
:1045400057E029EB37E0E3E8CE2EE7E0DE2E0E94CD
:104550008B5B0E948A69EEE4F5E065917591859127
:1045600094912091640730916507409166075091BE
:1045700067070E94D9D360935407709355078093BF
:10458000560790935707EAE5F5E065917591859197
:10459000949120916407309165074091660750918E
:1045A00067070E94D9D36093700770937107809357
:1045B000720790937307E6E6F5E065917591859132
:1045C000949120916407309165074091660750915E
:1045D00067070E94D9D36093890370938A038093FD
:1045E0008B0390938C03E2E5F5E0659175918591DD
:1045F0009491209168073091690740916A07509122
:104600006B070E94D9D36093580770935907809322
:104610005A0790935B07EEE5F5E0659175918591FA
:104620009491209168073091690740916A075091F1
:104630006B070E94D9D360937407709375078093BA
:10464000760790937707EAE6F5E065917591859195
:104650009491209168073091690740916A075091C1
:104660006B070E94D9D360938D0370938E03809360
:104670008F039093900384E597E068E577E04CE53D
:1046800057E020E637E00E947C56809154079091D5
:104690005507A0915607B09157078093AD079093A7
:1046A000AE07A093AF07B093B007809158079091E1
:1046B0005907A0915A07B0915B078093B107909377
:1046C000B207A093B307B093B40760919B037091B6
:1046D0009C0380919D0390919E0320E030E040E791
:1046E00052E40E94B9D47B018C018DEA97E061EB22
:1046F00077E045EB57E029EB37E00E948B5B80E0E9
:1047000090E0A0E0B0E080939B0390939C03A09383
:104710009D03B0939E030E948A690E940E68809157
:10472000AD079091AE07A091AF07B091B00780930D
:10473000540790935507A0935607B093570780915D
:10474000B1079091B207A091B307B091B4078093DD
:10475000580790935907A0935A07B0935B0780912D
:10476000B5079091B607A091B707B091B8078093AD
:104770005C0790935D07A0935E07B0935F078091FD
:104780009F03882329F488E50E94B51E882321F021
:1047900080E090E00E94261D80919F03882329F4E9
:1047A00089E50E94B51E882321F081E090E00E94F7
:1047B000261D88E50E94B51E8823D9F00E94FB1EA5
:1047C0006115710581059105A1F00E94071F2091D7
:1047D00064073091650740916607509167070E9412
:1047E000D9D36093540770935507809356079093DD
:1047F000570789E50E94B51E8823D9F00E94FB1E49
:104800006115710581059105A1F00E94071F209196
:1048100068073091690740916A0750916B070E94C1
:10482000D9D3609358077093590780935A07909390
:104830005B0780919F03882329F48AE50E94B51EB7
:10484000882321F082E090E00E94261D8AE50E94E4
:10485000B51E8823D9F00E94FB1E611571058105E4
:104860009105A1F00E94071F20916C0730916D0700
:1048700040916E0750916F070E94D9D360935C07F7
:1048800070935D0780935E0790935F0784E597E0E0
:1048900068E577E04CE557E020E637E00E947C567B
:1048A00080E00E9415688091C8079091C907A09187
:1048B000CA07B091CB0780939B0390939C03A0936E
:1048C0009D03B0939E03809152079091530790935C
:1048D000800380937F030E948F14609399077093E5
:1048E0009A0780939B0790939C070E940E680C94F4
:1048F000BA371092BD070C94BA3781E08093BD0798
:104900000C94BA3785E40E94B51E882311F40E94E6
:104910008A6944E5E42E47E0F42E34E6C32E37E0FE
:10492000D32E00E010E0F801E052FC4F80810E949D
:10493000B51E882331F1033061F40E94071FF7018F
:10494000608371838283938380E697E00E945E5642
:1049500018C00E94071FF6012081318142815381D6
:104960000E94D9D3F701608371838283938384E5A6
:1049700097E068E577E04CE557E020E637E00E94F5
:104980007C560F5F1F4F24E030E0E20EF31EC20E94
:10499000D31E0430110539F60C94BA378DE40E9409
:1049A000B51E882311F40C94DC360E94071F0E9468
:1049B00021D56237710511F40C94C92E6337710546
:1049C0000CF09BC06E31710509F493C26F31710513
:1049D0000CF042C06631710509F4F1C1673171050F
:1049E000E4F46131710509F4AAC16231710534F44E
:1049F0006230710510F00C94BA3742C16431710510
:104A000009F4A7C1653171050CF0D3C1623171059C
:104A100011F00C94BA370C94AC2D6931710509F47E
:104A200000C26A31710554F46731710509F4CDC1D2
:104A30006831710511F00C94BA37E3C16B3171051F
:104A400009F414C26B3171050CF4F1C16C317105BC
:104A500011F00C94BA3710C26435710511F40C943E
:104A6000AC2D6535710514F56A32710509F4B7C3CB
:104A70006B32710554F46F31710509F42BC3603248
:104A8000710511F00C94BA377AC26235710511F4D0
:104A90000C94A32D6335710514F00C94A72D61358A
:104AA000710511F00C94BA370C94882D6936710594
:104AB00009F410C46A36710584F46C35710511F47B
:104AC0000C941C2E6836710509F4D3C36535710545
:104AD00011F00C94BA370C94052E6B36710511F455
:104AE0000C94822D6B36710514F40C94512D6D3697
:104AF000710511F00C94BA3711C56D3D710511F4B3
:104B00000C94B2316E3D71050CF054C06E3B7105D2
:104B100009F4B4C66F3B71051CF56737710509F4DC
:104B2000ABC06837710564F46337710511F40C94F8
:104B3000A22E6537710511F00C94BA370C94B22E81
:104B40006937710511F40C94C32F6937710514F49A
:104B50000C94BE2F6C38710511F00C94BA37A9C3B0
:104B60006C3C710511F40C9407316D3C71058CF4AB
:104B7000693C710511F40C94C7306B3C710511F45C
:104B80000C94E930683C710511F00C94BA370C9420
:104B90004F306E3C710511F40C9485316E3C7105FB
:104BA00014F40C9427316C3D710511F00C94BA3754
:104BB0000C94A33131E0653F730711F40C945E331C
:104BC00041E0663F74074CF551E06E32750711F411
:104BD0000C94093381E06F32780764F4623E71050A
:104BE00011F40C94D9316D52714011F00C94BA3714
:104BF0000C943132E1E060397E0711F40C945833A3
:104C0000F1E0643F7F0711F40C945B336F52714005
:104C100011F00C94BA370C94183333E063357307F2
:104C200011F40C94673343E0643574079CF451E04D
:104C3000673F750711F40C94643381E0673F780790
:104C400014F40C9461336855724011F00C94BA3727
:104C50000C946C34E3E0603A7E0709F400C2F3E0A0
:104C6000673E7F0711F40C94C5366B58734011F002
:104C70000C94BA370C949636E3E7F2E00C94CF2FFD
:104C800085E295E00E946ECA80E50E94B51E8823E9
:104C900021F4EE24FF24870106C00E94071F0E9412
:104CA00026D57B018C0183E50E94B51E882361F027
:104CB0000E94071F20E030E04AE754E40E9492D7A8
:104CC0000E9426D57B018C010E948A690E948F1464
:104CD0006093990770939A0780939B0790939C0722
:104CE000E114F1040105110501F10E948F145B012B
:104CF0006C01AE0CBF1CC01ED11E0E948F146A1521
:104D00007B058C059D05A8F40E94F393882389F404
:104D10000E940C760E94151B0E94A0CAEECF0E9432
:104D20000C760E94151B0E94A0CA0E94F393882350
:104D3000B1F386E195E00E946ECA0C94BA378DE01B
:104D400095E00E946ECA15984698439840980C9436
:104D5000BA37EDEFF4E0949108C08091C00085FF70
:104D6000FCCF9093C600319694919923B1F780912E
:104D7000C00085FFFCCF8AE08093C60081EC94E000
:104D80000E942D89EFEEF4E0949108C08091C0005C
:104D900085FFFCCF9093C600319694919923B1F78B
:104DA0008091C00085FFFCCF8AE08093C6000C9400
:104DB000BA3781EC94E00E948C840C94BA3781EC71
:104DC00094E00E94C47C0C94BA378091CC079091F7
:104DD000CD0704966AE270E00E947711FC0100970B
:104DE00011F0319710826091CC077091CD076C5F04
:104DF0007F4F81EC94E041E021E00E94A2800C947E
:104E0000BA3781EC94E00E94C87C0E948F146093B2
:104E100086077093870780938807909389070C947F
:104E2000BA3781EC94E00E94CF7C0C94BA37809121
:104E3000C404882311F40C94BA3783E50E94B51E8C
:104E4000882311F40C94BA370E94FB1EAB01BC01FD
:104E50004093440750934507809346077093470754
:104E60008FE896E00E94A9440C94BA3781EC94E054
:104E70000E948D7E0C94BA378091CC079091CD071B
:104E800004966AE270E00E9477118C01009719F194
:104E90002091C2073091C30780E690E0AC01249FC7
:104EA000C001259F900D349F900D11248253984F7F
:104EB0006EE470E00E94771160E270E00E9477116A
:104EC0009C012F5F3F4F3093CD072093CC070150BB
:104ED0001040F80110826091CC077091CD076C5F93
:104EE0007F4F81EC94E040E021E00E94A2800C948E
:104EF000BA378091C404882311F40C94BA3781EC3A
:104F000094E060E00E94FC7D8091CC079091CD07F9
:104F100004966AE270E00E9477118C01009719F103
:104F20002091C2073091C30780E690E0AC01249F36
:104F3000C001259F900D349F900D11248253984FEE
:104F40006EE470E00E94771160E270E00E947711D9
:104F50009C012F5F3F4F3093CD072093CC0701502A
:104F60001040F80110826091CC077091CD076C5F02
:104F70007F4F81EC94E00E94E77E0C94BA378091D9
:104F8000C304882311F00E948A69E090CC07F09056
:104F9000CD0724E030E0E20EF31EC7016AE270E0C4
:104FA0000E9477118C01C70161E270E00E947711C5
:104FB000009721F07C010894E11CF11C01151105FA
:104FC00021F001501040F801108280E50E94B51ECA
:104FD000182F8091CC079091CD07E816F90608F4B8
:104FE00010E08091C404882311F40C94BA3721E0B6
:104FF000212781EC94E0B70141E00E94A28083E583
:105000000E94B51E8823B9F08091CC079091CD07FE
:105010008E159F0580F40E94FB1EAB01BC014093DE
:1050200044075093450780934607709347078FE8DE
:1050300096E00E94A94481EC94E00E94C87C112370
:1050400011F00C94BA370E948F1460938607709306
:10505000870780938807909389070C94BA378091CB
:10506000CC079091CD0705966AE270E00E94771117
:105070008C01009719F12091C2073091C30780E697
:1050800090E0AC01249FC001259F900D349F900DAE
:1050900011248253984F6EE470E00E94771160E211
:1050A00070E00E9477119C012F5F3F4F3093CD0736
:1050B0002093CC0701501040F80110826091CC077A
:1050C0007091CD076B5F7F4F81EC94E00E948384E9
:1050D0000C94BA370E948F1460938A0770938B07E1
:1050E00080938C0790938D072091860730918707D6
:1050F0004091880750918907621B730B840B950BB5
:1051000028EE33E040E050E00E94AAD8F22EE32ED1
:10511000D42EC52E2DB73EB7285030400FB6F89488
:105120003EBF0FBE2DBF0DB71EB70F5F1F4FCE0185
:105130008196EDB7FEB79283818380EE94E0F8010B
:10514000938382836F2D7E2D842F952F2CE330E067
:1051500040E050E00E94AAD8F801358324836F2DE7
:105160007E2D8D2D9C2D2CE330E040E050E00E9400
:10517000AAD8F801778366830E94A611EFE4F2E0D3
:1051800094912DB73EB7285F3F4F0FB6F8943EBFBE
:105190000FBE2DBF08C08091C00085FFFCCF90934B
:1051A000C600319694919923B1F7FE01B19607C0DC
:1051B0008091C00085FFFCCF31969093C60090810E
:1051C0009923B1F78091C00085FFFCCF8AE08093DE
:1051D000C600CE0181960E9491CA0C94BA3783E52D
:1051E0000E94B51E882311F40C94BA370E94071F41
:1051F0000E9421D57B018C016B0180E50E94B51EC8
:10520000882369F0F7FC0BC03FEFE316F10409F0C7
:1052100034F40E94071F0E9421D58B0102C008E0D0
:1052200010E0E4EEF3E0808191818017910711F4A2
:105230000C94BA37329644E0E435F407A1F707300E
:10524000110529F4D0928507C092840704C017FF86
:1052500002C00C94BA37802F61E00E944216802F62
:105260006C2D0E94F516802FB6010E9462150C94D9
:10527000BA3788E690E00E94111F882311F00C9441
:10528000BA3783E50E94B51E882379F00E94071F74
:1052900020919007022F10E0000F111F05571E4E9E
:1052A0000E9421D5F801718360830E94D1730C9410
:1052B000BA3783E50E94B51E882311F40C94BA37DF
:1052C0000E94071F0E9421D570938E1160938D114B
:1052D0000C94BA3789E690E00E94111F882311F0E0
:1052E0000C94BA37EAEDF4E0949108C08091C000C4
:1052F00085FFFCCF9093C600319694919923B1F726
:10530000E0919007F0E0EE0FFF1FEE0FFF1FEF564A
:10531000FE4E40815181628173818FED99E021E0E1
:1053200030E00E94A641E7EDF4E0949108C080913E
:10533000C00085FFFCCF9093C600319694919923CD
:10534000B1F7E0919007F0E0EE0FFF1FE557FE4E3A
:1053500060817181882777FD8095982F0E9454D5B0
:10536000AB01BC018FED99E021E030E00E94A64145
:10537000E3EDF4E0949108C08091C00085FFFCCF7C
:105380009093C600319694919923B1F7409197116B
:10539000509198116091991170919A118FED99E047
:1053A00021E030E00E94A641E0EDF4E0949108C0D5
:1053B0008091C00085FFFCCF9093C60031969491F8
:1053C0009923B1F760918D1170918E11882777FD27
:1053D0008095982F0E9454D5AB01BC018FED99E0C8
:1053E00021E030E00E94A641EDECF4E0949108C089
:1053F0008091C00085FFFCCF9093C60031969491B8
:105400009923B1F78FED99E060E070E04AE050E059
:105410000E94CB40EBECF4E0949108C08091C00076
:1054200085FFFCCF9093C600319694919923B1F7F4
:10543000409191115091921160919311709194113A
:105440008FED99E021E030E00E94A641E8ECF4E025
:10545000949108C08091C00085FFFCCF9093C60056
:10546000319694919923B1F760918B1170918C11C1
:10547000882777FD8095982F0E9454D5AB01BC01F9
:105480008FED99E021E030E00E94A641E4ECF4E0E9
:10549000949108C08091C00085FFFCCF9093C60016
:1054A000319694919923B1F7809190070E94CB7027
:1054B000BC018FED99E04AE050E00E94CB40EFEB59
:1054C000F4E0949108C08091C00085FFFCCF9093D8
:1054D000C600319694919923B1F78FEF9FEF0E9408
:1054E000CB70BC018FED99E04AE050E00E94CB40C8
:1054F000ECE8F2E007C08091C00085FFFCCF319658
:105500009093C60090819923B1F78091C00085FFE8
:10551000FCCF8AE08093C6000C94E1378DE690E0E2
:105520000E94111F882311F00C94BA3784EB94E089
:105530000E946ECA83E50E94B51E882399F00E94DE
:10554000071F20919007022F10E0000F111F055731
:105550001E4E0E9421D5F8017183608381E0809303
:10556000960316C082E50E94B51E882389F00E942A
:10557000071F20919007022F10E0000F111F055701
:105580001E4E0E9421D5F80171836083109296030C
:105590000E94D1730E948F144B015C0120919007EF
:1055A000022F10E010928F07000F111FF801E5572E
:1055B000FE4E60817181882777FD8095982F0E942B
:1055C00054D5000F111F0F561E4EF8012081318156
:1055D000428153810E94C0D618161CF481E080934A
:1055E0008F07CC24CA94DC2C7601E1EBF4E05490D4
:1055F000EDEAF4E06490E9EAF4E074906AE0462EA3
:1056000030C1952DE1EBF4E008C08091C00085FF2A
:10561000FCCF9093C600319694919923B1F7E09115
:105620009007F0E0EE0FFF1FEE0FFF1FEF56FE4E4C
:1056300040815181628173818FED99E021E030E0FA
:105640000E94A641962DEDEAF4E008C08091C000CA
:1056500085FFFCCF9093C600319694919923B1F7C2
:10566000609190078FED99E070E04AE050E00E9471
:10567000CB40972DE9EAF4E008C08091C00085FF97
:10568000FCCF9093C600319694919923B1F7F7FE21
:1056900003C0EDE8F2E028C00E948F14A701960134
:1056A0002854344F4F4F5F4F261B370B480B590B75
:1056B000CA01B90128EE33E040E050E00E94AAD8C8
:1056C0008FED99E0BA01A9012AE030E00E9477400D
:1056D0008091C00085FFFCCF0EC08091C00085FF87
:1056E000FCCF31969093C60090819923B1F78091B9
:1056F000C00085FFFCCF4092C6000E948F144B0172
:105700005C010E940C760E94151B0E94A0CAFFEF4C
:10571000CF16FFEFDF06FFEFEF06FFEFFF0609F002
:1057200052C080918F07E0919007882331F1F0E01B
:105730008F01000F111F000F111F0F561E4EEE0F8D
:10574000FF1FE557FE4E60817181882777FD8095A8
:10575000982F0E9454D520E030E040E85FE30E949B
:10576000D8D39B01AC01F801608171818281938162
:105770000E94C0D687FF58C05EC0F0E08F01000FC6
:10578000111F000F111F0F561E4EEE0FFF1FE55782
:10579000FE4E60817181882777FD8095982F0E9449
:1057A00054D520E030E040E85FE30E94D9D39B016C
:1057B000AC01F80160817181828193810E94B2D431
:1057C000181694F538C0F7FC36C0E0919007F0E069
:1057D0008F01000F111F000F111F0F561E4EEE0FED
:1057E000FF1FE557FE4E60817181882777FD809508
:1057F000982F0E9454D59B01AC01F8016081718102
:10580000828193810E94D8D30E9421D597FF07C03F
:1058100090958095709561957F4F8F4F9F4F643025
:105820007105810591053CF00E948F14AC01CB01FC
:10583000DA016C017D01FFEFCF16FFEFDF06FFEF0E
:10584000EF06FFEFFF0669F0F7FE02C00C94BD37CC
:105850000E948F146C197D09685B7B4010F00C94DA
:10586000BD370E948F14681979098A099B09695EFE
:1058700073408040904008F0C4CE43CF8EE894E05F
:105880000E946ECA83E50E94B51E882361F00E94C3
:10589000071F0E9421D570938E1160938D1181E0B6
:1058A000809396030FC082E50E94B51E882351F0B5
:1058B0000E94071F0E9421D570938E1160938D1155
:1058C000109296030E948F147B018C0110928F0717
:1058D00060918D1170918E11882777FD8095982F9A
:1058E0000E9454D5209197113091981140919911AF
:1058F00050919A110E94C0D618160CF082C081E017
:1059000080938F077EC00E948F146E197F09800BD1
:10591000910B695E73408040904008F46BC0E09149
:105920008307F0E0EE0FFF1FEE0FFF1FEF56FE4E56
:1059300040815181628173819B2DEBE8F4E008C0C6
:105940008091C00085FFFCCF9093C6003196949162
:105950009923B1F78FED99E022E030E00E94A64153
:105960009C2DE7E8F4E008C08091C00085FFFCCFE3
:105970009093C600319694919923B1F76091830773
:105980008FED99E070E04AE050E00E94CB409D2D01
:10599000E3E8F4E008C08091C00085FFFCCF90935D
:1059A000C600319694919923B1F740919711509187
:1059B00098116091991170919A118FED99E021E001
:1059C00030E00E94A641ECE8F2E007C08091C00000
:1059D00085FFFCCF31969093C60090819923B1F753
:1059E0008091C00085FFFCCFA092C6000E948F145A
:1059F0007B018C010E940C760E94151B0E94A0CA9C
:105A00000BC0EBE8F4E0B490E7E8F4E0C490E3E81E
:105A1000F4E0D4907AE0A72E80918F0720918D1129
:105A200030918E118823A9F0B901882777FD8095E0
:105A3000982F0E9454D52091971130919811409140
:105A4000991150919A110E94C0D618160CF45BCF90
:105A500018C0B901882777FD8095982F0E9454D5EA
:105A600020919711309198114091991150919A116C
:105A70000E94B2D488232CF480919603882309F4E1
:105A800042CF89E794E00E946ECA0E948F1460930F
:105A9000990770939A0780939B0790939C070C94A7
:105AA000BA3783E50E94B51E882321F10E94071FA3
:105AB00020E030E040E050E00E94B2D488231CF4A3
:105AC00060E070E011C00E94071F20E030E04FE767
:105AD00053E40E94C0D618161CF46FEF70E004C0A7
:105AE0000E94071F0E9421D5709385076093840749
:105AF0000C94BA378FEF90E09093850780938407DA
:105B00000C94BA3710928507109284070C94BA3718
:105B10000E9486710E948A69409A0E949869109238
:105B200085071092840768EE73E080E090E00E94A1
:105B30009D14109295038AE694E00E946ECA0E941A
:105B4000A0CA0C94BA37109251070C94BA3781E06E
:105B5000809351070C94BA3783E50E94B51E8823C1
:105B6000A1F00E94071F20E030E04AE754E40E94C1
:105B700092D70E9426D560939703709398038093E1
:105B8000990390939A030C94BA3788E50E94B51E46
:105B9000882311F00C94D63789E50E94B51E88231E
:105BA00011F00C94D6378AE50E94B51E882311F0B7
:105BB0000C94D63785E40E94B51E882311F00C940E
:105BC000D6370E948A69409A0E9498690C94BA3725
:105BD000159A10927C0789E50E94B51E882319F05A
:105BE000469A10927D078AE50E94B51E882319F017
:105BF000439A10927E0785E40E94B51E882311F413
:105C00000C94BA37409A0C94BA3783E50E94B51EBB
:105C10000E94071F20E030E04AE754E40E9492D738
:105C20000E9426D560939D0770939E0780939F07DF
:105C30009093A0070C94BA3761E0662E6CE0762E44
:105C400051EF252E5BE0352E4DE3442E4CE0542ED3
:105C500088249924F401E052FC4F80810E94B51EF3
:105C6000882309F45DC053E0851609F052C00E94F4
:105C7000071F5B016C0120E030E040EA51E40E9424
:105C8000B2D488230CF03FC0F3016081718182811E
:105C90009381A60195010E94B9D47B018C0160918A
:105CA000350C7091360C8091370C9091380CA8010E
:105CB00097010E9492D76093350C7093360C8093B5
:105CC000370C9093380CF10160817181828193814E
:105CD000A80197010E9492D7F101608371838283AA
:105CE0009383F20160817181828193810E9452D5F8
:105CF000A80197010E9492D70E9426D5F2016083E5
:105D0000718382839383F301A082B182C282D382A2
:105D100007C00E94071FF30160837183828393830E
:105D20000894811C911C24E030E0620E731E220E48
:105D3000331E420E531E34E08316910409F08ACFBD
:105D40000C94BA37E0EAF3E0949108C08091C00067
:105D500085FFFCCF9093C600319694919923B1F7BB
:105D60000C94BA378091CC079091CD0705966AE2E2
:105D700070E00E947711FC01009711F031971082BA
:105D80008091CC079091CD0705960E9491CA0C9402
:105D9000BA37EDE9F3E0949108C08091C00085FF27
:105DA000FCCF9093C600319694919923B1F740911E
:105DB00054075091550760915607709157078FED22
:105DC00099E022E030E00E94A641E9E9F3E09491F5
:105DD00008C08091C00085FFFCCF9093C60031962B
:105DE00094919923B1F740915807509159076091C8
:105DF0005A0770915B078FED99E022E030E00E9436
:105E0000A641E5E9F3E0949108C08091C00085FFC8
:105E1000FCCF9093C600319694919923B1F74091AD
:105E20005C0750915D0760915E0770915F078FED91
:105E300099E022E030E00E94A641E1E9F3E094918C
:105E400008C08091C00085FFFCCF9093C6003196BA
:105E500094919923B1F74091600750916107609147
:105E60006207709163078FED99E022E030E00E94B5
:105E7000A641E6E8F3E0949108C08091C00085FF58
:105E8000FCCF9093C600319694919923B1F780E0AE
:105E90000E9469680E9454D52091010C3091020C37
:105EA0004091030C5091040C0E94B9D4AB01BC0189
:105EB0008FED99E022E030E00E94A641E2E8F3E0B5
:105EC000949108C08091C00085FFFCCF9093C600DC
:105ED000319694919923B1F781E00E9469680E94FC
:105EE00054D52091050C3091060C4091070C50912F
:105EF000080C0E94B9D4AB01BC018FED99E022E0FF
:105F000030E00E94A641EEE7F3E0949108C0809152
:105F1000C00085FFFCCF9093C600319694919923E1
:105F2000B1F782E00E9469680E9454D52091090C63
:105F300030910A0C40910B0C50910C0C0E94B9D47A
:105F4000AB01BC018FED99E022E030E00E94A64158
:105F5000ECE8F2E007C08091C00085FFFCCF3196ED
:105F60009093C60090819923B1F78091C00085FF7E
:105F7000FCCF8AE08093C6000C94BA3780E00E9480
:105F800015680C94BA3781E00E9415680C94BA37F2
:105F90008091C00085FFFCCF31969093C600908120
:105FA0009923B1F78091C00085FFFCCF8AE08093F0
:105FB000C600E6E7F3E0949108C08091C00085FF39
:105FC000FCCF9093C600319694919923B1F7009B32
:105FD00003C0EFE8F2E00AC0E4E9F2E007C0809114
:105FE000C00085FFFCCF31969093C6009081992325
:105FF000B1F78091C00085FFFCCF8AE08093C60096
:10600000EEE6F3E0949108C08091C00085FFFCCFDC
:106010009093C600319694919923B1F7049B03C0E5
:10602000EFE8F2E00AC0E4E9F2E007C08091C000C6
:1060300085FFFCCF31969093C60090819923B1F7EC
:106040008091C00085FFFCCF8AE08093C600E6E621
:10605000F3E0949108C08091C00085FFFCCF90933D
:10606000C600319694919923B1F7079B03C0EFE8DE
:10607000F2E00AC0E4E9F2E007C08091C00085FFC9
:10608000FCCF31969093C60090819923B1F780910F
:10609000C00085FFFCCF8AE08093C6006BC784E414
:1060A0000E94B51E882309F465C70E94071F20E0DF
:1060B00030E040E05FE30E9492D77B018C0120E05A
:1060C00030E040E050E00E94B2D4882359F40F2E13
:1060D000F0E0CF2EF0E0DF2EF0E8EF2EFFE3FF2E12
:1060E000F02D11C0C801B701A80197010E9492D7F5
:1060F0009B01AC01CA012BED3FE049E450E40E9452
:1061000092D76B017C01809183078093900784E58F
:106110000E94B51E882319F10E94071F0E9426D5F0
:10612000609390076623D9F0EFE4F2E0949108C001
:106130008091C00085FFFCCF9093C600319694916A
:106140009923B1F7EEE9F2E007C08091C00085FF26
:10615000FCCF31969093C60090819923B1F780913E
:106160009007082F10E0000F111F000F111F0B5791
:106170001C4F60E070E080E89FE3A70196010E9459
:10618000B9D4F8016083718382839383F3C600EEF0
:1061900013E021E1E22E2CE0F22EF80180810E9432
:1061A000B51E882349F00E94071F0E9426D5F701DB
:1061B00060837183828393830F5F1F4F24E030E0FD
:1061C000E20EF31E33E0043E130739F70E94335604
:1061D000D1C600EE13E091EFE92E9BE0F92EF80115
:1061E00080810E94B51E882339F00E94071FF701A5
:1061F00060837183828393830F5F1F4F24E030E0BD
:10620000E20EF31E33E0043E130749F7B3C683E5FD
:106210000E94B51E882351F00E94071F6093250C31
:106220007093260C8093270C9093280C84E50E9491
:10623000B51E882309F49EC60E94071F6093290C8F
:1062400070932A0C80932B0C90932C0C93C683E5AF
:106250000E94B51E882351F00E94071F6093210CF5
:106260007093220C8093230C9093240C84E50E945D
:10627000B51E882351F00E94071F6093390C70935C
:106280003A0C80933B0C90933C0C82E40E94B51E28
:10629000882361F00E94071F0E9426D56093ED0BB2
:1062A0007093EE0B8093EF0B9093F00B88E50E94B8
:1062B000B51E882351F00E94071F60932D0C709328
:1062C0002E0C80932F0C9093300C8AE50E94B51E03
:1062D000882351F00E94071F6093310C7093320C99
:1062E0008093330C9093340C85E40E94B51E882370
:1062F00009F440C60E94071F6093350C7093360C5A
:106300008093370C9093380C35C600EE13E084E68A
:10631000E82E87E0F82EF80180810E94B51E8823C0
:1063200039F00E94071FF701608371838283938392
:106330000F5F1F4F24E030E0E20EF31E33E0033E18
:10634000130749F717C683E50E94B51E882309F491
:1063500011C60E94071F0E9421D57093800360938D
:106360007F0308C683E50E94B51E882309F402C690
:106370000E94071F0E9421D57B018C0184E50E94A9
:10638000B51E882389F08DED90E00E94111F8823AF
:1063900009F0F0C5E0919007F0E0EE0FFF1FED5718
:1063A000FC4FF182E082E6C5F0928203E092810325
:1063B000E1C580E50E94B51E882309F4DBC50E9473
:1063C000071F0E9421D57B0183E50E94B51E88230B
:1063D00019F40FEF1FEF05C00E94071F0E9421D57F
:1063E0008B01C8010196039708F0C4C5E4EEF3E001
:1063F000808191818E159F0509F4BCC5329644E0D9
:10640000E435F407A9F7F7FCB5C50E948A69DE2CCC
:106410008E2D60E00E9442160115110541F00130F9
:10642000110579F05FEF0F3F1507A1F403C000E0FD
:1064300010E010C08E2D0E94281700E010E0892B7C
:1064400049F401E010E006C00E940C760E94151B82
:106450000E94A0CA8D2D0E94281780179107A1F7CE
:1064600089C580E50E94B51E882351F00E94071F50
:106470006093AF037093B0038093B1039093B20322
:1064800089E40E94B51E882361F00E94071F0E94C4
:106490009C716093B3037093B4038093B50390939E
:1064A000B60384E40E94B51E882361F00E94071F92
:1064B0000E94AA716093B7037093B8038093B903E5
:1064C0009093BA0383E40E94B51E882351F00E9482
:1064D000071F6093BB037093BC038093BD0390932D
:1064E000BE030E94B470E5EBF2E007C08091C000EB
:1064F00085FFFCCF31969093C60090819923B1F728
:10650000E8EBF2E007C08091C00085FFFCCF319638
:106510009093C60090819923B1F74091AF035091B9
:10652000B0036091B1037091B2038FED99E022E066
:1065300030E00E94A641ECEBF2E007C08091C00081
:1065400085FFFCCF31969093C60090819923B1F7D7
:106550006091B3037091B4038091B5039091B60339
:106560000E94A371AB01BC018FED99E022E030E005
:106570000E94A641E0ECF2E007C08091C00085FFD8
:10658000FCCF31969093C60090819923B1F760912A
:10659000B7037091B8038091B9039091BA030E9438
:1065A000B171AB01BC018FED99E022E030E00E94B7
:1065B000A641E4ECF2E007C08091C00085FFFCCF6B
:1065C00031969093C60090819923B1F74091BB0317
:1065D0005091BC036091BD037091BE038FED99E0B3
:1065E00022E030E00E94A641ECE8F2E007C0809192
:1065F000C00085FFFCCF31969093C600908199230F
:10660000B1F78091C00085FFFCCF8AE08093C6007F
:10661000B1C483E50E94B51E882329F460E070E0D0
:1066200080E090E002C00E94071F0E942A56A2C488
:1066300085E40E94B51E882319F4CC24DD2412C001
:106640000E94071F0E9421D56B0177FF0BC00F2E00
:10665000F0E0EF2EF0E0FF2EFCE80F2FF2E41F2F0A
:10666000F02D0AC00F2EF0E0EF2EF0E0FF2EF6E145
:106670000F2FF3E41F2FF02D83E50E94B51E882312
:1066800021F00E94071F7B018C0183E40E94B51E4C
:10669000882319F425E030E005C00E94071F0E94FE
:1066A00021D59B01C801B701A6010E944F7862C4A1
:1066B0000E948A695FC40E94168A5CC40E945B9132
:1066C00059C40E94788C56C40E94258E53C48AE512
:1066D0000E94B51E882309F4B8C00E94071F7B01E1
:1066E0008C0120E030E040E751EC0E94C0D68823C6
:1066F0000CF44EC0C801B70120E030E040EA50EC95
:106700000E94B2D418160CF443C0D801C701B05887
:1067100080937F0790938007A0938107B0938207AF
:10672000EFE4F2E0949108C08091C00085FFFCCFB7
:106730009093C600319694919923B1F7EAE5F3E07E
:10674000949108C08091C00085FFFCCF9093C60053
:10675000319694919923B1F78091C00085FFFCCFC9
:106760008AE08093C600ECE8F2E007C08091C000A8
:1067700085FFFCCF31969093C60090819923B1F7A5
:106780008091C00085FFFCCF8AE08093C600F2C3F1
:10679000EFE4F2E0949108C08091C00085FFFCCF47
:1067A0009093C600319694919923B1F7E1E5F3E017
:1067B000949108C08091C00085FFFCCF9093C600E3
:1067C000319694919923B1F7E9E4F3E0949108C0EC
:1067D0008091C00085FFFCCF9093C60031969491C4
:1067E0009923B1F78FED99E061EF7FEF4AE050E038
:1067F0000E94CB40E1E4F3E0949108C08091C00096
:1068000085FFFCCF9093C600319694919923B1F700
:106810008FED99E06BEF7FEF4AE050E00E94CB40B4
:10682000ECE8F2E007C08091C00085FFFCCF319614
:106830009093C60090819923B1F78091C00085FFA5
:10684000FCCF8AE08093C60095C3EFE4F2E0949118
:1068500008C08091C00085FFFCCF9093C6003196A0
:1068600094919923B1F7E5E3F3E0949108C0809106
:10687000C00085FFFCCF9093C60031969491992378
:10688000B1F78091C00085FFFCCF8AE08093C600FD
:1068900040917F0750918007609181077091820736
:1068A00070588FED99E022E030E00E94A641ECE8BC
:1068B000F2E007C08091C00085FFFCCF3196909335
:1068C000C60090819923B1F78091C00085FFFCCF6D
:1068D0008AE08093C6004EC3A0905407B09055073D
:1068E000C0905607D0905707A982BA82CB82DC822B
:1068F000E0905807F090590700915A0710915B07F4
:10690000ED82FE820F83188720915C0730915D072E
:1069100040915E0750915F0729873A874B875C87D4
:106920008091600790916107A0916207B091630721
:106930008D879E87AF87B88BA98ABA8ACB8ADC8A73
:10694000ED8AFE8A0F8B188F298F3A8F4B8F5C8FC1
:106950008D8F9E8FAF8FB8A385E40E94B51E8823CC
:1069600069F0ED84FE840F8518890E94071F9B0142
:10697000AC01C801B7010E94D9D30AC06D857E85DC
:106980008F85988920E030E040E050E40E94D8D321
:106990006D877E878F87988B60919B0370919C0396
:1069A00080919D0390919E0320E030E040E752E407
:1069B0000E94B9D47B018C01CE010196BE016B5FB0
:1069C0007F4FAE01475F5F4F9E01235F3F4FA3E8BC
:1069D000CA2EA7E0DA2E0E948B5B8AE50E94B51EC4
:1069E000882359F0E984FA840B851C850E94071FCF
:1069F0009B01AC01C801B70108C069857A858B8508
:106A00009C8520E030E040E251E40E94D9D36987C0
:106A10007A878B879C8760919B0370919C03809100
:106A20009D0390919E0320E030E040E752E40E94F5
:106A3000B9D47B018C01CE010196BE016B5F7F4F03
:106A4000AE01475F5F4F9E01235F3F4FF3E8CF2EBC
:106A5000F7E0DF2E0E948B5B88E50E94B51E88233D
:106A600089F0E980FA800B811C810E94071F9B013D
:106A7000AC01C801B7010E94D9D369837A838B83A3
:106A80009C8308C080E090E0A0E4B0E489839A830E
:106A9000AB83BC8389E50E94B51E882339F00E9430
:106AA000071F6D837E838F83988708C080E090E006
:106AB000A0E4B0E48D839E83AF83B88760919B038D
:106AC00070919C0380919D0390919E0320E030E0A3
:106AD00040E752E40E94B9D47B018C01CE010196BB
:106AE000BE016B5F7F4FAE01475F5F4F9E01235F2B
:106AF0003F4FE3E8CE2EE7E0DE2E0E948B5B8CE476
:106B00000E94B51E882369F0ED84FE840F851889E4
:106B10000E94071F9B01AC01C801B7010E94D9D395
:106B20000AC06D857E858F85988920E030E048EC2D
:106B300052E40E94D8D36D877E878F87988B6091AF
:106B40009B0370919C0380919D0390919E0320E094
:106B500030E040E752E40E94B9D47B018C01CE01C1
:106B60000196BE016B5F7F4FAE01475F5F4F9E0195
:106B7000235F3F4FB3E8CB2EB7E0DB2E0E948B5B49
:106B80000E948A69409A64E670E080E090E00E948A
:106B90009D1485E293E00E947DCA10E018C01F5F3B
:106BA0000E940C760E94151B0E94A0CA112379F442
:106BB000539A5B9A63E070E080E090E00E949D143D
:106BC0005B9863E070E080E090E00E949D140E947A
:106BD000F393882321F38CE40E94B51E882369F087
:106BE000ED84FE840F8518890E94071F9B01AC016C
:106BF000C801B7010E94D8D30AC06D857E858F85F4
:106C0000988920E030E048EC52E40E94D9D36D87A7
:106C10007E878F87988B8D859E85AF85B889809379
:106C2000600790936107A0936207B093630780E6C3
:106C300097E00E945E56A9E04A2E512C4C0E5D1E34
:106C4000FDE06F2E712C6C0E7D1E60919B03709188
:106C50009C0380919D0390919E0320E030E040E7EB
:106C600052E40E94B9D47B018C01CE010196BE0191
:106C70006B5F7F4FA2019301E3E8CE2EE7E0DE2EAB
:106C80000E948B5B91E1A92EB12CAC0EBD1E85E15B
:106C9000882E912C8C0E9D1E60919B0370919C03FD
:106CA00080919D0390919E0320E030E040E752E404
:106CB0000E94B9D47B018C01C501B401A2019301EA
:106CC0000E948B5B09E1402E512C4C0E5D1E6091A1
:106CD0009B0370919C0380919D0390919E0320E003
:106CE00030E040E752E40E94B9D47B018C01C50139
:106CF000B401A20193010E948B5B60919B03709190
:106D00009C0380919D0390919E0320E030E040E73A
:106D100052E40E94B9D47B018C01C501B401A201E7
:106D20009E01235E3F4F0E948B5B24C188E50E9439
:106D3000B51E882351F00E94071F0E9421D59B0198
:106D4000AC0180E0B9010E949E688AE50E94B51EF0
:106D5000882351F00E94071F0E9421D59B01AC019E
:106D600081E0B9010E949E6885E40E94B51E8823D7
:106D700009F400C10E94071F0E9421D59B01AC01AC
:106D800082E0B9010E949E68F5C010928E070E94B1
:106D9000F0938091950790919607A0919707B091F5
:106DA00098078093910790939207A0939307B093CD
:106DB00094070E94F81CDEC084E50E94B51E88235B
:106DC00009F48DC00E94071F0E9426D5262F6093CC
:106DD00090076623B9F1EFE4F2E0949108C0809146
:106DE000C00085FFFCCF9093C60031969491992303
:106DF000B1F7E8ECF2E007C08091C00085FFFCCF5E
:106E000031969093C60090819923B1F78FED99E068
:106E1000622F40E050E00E948440EAECF2E007C0BC
:106E20008091C00085FFFCCF31969093C600908181
:106E30009923B1F78091C00085FFFCCF8AE0809351
:106E4000C60098C086E40E94B51E8823E1F00E9427
:106E5000071F7B018C016093BE077093BF0780936F
:106E6000C0079093C10720E030E040E050E00E946E
:106E7000C0D6181644F4E0929B03F0929C03009352
:106E80009D0310939E03EFE4F2E0949108C080917B
:106E9000C00085FFFCCF9093C60031969491992352
:106EA000B1F7EBEDF2E007C08091C00085FFFCCFA9
:106EB00031969093C60090819923B1F76091830732
:106EC0008FED99E070E04AE050E00E94CB40809165
:106ED000C00085FFFCCF8AE08093C6004BC0EFE482
:106EE000F2E0949108C08091C00085FFFCCF9093A0
:106EF000C600319694919923B1F7E2E1F3E09491C1
:106F000008C08091C00085FFFCCF9093C6003196E9
:106F100094919923B1F72091C2073091C30780E67D
:106F200090E0289FF001299FF00D389FF00D11246B
:106F3000E253F84F07C08091C00085FFFCCF319627
:106F40009093C60090819923B1F7E0E1F3E094912A
:106F500008C08091C00085FFFCCF9093C600319699
:106F600094919923B1F78091C00085FFFCCF8AE00E
:106F70008093C6000E94E11A24C08BE994E00E942D
:106F80006ECA0E948F146093860770938707809360
:106F90008807909389070E948F14609399077093D4
:106FA0009A0780939B0790939C07E4CF0E948A697D
:106FB00088E50E94B51E882311F00C94E82D0C94EE
:106FC000EB2DEE960FB6F894DEBF0FBECDBFCF917E
:106FD000DF911F910F91FF90EF90DF90CF90BF90C6
:106FE000AF909F908F907F906F905F904F903F9069
:106FF0002F9008952F923F924F925F926F927F92BF
:107000008F929F92AF92BF92CF92DF92EF92FF92B8
:107010000F931F93DF93CF93CDB7DEB76E970FB665
:10702000F894DEBF0FBECDBF20E6A22EB12CEFEA52
:10703000F5E084909AE0792EE5E2F6E094906624FB
:10704000639413C22D3071F02A3321F480914F09DB
:10705000882341F080915009909151098F35910515
:107060000CF4DFC1E0915009F0915109309709F417
:1070700004C3A0915209B0915309AA9D7001AB9D20
:10708000F00CBA9DF00C1124EE0DFF1DE253F84FE9
:10709000108280914F09882309F0BEC110924F09D8
:1070A000AC53B84F1C9287010253184FC8016EE4CD
:1070B00070E00E9477119C01009709F4F7C090934B
:1070C000CD078093CC072F5F3F4F201B310B2E0D38
:1070D0003F1DC9018253984F60E070E04AE050E0E4
:1070E0000E94DF0F609354097093550980935609ED
:1070F00090935709C0909107D0909207E090930722
:10710000F0909407A70196012F5F3F4F4F4F5F4FBD
:10711000621773078407950709F457C380915209D2
:10712000909153099C012A9DC0012B9D900D3A9D81
:10713000900D11248253984F6EEC76E00E943C1122
:10714000892B09F042C3E5E5F2E0949108C08091F3
:10715000C00085FFFCCF9093C6003196949199238F
:10716000B1F7EBE9F6E0949108C08091C00085FF8B
:10717000FCCF9093C600319694919923B1F78FED8F
:1071800099E0B701A6012AE030E00E949640809184
:10719000C00085FFFCCF73C0FE264F5FFC01E40FEB
:1071A000F11DE253F84FE081EA32B1F73093CD0799
:1071B0002093CC07C901019660E070E00E947F0E29
:1071C0000E9421D52F2D30E02617370709F45DC026
:1071D000E5E5F2E0949108C08091C00085FFFCCF06
:1071E0009093C600319694919923B1F7ECE7F6E0BD
:1071F000949108C08091C00085FFFCCF9093C60099
:10720000319694919923B1F740919107509192074B
:1072100060919307709194078FED99E02AE030E038
:107220000E9496408091C00085FFFCCF28C0E5E514
:10723000F2E0949108C08091C00085FFFCCF90934C
:10724000C600319694919923B1F7E2E5F6E0949166
:1072500008C08091C00085FFFCCF9093C600319696
:1072600094919923B1F78FED99E0B701A6012AE037
:1072700030E00E9496408091C00085FFFCCF8AE0FC
:107280008093C6000E94F81C4AC0809154099091D6
:107290005509A0915609B091570980939107909391
:1072A0009207A0939307B09394073EC0C8016AE287
:1072B00070E00E947711009709F436C0E5E5F2E02E
:1072C000949108C08091C00085FFFCCF9093C600C8
:1072D000319694919923B1F7E8E2F6E0949108C0D1
:1072E0008091C00085FFFCCF9093C60031969491A9
:1072F0009923B1F7409191075091920760919307BC
:10730000709194078FED99E02AE030E00E9496405A
:107310008091C00085FFFCCF8AE08093C600109268
:1073200051091092500970C28091520990915309ED
:107330008A9D70018B9DF00C9A9DF00C11248701A1
:107340000253184FC80167E470E00E9477119C0156
:10735000009709F44BC09093CD078093CC072F5F23
:107360003F4F201B310B2E0D3F1DC9018253984FFB
:1073700060E070E00E947F0E0E9421D564307105AC
:10738000A8F580918E078823C9F48091C1048823D1
:1073900069F5992DE5E2F6E008C08091C00085FF0F
:1073A000FCCF9093C600319694919923B1F78091C8
:1073B000C00085FFFCCF7092C60018C0982DEFEA80
:1073C000F5E008C08091C00085FFFCCF9093C60017
:1073D000319694919923B1F78091C00085FFFCCF3D
:1073E0007092C60085EA95E00E946ECA80915209AB
:1073F00090915309019664E070E00E9497D89093B1
:107400005309809352098091580990915909019626
:10741000909359098093580910925109109250097C
:1074200024C02B3311F460924F0980914F098823B7
:10743000E1F42091500930915109809152099091C5
:1074400053098A9DF0018B9DF00D9A9DF00D11243A
:10745000E20FF31FE253F84F80914E0980832F5FB4
:107460003F4F30935109209350098091DB0990914F
:10747000DC092091DD093091DE09821B930B8F77A7
:107480009070892B09F4BBC18091580990915909DA
:1074900004970CF0B4C18FED99E00E94B73F282FFC
:1074A00080934E098A3009F0CDCDDCCD8091500912
:1074B00090915109892B09F0A7C1809158099091A9
:1074C0005909892B09F02FC110925A092CC14D304E
:1074D00099F0433211F04A3321F480914F09882307
:1074E00059F080915009909151098F35910524F4FC
:1074F0002F5F3F4F09F0F2C02091440730914507BC
:10750000409146075091470780913C0790913D0775
:10751000A0913E07B0913F07281739074A075B073C
:1075200008F49EC0932DE2E9F5E008C08091C00008
:1075300085FFFCCF9093C600319694919923B1F7C3
:107540008091C00085FFFCCF2092C6000E948F145E
:1075500060938A0770938B0780938C0790938D07B5
:1075600020918607309187074091880750918907BD
:10757000621B730B840B950B28EE33E040E050E068
:107580000E94AAD8F22EE32ED42EC52EEDB7FEB758
:1075900038970FB6F894FEBF0FBEEDBF0DB71EB7FC
:1075A0000F5F1F4FB282A182F80153824282622F85
:1075B000732F842F952F20E13EE040E050E00E94A1
:1075C000AAD8F801358324836F2D7E2D8D2D9C2D17
:1075D0002CE330E040E050E00E94AAD8CA01B90193
:1075E0002CE330E040E050E00E94AAD8F801778315
:1075F00066830E94A611982DEFE4F2E02DB73EB706
:10760000285F3F4F0FB6F8943EBF0FBE2DBF08C096
:107610008091C00085FFFCCF9093C6003196949175
:107620009923B1F7F50107C08091C00085FFFCCF19
:1076300031969093C60090819923B1F78091C00054
:1076400085FFFCCF2092C600C5010E9491CA81EC43
:1076500094E00E94288481EC94E061E00E946C85B3
:1076600080914E09833211F490925A092091500969
:10767000309151092115310519F410924F09C4C0F8
:107680008091520990915309869DF001879DF00DDC
:10769000969DF00D1124E20FF31FE253F84F108274
:1076A000FC01EC53F84F9082209158093091590910
:1076B0002F5F3F4F3093590920935809019664E09A
:1076C00070E00E9497D890935309809352091092CA
:1076D0004F0910925109109250093AC04B3311F4DE
:1076E00090924F0980914F09882391F5209150097C
:1076F000309151098091520990915309869DF00172
:10770000879DF00D969DF00D1124E20FF31FE253BB
:10771000F84F80914E0980832F5F3F4F309351097E
:107720002093500915C080E6682E712C99249394FB
:10773000E2E9F5E034900AE0202E5E010894A11CF5
:10774000B11C1EE7412E15E0512EEFE4F2E08490CB
:1077500020914407309145074091460750914707D3
:1077600080913C0790913D07A0913E07B0913F0763
:10777000281739074A075B0708F046C08091580967
:107780009091590904970CF03FC080915A098823C1
:10779000D9F58091970690919806A0919906B0919D
:1077A0009A068093440790934507A0934607B093A9
:1077B00047078FE896E00E9470489C01482F80930D
:1077C0004E098A3009F083CE97CE8091520990916C
:1077D00053098A9D80018B9D100D9A9D100D1124D7
:1077E000C8018253984F6AE270E00E9477119C01B1
:1077F000009709F41CCDFF2440E0C801CFCC809154
:10780000C304882309F052CE6E960FB6F894DEBFFB
:107810000FBECDBFCF91DF911F910F91FF90EF90E1
:10782000DF90CF90BF90AF909F908F907F906F90A0
:107830005F904F903F902F900895CF93DF9380916A
:10784000580990915909039714F40E94FA3781EC72
:1078500094E060E00E946C858091580990915909EC
:10786000892B09F46AC08091C104882309F44DC0B2
:107870002091C2073091C30780E690E0289FE00185
:10788000299FD00D389FD00D1124C253D84FCE015F
:1078900068EE76E00E943C11892BE1F481EC94E0E3
:1078A000BE010E94157E8091C204882371F5E5EE29
:1078B000F6E0949108C08091C00085FFFCCF9093C2
:1078C000C600319694919923B1F78091C00085FF4D
:1078D000FCCF17C081EC94E060E00E94FC7DE3EDFA
:1078E000F6E0949108C08091C00085FFFCCF909392
:1078F000C600319694919923B1F78091C00085FF1D
:10790000FCCF8AE08093C60002C00E946020809174
:1079100058099091590901979093590980935809F2
:107920008091C2079091C307019664E070E00E94C5
:1079300097D89093C3078093C2070E940C760E9449
:10794000151B0E940A700E94A0CADF91CF91089572
:10795000DF93CF930F920F92CDB7DEB78FED99E003
:1079600040E950ED63E070E00E947F3FEEEBF7E00E
:10797000949108C08091C00085FFFCCF9093C60011
:10798000319694919923B1F78091C00085FFFCCF87
:107990008AE08093C6004FE452E0FA01949108C057
:1079A0008091C00085FFFCCF9093C60031969491E2
:1079B0009923B1F784B7282F80FF15C0E6EBF7E0D5
:1079C000949108C08091C00085FFFCCF9093C600C1
:1079D000319694919923B1F78091C00085FFFCCF37
:1079E0008AE08093C60021FF15C0E6EAF7E0949193
:1079F00008C08091C00085FFFCCF9093C6003196EF
:107A000094919923B1F78091C00085FFFCCF8AE063
:107A10008093C60022FF15C0E5E9F7E0949108C005
:107A20008091C00085FFFCCF9093C6003196949161
:107A30009923B1F78091C00085FFFCCF8AE0809345
:107A4000C60023FF15C0E5E8F7E0949108C08091D7
:107A5000C00085FFFCCF9093C60031969491992386
:107A6000B1F78091C00085FFFCCF8AE08093C6000B
:107A700025FF15C0E5E7F7E0949108C08091C000AC
:107A800085FFFCCF9093C600319694919923B1F76E
:107A90008091C00085FFFCCF8AE08093C60014BEB1
:107AA000EEE6F7E0949108C08091C00085FFFCCF1E
:107AB0009093C600319694919923B1F7E8E6F7E0E8
:107AC000949108C08091C00085FFFCCF9093C600C0
:107AD000319694919923B1F78091C00085FFFCCF36
:107AE0008AE08093C600FA019491EFE4F2E008C0C6
:107AF0008091C00085FFFCCF9093C6003196949191
:107B00009923B1F7E8E5F7E0949108C08091C000AF
:107B100085FFFCCF9093C600319694919923B1F7DD
:107B2000E3E4F7E0949108C08091C00085FFFCCFAA
:107B30009093C600319694919923B1F7E7E3F7E06B
:107B4000949108C08091C00085FFFCCF9093C6003F
:107B5000319694919923B1F7E9E2F7E0949108C046
:107B60008091C00085FFFCCF9093C6003196949120
:107B70009923B1F78091C00085FFFCCF8AE0809304
:107B8000C600EEE1F7E0949108C08091C00085FF47
:107B9000FCCF9093C600319694919923B1F7E2E11E
:107BA000F7E0949108C08091C00085FFFCCF9093CE
:107BB000C600319694919923B1F78091C00085FF5A
:107BC000FCCF8AE08093C600FA019491EFE4F2E0E2
:107BD00008C08091C00085FFFCCF9093C60031960D
:107BE00094919923B1F7E3E0F7E0949108C0809174
:107BF000C00085FFFCCF9093C600319694919923E5
:107C0000B1F72091451230914612CE01019621150F
:107C1000310519F48B54924102C0821B930B9A8355
:107C2000898369817A818FED99E04AE050E00E9472
:107C3000CB40ECEEF6E0949108C08091C00085FF47
:107C4000FCCF9093C600319694919923B1F78FEDB4
:107C500099E060ED74E04AE050E00E94CB408091F2
:107C6000C00085FFFCCF8AE08093C6001092C40755
:107C70001092C5071092C6071092C7070E945B9129
:107C80000E9438750E94C8580E9438930E940C695F
:107C90000E947BCB80E197E220E931E0F901319746
:107CA000F1F70197D9F70F900F90CF91DF910895D9
:107CB000BC01809158099091590904970CF070C04B
:107CC000209152093091530980E690E0AC01249F45
:107CD000C001259F900D349F900D11248253984F21
:107CE0000E940E11EFE4F2E0949108C08091C00070
:107CF00085FFFCCF9093C600319694919923B1F7FC
:107D0000E6ECF7E0949108C08091C00085FFFCCFBD
:107D10009093C600319694919923B1F7209152091E
:107D20003091530980E690E0289FF001299FF00DE3
:107D3000389FF00D1124E253F84F07C08091C00026
:107D400085FFFCCF31969093C60090819923B1F7BF
:107D5000E4ECF7E0949108C08091C00085FFFCCF6F
:107D60009093C600319694919923B1F78091C00009
:107D700085FFFCCF8AE08093C600C901019664E0CC
:107D800070E00E9497D89093530980935209809194
:107D9000580990915909019690935909809358096F
:107DA0000895BC01809158099091590904970CF0ED
:107DB00070C0209152093091530980E690E0AC01E7
:107DC000249FC001259F900D349F900D1124825354
:107DD000984F0E948211EFE4F2E0949108C08091E4
:107DE000C00085FFFCCF9093C600319694919923F3
:107DF000B1F7E3EDF7E0949108C08091C00085FFF2
:107E0000FCCF9093C600319694919923B1F72091BD
:107E100052093091530980E690E0289FF001299F94
:107E2000F00D389FF00D1124E253F84F07C08091F8
:107E3000C00085FFFCCF31969093C60090819923B6
:107E4000B1F7E1EDF7E0949108C08091C00085FFA3
:107E5000FCCF9093C600319694919923B1F780910D
:107E6000C00085FFFCCF8AE08093C600C90101965F
:107E700064E070E00E9497D8909353098093520970
:107E800080915809909159090196909359098093CE
:107E9000580908951F920F920FB60F920BB60F92CA
:107EA00011242F933F934F938F939F93EF93FF93BF
:107EB0004091C600E091DB09F091DC0931969F0109
:107EC0002F77307031978091DD099091DE09281766
:107ED000390739F0E55AF64F40833093DC09209397
:107EE000DB09FF91EF919F918F914F913F912F91DE
:107EF0000F900BBE0F900FBE0F901F9018959A0118
:107F0000AB01203081EE380780E0480780E0580759
:107F100049F182E08093C00060E079E08DE390E079
:107F20000E94CCD82150304040405040CA01B90195
:107F300022E030E040E050E00E94CCD83093C50011
:107F40002093C4008091C10080618093C100809122
:107F5000C10088608093C1008091C10080688093D7
:107F6000C10008951092C00020E130E0E7CF2091D9
:107F7000DD093091DE098091DB099091DC098217DF
:107F8000930719F42FEF3FEF0EC0F901E55AF64FB2
:107F900080812F5F3F4F2F7730703093DE09209321
:107FA000DD09282F30E0C90108958091DD09909105
:107FB000DE099093DC098093DB09089508952F92E0
:107FC0003F924F925F926F927F928F929F92AF9269
:107FD000BF92CF92DF92EF92FF920F931F93DF93A6
:107FE000CF93CDB7DEB7A0970FB6F894DEBF0FBE24
:107FF000CDBF1C016A017B01411551056105710569
:1080000049F440E350E060E070E020E030E00E949E
:10801000964054C0882499245401422E5524662445
:10802000772401E010E00C0F1D1F080D191DC7017A
:10803000B601A30192010E94AAD8F80160830894B6
:10804000811C911CA11CB11CC701B601A3019201A6
:108050000E94AAD8C901DA016C017D01C114D104C2
:10806000E104F104F1F681E0E82EF12CEC0EFD1EA6
:10807000E80CF91C3E010894611C711CD501C40177
:108080000197A109B1096C01C818D90814C0F601FB
:10809000EE0DFF1D40814A3010F4405D01C0495C87
:1080A00050E060E070E0C10120E030E00E949640C6
:1080B0000894E108F1086E147F0449F7A0960FB602
:1080C000F894DEBF0FBECDBFCF91DF911F910F910E
:1080D000FF90EF90DF90CF90BF90AF909F908F90E8
:1080E0007F906F905F904F903F902F900895211553
:1080F000310539F48091C00085FFFCCF4093C60064
:1081000008950E94DF3F0895EF92FF920F931F930F
:108110009A01E62EFF2400E010E0B801A7010E94BA
:1081200077401F910F91FF90EF900895EF92FF928B
:108130000F931F93CF93DF93EC017A018B012115ED
:10814000310539F48091C00085FFFCCFE092C60074
:108150001BC02A303105B1F477FF10C04DE250E06A
:1081600060E070E020E030E00E94964010950095BD
:10817000F094E094E11CF11C011D111DCE01B80129
:10818000A7012AE00E94DF3FDF91CF911F910F915D
:10819000FF90EF900895EF92FF920F931F937B0152
:1081A0009A010027F7FC0095102FB801A7010E9443
:1081B00096401F910F91FF90EF9008950F931F939A
:1081C0008C014DE050E060E070E020E030E00E9483
:1081D0009640C8014AE050E060E070E020E030E006
:1081E0000E9496401F910F910895CF92DF92EF92D7
:1081F000FF920F931F938C019A016B01EE24FF24D1
:10820000B701A6010E947740C8010E94DE401F917D
:108210000F91FF90EF90DF90CF9008959F92AF92D3
:10822000BF92CF92DF92EF92FF920F931F93CF9363
:10823000DF93EC017A018B01922ECB01BA0120E091
:1082400030E040E050E00E94B2D488236CF4CE01CC
:108250004DE250E060E070E020E030E00E949640A7
:1082600017FB109517F9109520E030E040E05FE330
:10827000AA240BC0CA01B90120E030E040E251E479
:108280000E94B9D49B01AC01A394A91498F3C8012E
:10829000B7010E94D9D37B018C010E9426D55B01D6
:1082A0006C010E9452D59B01AC01C801B7010E942C
:1082B000D8D37B018C01CE01B601A5012AE030E0C4
:1082C0000E9477409920A1F1EDEEF2E007C0809185
:1082D000C00085FFFCCF31969093C6009081992312
:1082E000B1F726C0C801B70120E030E040E251E418
:1082F0000E9492D77B018C010E9421D55B016C0109
:10830000CC24B7FCC094DC2CCE01B601A5012AE038
:1083100030E00E949640C601B5010E9454D59B01F1
:10832000AC01C801B7010E94D8D37B018C019A949B
:108330009920C1F6DF91CF911F910F91FF90EF909F
:10834000DF90CF90BF90AF909F9008950E940E4114
:108350000895FF920F931F93CF93DF938B010E9499
:108360008F14EB01FF24FA9409C00E948F146C1B38
:108370007D0B6017710710F080E008C0FEBC0DB4E3
:1083800007FEFDCF8EB58F3F81F781E0DF91CF9162
:108390001F910F91FF900895FC014281242F30E03E
:1083A000C9019595879580658CBD40FF02C080E02E
:1083B00004C080E0463009F081E08DBD808160E03E
:1083C0000E94F5160895DF92EF92FF920F931F938C
:1083D000CF93DF93EC01D62E79018A010E94CC4124
:1083E000CE016CE271E00E94A9418D2D80648EBDAA
:1083F0000DB407FEFDCF28E130E0D801C701022E01
:1084000004C0B695A795979587950A94D2F78EBD27
:108410000DB407FEFDCF285030408FEF283F3807BE
:1084200061F7DD2011F485E906C088E0D81611F463
:1084300087E801C08FEF8EBD0DB407FEFDCF8CE045
:10844000D81631F48FEF8EBD0DB407FEFDCF8EB57B
:108450009FEF2FEF2EBD0DB407FEFDCF8EB587FF2A
:1084600004C0992311F09150F5CF8B83DF91CF9108
:108470001F910F91FF90EF90DF900895FC01808194
:1084800061E00E94F5160895DC016EBDFA0120E05E
:1084900030E00DB407FEFDCF80818EBD0DB407FE28
:1084A000FDCF81818EBD2E5F3F4F329682E020301E
:1084B000380779F70DB407FEFDCF8FEF8EBD0DB4F1
:1084C00007FEFDCF8FEF8EBD0DB407FEFDCF8FEF02
:1084D0008EBD0DB407FEFDCF8EB513968C9313970A
:1084E0008F71853011F481E0089583E111968C93AA
:1084F0001197CD010E943E4280E00895CF92DF9215
:10850000EF92FF920F931F93CF93DF93EC017A01C9
:108510008B0169018C81833039F059E0EE0CFF1C2E
:10852000001F111F5A95D1F7CE0168E1A8019701EC
:108530000E94E341882311F086E023C0CE016EEF54
:10854000A6010E9444428823E9F0CE0168E572E06A
:108550000E94A941882311F487E113C0CE016DE088
:1085600020E030E040E050E00E94E341882341F405
:108570008FEF8EBD0DB407FEFDCF8EB5882379F049
:1085800086E18983CE010E943E4280E0DF91CF9157
:108590001F910F91FF90EF90DF90CF900895CE0143
:1085A0000E943E4281E0F2CFBF92CF92DF92EF92E3
:1085B000FF920F931F93CF93DF93EC016B017A012E
:1085C0000E948F148B01BB24BA9409C00E948F149F
:1085D000601B710B6D52714010F081E10BC0BEBC8D
:1085E0000DB407FEFDCF8EB58B838F3F79F38E3FA1
:1085F00039F08FE08983CE010E943E4280E02FC097
:10860000D7011197EF28D9F08FEF8EBD20E030E031
:108610009FEF0BC00DB407FEFDCF8EB5F601E20F44
:10862000F31F80839EBD2F5F3F4F2A173B0790F3B8
:108630000DB407FEFDCF8EB5AC0DBD1D8C938FEF35
:108640008EBD0DB407FEFDCF8EB58FEF8EBD0DB480
:1086500007FEFDCF8EB5CE010E943E4281E0DF9144
:10866000CF911F910F91FF90EF90DF90CF90BF902F
:108670000895CF92DF92EF92FF920F931F93CF93C3
:10868000DF93EC017A018B0169018C81833039F031
:10869000A9E0EE0CFF1C001F111FAA95D1F7CE0117
:1086A00061E1A80197010E94E341882339F084E049
:1086B0008983CE010E943E4280E006C0CE01B60111
:1086C00040E052E00E94D442DF91CF911F910F9180
:1086D000FF90EF90DF90CF900895BF92CF92DF92FE
:1086E000EF92FF920F931F93CF93DF93EC01B62E7F
:1086F0001C82198248830E948F146B01888161E07B
:108700000E944216CE010E943E4282E360E00E9437
:10871000421683E361E00E94421684E361E00E9416
:10872000421685E361E00E94421685E361E00E9403
:10873000F51685E08A8382E58CBD1DBC80E09FEF45
:108740009EBD0DB407FEFDCF8F5F8A30C9F709C00B
:108750000E948F146C197D09615D774010F081E0F3
:108760005EC0CE0160E020E030E040E050E00E94DA
:10877000E341182F8B83813059F7CE0168E02AEA54
:1087800031E040E050E00E94E34182FF02C01C83E0
:1087900011C080E02FEF2EBD0DB407FEFDCF9EB5BA
:1087A0008F5F8430C1F79B839A3A11F082E037C023
:1087B00082E08C838C81823021F0EE24FF248701BB
:1087C0000FC0E12CF12C012D00E4102F09C00E94F4
:1087D0008F146C197D09615D774010F08AE01FC02D
:1087E000CE0167E320E030E040E050E00E94E3414A
:1087F000CE0169E2A80197010E94E3418B8388239F
:1088000031F78C81823029F5CE016AE320E030E037
:1088100040E050E00E94E341882331F088E0898302
:10882000CE010E943E4221C08FEF8EBD0DB407FEE7
:10883000FDCF8EB5807C803C11F483E08C8380E09A
:108840009FEF9EBD0DB407FEFDCF2EB58F5F833029
:10885000C1F7CE010E943E4286E08B1518F488E1F4
:10886000898303C0BA8281E001C080E0DF91CF91AB
:108870001F910F91FF90EF90DF90CF90BF900895E0
:10888000CF93DF93EB01DC0190E020E03EE28C919E
:10889000803269F0283029F4FE01E90FF11D3083A0
:1088A0009F5FFE01E90FF11D8C9180839F5F2F5F19
:1088B00011962B3061F7C90FD11D1882DF91CF912E
:1088C0000895CF93DF93DC01EB01BA0180E090E0E3
:1088D00020E2FE01E80FF91F208301968B309105FD
:1088E000C1F757E040E022C02E3219F08EED97E03C
:1088F00007C05A3049F15AE048E017C0321721F159
:10890000FC01019634913323C9F75417E8F0213262
:10891000D8F02F37C8F4822F81568A3108F42052BC
:10892000FE01E40FF11D20834F5F11962C9122234D
:1089300011F02F32C9F6FB01B183A08390E088814A
:10894000803219F091E001C090E0892FDF91CF9142
:1089500008956F927F928F929F92AF92BF92CF9223
:10896000DF92EF92FF920F931F93CF93DF93EC016F
:108970007A018B012B81222309F480C089899A898D
:10898000AB89BC8984179507A607B70708F476C09A
:1089900085C0E114F1040105110551F41C821D820A
:1089A0001E821F82188619861A861B8681E067C080
:1089B000288539854A855B85E98DFA8D858590E026
:1089C0000996215030404040504039014A01082E5C
:1089D00004C096948794779467940A94D2F72F5F93
:1089E0003F4F4F4F5F4F0894E108F108010911090B
:1089F0005701680104C0D694C794B794A7948A9588
:108A0000D2F70894E11CF11C011D111DA614B70436
:108A1000C804D90428F0211531054105510549F450
:108A20008D899E89AF89B88D8C839D83AE83BF83EA
:108A300016C0A618B708C808D90811C04C815D81B6
:108A40006E817F81898D9A8D94010E945550089482
:108A5000A108B108C108D108882331F40FC084E00F
:108A6000882E912C8C0E9D1EA114B104C104D1043A
:108A700029F7E886F9860A871B8798CF80E0DF917F
:108A8000CF911F910F91FF90EF90DF90CF90BF900B
:108A9000AF909F908F907F906F900895223009F053
:108AA00078CFE7CFCF93DF93EC018C859D85AE85A2
:108AB000BF8540E0611141E0BC01CD010E942B4E19
:108AC000882319F420E030E00AC08889282F30E09C
:108AD00095E0220F331F9A95E1F72A51364FC901CD
:108AE000DF91CF9108950F931F93CF93DF938C0164
:108AF000FC0183818823F1F1818187FF38C0C8019F
:108B000061E00E945245EC010097A1F18881853E09
:108B100089F1F8018381823040F481899289A389A7
:108B2000B4898C8F9D8FAE8FBF8FF8018589968910
:108B30009B8F8A8F85899689A789B08DCD01AA27B9
:108B4000BB279D8B8C8BE091E009F091E109309778
:108B500051F0BE016A5E7F4FCE0148961995888D0F
:108B6000998D9B8B8A8BF80181818F7781830E94FD
:108B7000F04D04C081E0F801808380E0DF91CF9167
:108B80001F910F9108950F931F938C010E947345BD
:108B9000F80113821F910F910895FC0183818823AE
:108BA00019F0CF010E94C3450895CF93DF93FC01D4
:108BB000EB018381882391F08250823020F48FE290
:108BC0008883198209C0CF0160E00E945245009756
:108BD00029F0BE010E94404481E001C080E0DF91A5
:108BE000CF9108956F927F928F929F92AF92BF9292
:108BF000CF92DF92EF92FF920F931F93DF93CF9369
:108C000000D00F92CDB7DEB77C015A016B01DC01B9
:108C100013968C911397813009F091C011968C9125
:108C200081FF8DC0A0C00097A105B10511F481E0BE
:108C300087C0F7016084718482849384C701B60180
:108C4000A5010E94A944882309F479C0D701599647
:108C50008D919C915A97A114B104C104D10489F457
:108C600055964D915D916D917C9158970E94CB5096
:108C7000882309F464C0F701158A168A178A108EB2
:108C800044C0D70114964D915D916D917C911797D9
:108C90009E012F5F3F4F0E945550882309F44FC01B
:108CA000D7015996ED91FC915A9749815A816B8170
:108CB0007C818789803149F4483FBFEF5B07B0E092
:108CC0006B07B0E07B0748F020C0483F8FEF5807A4
:108CD0008FEF68078FE07807C0F4CF010E94CB5078
:108CE000882369F1D70114964D915D916D917C9126
:108CF000179759968D919C915A970FEF1FEF2FEF71
:108D00003FE00E94CE4F8823D1F0F701A18AB28ABA
:108D1000C38AD48A818180688183C7010E94734598
:108D2000882369F0B601A5016A147B048C049D04B4
:108D300010F4B401A301C7010E94A94401C080E05E
:108D40000F900F900F900F90CF91DF911F910F9187
:108D5000FF90EF90DF90CF90BF90AF909F908F905B
:108D60007F906F900895F70181899289A389B489D2
:108D700084179507A607B70708F055CFE0CFCF9324
:108D8000DF93EC0140E050E060E070E00E94F245CB
:108D9000882369F0CE0161E00E945245FC010097F2
:108DA00031F085EE80831B820E94F04D01C080E08F
:108DB000DF91CF9108952F923F924F925F926F92E1
:108DC0007F928F929F92AF92BF92CF92DF92EF925B
:108DD000FF920F931F93CF93DF93EC012A018B81B6
:108DE000882309F4B6C0898180FFB3C0C8C02501BB
:108DF0004E185F083B0174E0272E312C2C0E3D1ECF
:108E00004201A1C0288539854A855B856FEFA62E72
:108E100061E0B62EA222B3228B8179018A0199E00A
:108E200016950795F794E7949A95D1F7E98DFA8D01
:108E3000823049F4428D538D648D758D4E0D5F1DCA
:108E4000601F711F3FC0D480DA94DE20A114B104EA
:108E5000D9F4DD20C9F4211531054105510549F446
:108E60008D899E89AF89B88D8C839D83AE83BF83A6
:108E70000BC04C815D816E817F81CF0191010E9489
:108E80005550882309F465C0E98DFA8D4C815D81C8
:108E90006E817F814250504060407040058404C024
:108EA000440F551F661F771F0A94D2F78685978552
:108EB000A089B189480F591F6A1F7B1F4D0D511D95
:108EC000611D711D80E092E08A199B09840188155B
:108ED000990508F48C0182E00030180709F067C09A
:108EE0008091E2099091E309A091E409B091E5092C
:108EF000481759076A077B0709F459C08091E60BA8
:108F00009091E70B93010E943943882349F421C0D3
:108F100095012A51364FC301B901A8010E9463117E
:108F2000600E711E980140E050E088859985AA8501
:108F3000BB85820F931FA41FB51F88879987AA87B7
:108F4000BB87801A910A8114910409F05BCFA201BA
:108F500002C04FEF5FEFCA01DF91CF911F910F91D8
:108F6000FF90EF90DF90CF90BF90AF909F908F9049
:108F70007F906F905F904F903F902F900895A988B9
:108F8000BA88CB88DC88E884F9840A851B859A0135
:108F900040E050E0D601C5018E199F09A00BB10B2E
:108FA000281739074A075B0708F021CF23CFCB01E9
:108FB000BA0140E00E942B4E882309F0A9CFC9CF07
:108FC000CF92DF92EF92FF920F931F93CF93DF9395
:108FD0007C01EB018A01FC018381823008F46FC0BF
:108FE00080859185A285B3858F719070A070B070D7
:108FF0000097A105B10509F062C06DC0F8011082AB
:10900000EDE0CE2ED12CC701BE0140E250E00E941F
:10901000DB469C018032910521F0009709F04FC09A
:1090200050C04881442309F44CC0453E61F34E32A0
:1090300051F38B858F738F30E9F501151105D1F14F
:109040008A8D9B8D892BB1F5842F90E08F71907064
:10905000009781F1833091056CF58C9D90018D9D79
:10906000300D9C9D300D11242D503040F801E20F41
:10907000F31F898180838B8181838D8182838F819E
:109080008383898584838E858583888986838A897D
:1090900087838C8980878E898187888D82878C8D54
:1090A00083878E8D8487888186FF04C0F801E20F54
:1090B000F31F15868B8583FDA6CF822F03C08FEF0C
:1090C00001C080E0DF91CF911F910F91FF90EF9051
:1090D000DF90CF9008954115510509F08FCF90CFC3
:1090E000DF93CF930F92CDB7DEB7BE016F5F7F4F97
:1090F00041E050E00E94DB46019719F02FEF3FEF6F
:1091000003C08981282F30E0C9010F90CF91DF91F2
:109110000895EF92FF920F931F93CF93DF93EC018B
:109120008B81823038F1E884F9840A851B85CE0171
:109130000E94704897FD1EC088859985AA85BB85C9
:109140004F96A11DB11D88879987AA87BB87A5E087
:1091500016950795F794E794AA95D1F72E2D30E050
:109160002F703070F5E0220F331FFA95E1F72A5186
:10917000364F02C020E030E0C901DF91CF911F914E
:109180000F91FF90EF9008950F931F93CF93DF936C
:10919000EC018B018B81882309F040C0FB0187899A
:1091A000803109F041C082E08B831D8A1E8A1F8AAC
:1091B000188E808D918DA0E0B0E045E0880F991F5A
:1091C000AA1FBB1F4A95D1F7898B9A8BAB8BBC8B9F
:1091D00013C083E08B83F801428D538D648D758DB0
:1091E0004D8B5E8B6F8B788F9E012F5E3F4FC8013A
:1091F0000E942951882391F01A8F098F81E0898379
:109200001C821D821E821F82188619861A861B8662
:109210001C861D861E861F86188A01C080E0DF918D
:10922000CF911F910F9108958032C1F7D2CF1F9334
:10923000CF93DF93EC01142F262F30E0F90175E076
:10924000EE0FFF1F7A95E1F7EA51F64F83858171A2
:1092500021F0842F827109F069C08091E209909118
:10926000E309A091E409B091E5098C879D87AE8759
:10927000BF87688BF90165E0EE0FFF1F6A95E1F784
:10928000EA51F64F84899589A0E0B0E0DC01992786
:1092900088278D8B9E8BAF8BB88F228D338DA90144
:1092A00060E070E0482B592B6A2B7B2B4D8B5E8B3B
:1092B0006F8B788F838590E088719070009751F460
:1092C000848D958DA68DB78D898B9A8BAB8BBC8B3E
:1092D00081E00CC0409751F59E012F5E3F4F898D74
:1092E0009A8D0E942951882309F184E08B83812F74
:1092F0008F7089831C821D821E821F8218861986A8
:109300001A861B8614FF18C0CE0140E050E060E0D2
:1093100070E00E94F245882379F40AC049895A898D
:109320006B897C89CE010E94A94402C01B8280E027
:10933000DF91CF911F91089515FDF0CF81E0F8CF17
:10934000CF93DF93EC019C012C5F3F4F898D9A8D69
:1093500041E050E060E070E00E9495518823A1F068
:109360008D899E89AF89B88D0097A105B10559F403
:109370008C819D81AE81BF818D8B9E8BAF8BB88F91
:1093800089818068898381E0DF91CF9108952F9250
:109390003F924F925F927F928F929F92AF92BF9235
:1093A000CF92DF92EF92FF920F931F93DF93CF93B1
:1093B00000D000D0CDB7DEB76C01162F072F5E832B
:1093C0004D83DC0113968C911397813009F06FC1A6
:1093D00011968C9181FF6BC188C1F6014189528938
:1093E0006389748980859185A285B38584179507E3
:1093F000A607B70731F0C6010E94A944882309F4E3
:1094000056C1812F902F9C0119014D805E8013C1A0
:10941000D6015996ED91FC915A97DA01C90149E0BC
:10942000B695A795979587954A95D1F774807A94C4
:1094300078228FEF882E81E0982E82229322772047
:1094400009F053C08114910409F04FC0D60114965D
:109450004D915D916D917C91179741155105610575
:10946000710581F455968D919D910D90BC91A02D23
:109470000097A105B10561F1F60184839583A68368
:10948000B78333C0CF019E012F5F3F4F0E945550DD
:10949000882309F40CC129813A814B815C81D60172
:1094A0005996ED91FC915A978789803149F4283F6C
:1094B000BFEF3B07B0E04B07B0E05B0778F008C0B8
:1094C000283FEFEF3E07EFEF4E07EFE05E0730F08B
:1094D000C6010E94A049882341F4E9C0D601149630
:1094E0002D933D934D935C93179780E092E08819FC
:1094F000990952018415950508F45C01D601599625
:10950000ED91FC915A971496ED90FD900D911C9160
:1095100017978EEF9FEFAFEFBFEFE80EF91E0A1F10
:109520001B1F058404C0EE0CFF1C001F111F0A94B2
:10953000D2F786859785A089B189E80EF91E0A1FA2
:109540001B1FE70CF11C011D111D90E0A91692E0F4
:10955000B90639F58091E2099091E309A091E409F7
:10956000B091E5098E159F05A007B10771F410921F
:10957000E80B8FEF9FEFAFEFBFEF8093E20990937F
:10958000E309A093E409B093E5098091E60B90917B
:10959000E70BB801A70191010E947E428823B9F52B
:1095A00086C08114910419F5D60118962D913D912C
:1095B0004D915C911B9751968D919D910D90BC9111
:1095C000A02D281739074A075B0788F00E94F04D45
:1095D000882309F46CC081E08093E80BE092E209F3
:1095E000F092E3090093E4091093E50908C0C8016B
:1095F000B70141E00E942B4E882309F458C0940122
:109600002A51364FC901B101A5010E94631195018C
:1096100040E050E0F60180859185A285B385820FF8
:10962000931FA41FB51F80879187A287B3872A0C39
:109630003B1C4A185B08D60118962D913D914D911F
:109640005C911B974114510409F0E2CE51968D9123
:109650009D910D90BC91A02D82179307A407B5078B
:1096600048F4F601218B328B438B548B81818068C7
:10967000818311C08091E0099091E109892B59F013
:109680008D819E81892B39F0D60111968C9111978D
:10969000806811968C93F601818183FF05C0C60115
:1096A0000E947345882319F04D815E8105C081E0D9
:1096B000D6018C934FEF5FEFCA0126960FB6F89450
:1096C000DEBF0FBECDBFCF91DF911F910F91FF90F5
:1096D000EF90DF90CF90BF90AF909F908F907F9052
:1096E0005F904F903F902F90089582FD76CE89CE67
:1096F000DF92EF92FF920F931F93CF93DF93EC01D2
:1097000089899A89AB89BC89805E9F4FAF41B040FF
:1097100008F071C0CE010E94A049882309F46BC0F3
:109720000E94F04D882309F466C0E98DFA8DEC8023
:10973000FD800E811F818EEF9FEFAFEFBFEFE80E30
:10974000F91E0A1F1B1F058404C0EE0CFF1C001F1E
:10975000111F0A94D2F786859785A089B189E80EF2
:10976000F91E0A1F1B1F81E08093E80BE092E209BB
:10977000F092E3090093E4091093E50980E092E098
:10978000E6EEF9E0DF019C011D9221503040E1F747
:10979000DD24D39411C0B801A7014D0D511D611DE9
:1097A000711D8091E60B9091E70B26EE39E00E9447
:1097B0007E42882301F1D394E98DFA8D8481D816F5
:1097C00050F320E032E040E050E0058404C0220F76
:1097D000331F441F551F0A94D2F789899A89AB8990
:1097E000BC89820F931FA41FB51F898B9A8BAB8BEB
:1097F000BC8B81E001C080E0DF91CF911F910F9180
:10980000FF90EF90DF9008958F929F92AF92BF925A
:10981000CF92DF92EF92FF920F931F93CF93DF933C
:109820006C01EB01942E852EA22E898D9A8DD60186
:109830005A969C938E935997CB0140E050E060E09C
:1098400070E00E94A944BB2438C0CE010E94894820
:10985000FC01009709F493C055E016950795F7941D
:10986000E7945A95D1F71E2D1F708081882311F03F
:10987000853EC9F4BB2099F42091E2093091E309B7
:109880004091E4095091E509D6011C962D933D9332
:109890004D935C931F9750961C93BB24B394808187
:1098A000882359F418C0892D982DBF014BE050E052
:1098B0000E945611009709F470C0E884F9840A8563
:1098C0001B8589899A89AB89BC89E816F9060A073C
:1098D0001B0708F4BACFA6FE52C0A1FE50C0BB20A1
:1098E00051F0F6011089C60161E00E945245EC0179
:1098F000009769F444C08B81823009F440C0CE01E6
:109900000E94784B8823D9F110E0C6EED9E080E2BE
:10991000DE011D928A95E9F7DE01292D382DC90156
:10992000FC018BE001900D928150E1F7E091E0099C
:10993000F091E109309739F0BE01625F7F4FCE01AF
:109940004096199508C081E298E2998B888B80E057
:1099500098E09F878E87888999899B8B8A8B998FBE
:10996000888F8E859F859F8B8E8B0E94F04D8823DC
:1099700031F0C601612F4A2D0E94174901C080E0D5
:10998000DF91CF911F910F91FF90EF90DF90CF90DB
:10999000BF90AF909F908F900895A7FEEACFEFCF32
:1099A0002F923F924F925F926F927F928F929F92EF
:1099B000AF92BF92CF92DF92EF92FF920F931F93DD
:1099C000DF93CF93CDB7DEB7C654D0400FB6F8942F
:1099D000DEBF0FBECDBF3C016B01DE01AE5BBF4FF2
:1099E00011965C934E9325962FAF25971C861F8664
:1099F0001FA21AA66115710509F480C0FC018381BC
:109A0000882309F07BC0FA0180818F32F1F0860152
:109A1000ECE0EE2EF12CEC0EFD1E72E4A72EB12C24
:109A2000AC0EBD1E4E010894811C911C2796FFAE02
:109A3000EEAE279767E2262E312C2C0E3D1E270115
:109A400024C01196B183A08301C0FD01A081B18122
:109A50008C918F32B1F3D60113968C91139782506B
:109A60008230A8F28E01095D1F4F59966D917C914D
:109A70005A97C8010E94C448882351F63FC0342D2C
:109A8000252D8701832F922F7C01F5018081918103
:109A9000B401A5010E946144882329F42FC03196A6
:109AA000D501ED93FC93D501ED91FC9180818F322E
:109AB000B1F38823C9F0C701B801A40121E00E94D5
:109AC000044C8823D9F00C151D0519F0C8010E941B
:109AD000C3452796EEADFFAD2797EE16FF0679F644
:109AE000C101322D292FCDCFC301B801A401259684
:109AF0002FAD25970E94044C182F01C010E0CE0115
:109B000087960E94CD45CE010C960E94CD45812FAF
:109B1000CA5BDF4F0FB6F894DEBF0FBECDBFCF914B
:109B2000DF911F910F91FF90EF90DF90CF90BF904A
:109B3000AF909F908F907F906F905F904F903F90ED
:109B40002F9008950F931F93DF93CF93CDB7DEB778
:109B50006B970FB6F894DEBF0FBECDBF9C01AB0173
:109B600019821C828E010F5F1F4FC801B90122E0CC
:109B70000E94D04C882311F410E004C0C8010E9458
:109B8000BF46182FCE0101960E94CD45812F6B96BE
:109B90000FB6F894DEBF0FBECDBFCF91DF911F91FE
:109BA0000F910895DB010D900020E9F71197A61B96
:109BB000B70B0496AD010E94C7490895DF93CF9378
:109BC0000F92CDB7DEB769830496BE016F5F7F4FFA
:109BD00041E050E00E94C7490F90CF91DF91089576
:109BE0008091E80B882399F14091E2095091E309B3
:109BF0006091E4097091E5098091E60B9091E70B83
:109C000026EE39E00E947E42882319F14091E90B4B
:109C10005091EA0B6091EB0B7091EC0B41155105E3
:109C20006105710591F08091E60B9091E70B26EEAE
:109C300039E00E947E42882361F01092E90B109275
:109C4000EA0B1092EB0B1092EC0B1092E80B81E0F8
:109C5000089580E00895DF92EF92FF920F931F9393
:109C60007B018C01D42E8091E2099091E309A091AF
:109C7000E409B091E5098E159F05A007B107C1F071
:109C80000E94F04D8823E1F08091E60B9091E70B64
:109C9000B801A70126EE39E00E943943882381F0FC
:109CA000E092E209F092E3090093E4091093E509D8
:109CB000DD2011F481E005C081E08093E80B01C054
:109CC00080E01F910F91FF90EF90DF9008958F92A9
:109CD0009F92AF92BF92CF92DF92EF92FF920F933B
:109CE0001F93CF93DF936C01142F7093E70B609356
:109CF000E60BFC01178A82E090E0A0E0B0E08083F0
:109D00009183A283B3831092E80B1092E90B109217
:109D1000EA0B1092EB0B1092EC0B8FEF9FEFAFEF73
:109D2000BFEF8093E2099093E309A093E409B09315
:109D3000E509442321F488249924540140C0453086
:109D400008F01EC160E070E080E090E040E00E941A
:109D50002B4E882309F414C1C12FD0E02197FE01B6
:109D600074E0EE0FFF1F7A95E1F7EA51F64FE254E7
:109D7000FE4F8081EE5BF14090E08F779070892BF1
:109D800009F0FEC0E653FE4F80819181A281B3812C
:109D900084369105A105B10508F4F2C064E0CC0F4A
:109DA000DD1F6A95E1F7C455D44F88809980AA8059
:109DB000BB8081149104A104B10409F4E1C0C50180
:109DC000B40140E00E942B4E882309F4D9C0809151
:109DD000F1099091F2098050924009F0D1C0209190
:109DE000F609222309F4CCC08091F4099091F50979
:109DF000892B09F4C5C08091F309882309F4C0C0F8
:109E0000F601228B8091F3098483158661E070E06E
:109E100007C04F5FF60145874150483008F0B0C099
:109E2000F6014585848190E09B01042E02C0220F3B
:109E3000331F0A94E2F78217930759F72091FC0920
:109E40003091FD092115310519F040E050E008C0BE
:109E500020910A0A30910B0A40910C0A50910D0A88
:109E6000F6012583368347835087E090F409F0900C
:109E7000F50900E010E0E80CF91C0A1D1B1DE38A3F
:109E8000F48A058B168B8091F7099091F809918FD0
:109E9000808F6091F60970E080E090E00E9464D8C5
:109EA0006E0D7F1D801F911FF601628F738F848F4F
:109EB000958F2091F7093091F80955E0220F331F53
:109EC0005A95E1F721503E4F232F3327269540E046
:109ED00050E0260F371F481F591F26873787408BB2
:109EE000518B8091F9099091FA09009719F0A0E03F
:109EF000B0E008C08091060A9091070AA091080A74
:109F0000B091090A85017401E21AF30A040B150BDA
:109F1000A8019701280F391F4A1F5B1FF60105840E
:109F200004C056954795379527950A94D2F721870F
:109F3000328743875487253FFFE03F07F0E04F0714
:109F4000F0E05F0720F48CE0F601878B19C0255FF5
:109F50003F4F4040504018F480E1F6010EC0809120
:109F6000120A9091130AA091140AB091150AF601F1
:109F7000828F938FA48FB58F80E2878B81E001C0A1
:109F800080E0DF91CF911F910F91FF90EF90DF90D4
:109F9000CF90BF90AF909F908F9008956F927F92D7
:109FA0008F929F92AF92BF92CF92DF92EF92FF92E9
:109FB0000F931F93CF93DF93EC015A016B0138018C
:109FC0004901423051056105710508F45EC089857B
:109FD0009A85AB85BC850196A11DB11D8417950797
:109FE000A607B70708F451C08F89803129F4E52E00
:109FF000F62E072F11270CC0803209F046C07A01D7
:10A000008B0187E016950795F794E7948A95D1F729
:10A010008B899C89AD89BE89E80EF91E0A1F1B1F1A
:10A02000C801B70141E00E942B4E882371F18F894E
:10A03000803149F4F501F070EE0FFF1FEA51F64F41
:10A04000718260820DC0F501EF77F070EE0FFF1F97
:10A05000EE0FFF1FEA51F64F608271828282938277
:10A060008A89823080F08D819E81AF81B885E80E2B
:10A07000F91E0A1F1B1FE092E90BF092EA0B0093F6
:10A08000EB0B1093EC0B81E001C080E0DF91CF91EE
:10A090001F910F91FF90EF90DF90CF90BF90AF9006
:10A0A0009F908F907F906F900895CF92DF92EF9264
:10A0B000FF920F931F93CF93DF93EC017A018B01F3
:10A0C000690189859A85AB85BC850196A11DB11D65
:10A0D00084179507A607B70708F453C08F89803106
:10A0E00029F45527412F302F2F2D0CC0803209F035
:10A0F00048C09A01AB0167E056954795379527957B
:10A100006A95D1F78B899C89AD89BE89280F391F43
:10A110004A1F5B1F8091E2099091E309A091E40935
:10A12000B091E509281739074A075B0739F0CA01DA
:10A13000B90140E00E942B4E882319F18F898031AC
:10A1400059F4F701F070EE0FFF1FEA51F64F8081CE
:10A150009181A0E0B0E00EC0F701EF77F070EE0F54
:10A16000FF1FEE0FFF1FEA51F64F80819181A28100
:10A17000B381BF70F60180839183A283B38381E0B2
:10A1800001C080E0DF91CF911F910F91FF90EF9080
:10A19000DF90CF900895AF92BF92CF92DF92EF926F
:10A1A000FF920F931F93DF93CF9300D00F92CDB701
:10A1B000DEB76C017A018B0182E090E0A0E0B0E0B4
:10A1C000F60180839183A283B3835E010894A11C6E
:10A1D000B11CC601B801A70195010E945550882302
:10A1E00041F1C601B801A70100E010E020E030E035
:10A1F0000E94CE4F8823E9F0E980FA800B811C8110
:10A20000F6018789803151F4F8EFEF16FFEFFF0672
:10A21000F0E00F07F0E01F07E0F209C088EFE81652
:10A220008FEFF8068FEF08078FE0180790F281E0B4
:10A2300001C080E00F900F900F900F90CF91DF91B1
:10A240001F910F91FF90EF90DF90CF90BF90AF9054
:10A2500008954F925F926F927F928F929F92AF92EA
:10A26000BF92CF92DF92EF92FF920F931F93DF93F3
:10A27000CF9300D00F92CDB7DEB76C0149835A83DC
:10A280006B837C833901EE24FF2487012E0108941F
:10A29000411C511C812CE2E09E2EA12CB12C498145
:10A2A0005A816B817C81C60192010E94555088239E
:10A2B00039F1D501C401F601058404C0880F991F46
:10A2C000AA1FBB1F0A94D2F7E80EF91E0A1F1B1F14
:10A2D00029813A814B815C818789803131F4285F03
:10A2E0003F4F40405040D8F205C0285F3F4F4F4F8E
:10A2F0005F40A8F2F301E082F1820283138381E0E0
:10A300000F900F900F900F90CF91DF911F910F91B1
:10A31000FF90EF90DF90CF90BF90AF909F908F9085
:10A320007F906F905F904F9008952F923F924F9241
:10A330005F926F927F928F929F92AF92BF92CF92D5
:10A34000DF92EF92FF920F931F93DF93CF93CDB7DE
:10A35000DEB72F970FB6F894DEBF0FBECDBF1C013E
:10A360004A875B876C877D873F872E87DC0119963C
:10A370008D919D910D90BC91A02D0196A11DB11DB7
:10A380008E839F83A887B987F9010081118122817B
:10A390003381011511052105310549F048015901A5
:10A3A0000894811C911CA11CB11C1D8210C0D101FC
:10A3B0008D909D90AD90BC901D828A859B85AC85CB
:10A3C000BD850197A105B10511F491E09D8375014B
:10A3D00064014424552432018E010F5F1F4FF101A7
:10A3E00081859285A385B485481659066A067B0641
:10A3F00008F090C08E819F81A885B9858C159D0538
:10A40000AE05BF0550F4A2E08A2E912CA12CB12CF0
:10A41000F2E0CF2ED12CE12CF12CC101B701A60125
:10A4200098010E945550882309F474C089819A814B
:10A43000AB81BC81A70196012F5F3F4F4F4F5F4F0C
:10A440000097A105B10519F049015A010DC028195D
:10A4500039094A095B098A859B85AC85BD85281722
:10A4600039074A075B0759F00894411C511C611CCD
:10A47000711C0894C11CD11CE11CF11CB0CFC1019E
:10A48000A601B7010FEF1FEF2FEF3FE00E94CE4F65
:10A49000882399F43FC026013701089441085108E8
:10A4A00061087108C101B301A201970186010E94F0
:10A4B000CE4F882379F1730162018C149D04AE04A0
:10A4C000BF0448F3AE85BF854D915D916D917C9140
:10A4D000411551056105710539F0C10195018401EE
:10A4E0000E94CE4F8823B1F0EE85FF858082918255
:10A4F000A282B382FD81FF2359F00894811C911C34
:10A50000A11CB11CD1018D929D92AD92BC9213976A
:10A5100081E001C080E02F960FB6F894DEBF0FBE39
:10A52000CDBFCF91DF911F910F91FF90EF90DF9002
:10A53000CF90BF90AF909F908F907F906F905F90E3
:10A540004F903F902F9008952F923F924F925F929D
:10A550006F927F928F929F92AF92BF92CF92DF9233
:10A56000EF92FF920F931F93DF93CF93CDB7DEB798
:10A57000CD55D0400FB6F894DEBF0FBECDBF2F969D
:10A580009FAF8EAF2F9761967FAF6EAF61972A0115
:10A5900062962FAF629763960FAF63976496EFAEA4
:10A5A00064976896ACAEBDAECEAEDFAE6897E22ED5
:10A5B000FF24EE0CFF1CEE0CFF1C9A012E0D3F1D1C
:10A5C0002D963FAF2EAF2D97D9016D907D908D9038
:10A5D0009C90FC01EE0DFF1DC401B301208131816F
:10A5E000428153810E94D9D369AF7AAF8BAF9CAFC0
:10A5F00010E0000F111F000F111FF201E00FF11FFB
:10A600002B96FFAFEEAF2B97A080B180C280D38096
:10A610002F96EEADFFAD2F97E00FF11FC601B501EC
:10A6200020813181428153810E94D9D36DAB7EABB1
:10A630008FAB98AF64962FAD6497E22FF0E0EE0FEA
:10A64000FF1FEE0FFF1F2F96AEADBFAD2F97AE0FC2
:10A65000BF1F4D915D916D917C9129964CAF5DAF7F
:10A660006EAF7FAF299761966EAD7FAD6197E60FB4
:10A67000F71F608171818281938129962CAD3DAD58
:10A680004EAD5FAD29970E94D8D369AB7AAB8BAB47
:10A690009CAB6196AEADBFAD61971C968D919D91BF
:10A6A0000D90BC91A02D25968CAF9DAFAEAFBFAFE6
:10A6B00025972F96AEADBFAD2F971C962D913D914E
:10A6C0004D915C911F9721962CAF3DAF4EAF5FAF80
:10A6D0002197A401930150582DA73EA74FA758AB2F
:10A6E000B601A501705849A75AA76BA77CA7619628
:10A6F0006EAD7FAD6197E60EF71ED7016D917D912E
:10A700008D919C9129AD3AAD4BAD5CAD0E94D8D3F3
:10A710003B014C016196EEADFFAD61970E0F1F1F1F
:10A72000D8016D917D918D919C912DA93EA94FA944
:10A7300058AD0E94D8D35B016C016DA57EA58FA595
:10A7400098A9A60195010E9492D77B018C0169A569
:10A750007AA58BA59CA5A40193010E9492D79B0189
:10A76000AC01C801B7010E94D8D31B012C016DA513
:10A770007EA58FA598A9A40193010E9492D77B0181
:10A780008C0169A57AA58BA59CA5A60195010E94BF
:10A7900092D79B01AC01C801B7010E94D9D39B019C
:10A7A000AC01C201B1010E944CD45B016C0120E0FC
:10A7B00030E040E050E00E94B2D4882354F4C60157
:10A7C000B5012BED3FE049EC50E40E94D9D35B0189
:10A7D0006C01E8968FADE897882351F0C601B5016A
:10A7E0002BED3FE049EC50E40E94D8D35B016C01B3
:10A7F000C601B501E7962CAD3DAD4EAD5FADE79717
:10A800000E9492D729A93AA94BA95CA95F770E9417
:10A81000CDD67B018C012FE632E143E85AE30E945A
:10A82000B2D487FDF6C1C801B7010E948FD50E943E
:10A8300026D578A76FA3672B21F4E1E0F0E0F8A715
:10A84000EFA32FA138A5B90180E090E00E9452D576
:10A850007B018C01C601B501A80197010E94B9D402
:10A860006BA37CA38DA39EA369A97AA98BA99CA99C
:10A87000A80197010E94B9D46F8F78A389A39AA3E6
:10A8800025966CAD7DAD8EAD9FAD259721962CADF7
:10A890003DAD4EAD5FAD21970E94D8D3A801970181
:10A8A0000E94B9D46B8F7C8F8D8F9E8F6BA17CA102
:10A8B0008DA19EA120E030E040E05FEB0E9492D7A6
:10A8C0002BA13CA14DA15EA10E9492D720E030E0D7
:10A8D00040E85FE30E94D9D36F8B788F898F9A8F7E
:10A8E00064963FAD6497E32FF0E0EE0FFF1FEE0F8D
:10A8F000FF1F9E012F5F3F4FE20FF31F29964CADC4
:10A900005DAD6EAD7FAD29974083518362837383C4
:10A910002F96AEADBFAD2F971C964D915D916D9169
:10A920007C911F974D875E876F87788B41E050E061
:10A930005A8B498B662462967FAD6297672F70E0D1
:10A94000660F771F660F771FC901860F971F6A96DC
:10A950009FAF8EAF6A976396BFAD6397AB2FB0E0A2
:10A96000AA0FBB1FAA0FBB1F21E030E02C0F3D1F19
:10A970002A0F3B1F6C963FAF2EAF6C976E96FFAFC2
:10A98000EEAF6E971AC138E136150CF446C06DA5CE
:10A990007EA58FA598A92BA13CA14DA15EA10E94E7
:10A9A00092D77B018C0169A57AA58BA59CA52F89DF
:10A9B000388D498D5A8D0E9492D79B01AC01C801F8
:10A9C000B7010E94D9D37B018C016DA57EA58FA50F
:10A9D00098A92F89388D498D5A8D0E9492D75B0195
:10A9E0006C0169A57AA58BA59CA52BA13CA14DA1C5
:10A9F0005EA10E9492D79B01AC01C601B5010E94E5
:10AA0000D8D36DA77EA78FA798AB6394C701D80151
:10AA100089A79AA7ABA7BCA765C049895A89BA017B
:10AA200080E090E00E9452D52BA13CA14DA15EA1F7
:10AA30000E9492D77B018C01C8010E94B6D46B8B17
:10AA40007C8B8D8B9E8BB701C8010E94F5D73B0193
:10AA50004C012D96AEADBFAD2D97ED90FD900D91B3
:10AA60001C9117FB109517F910952B96EEADFFADC5
:10AA70002B972080318042805380C801B7012B89F9
:10AA80003C894D895E890E9492D75B016C01C201AD
:10AA9000B101A40193010E9492D79B01AC01C601B0
:10AAA000B5010E94D9D36DA77EA78FA798ABC80127
:10AAB000B701A40193010E9492D77B018C01C201CE
:10AAC000B1012B893C894D895E890E9492D79B01F7
:10AAD000AC01C801B7010E94D8D369A77AA78BA798
:10AAE0009CA7662469AD7AAD8BAD9CAD2DA53EA526
:10AAF0004FA558A90E94D9D36A96AEADBFAD6A974B
:10AB00006D937D938D939C9313976DA97EA98FA9C7
:10AB100098AD29A53AA54BA55CA50E94D9D36C9602
:10AB2000EEADFFAD6C9760837183828393836E96E5
:10AB3000AEADBFAD6E976D917D918D919C912F8D36
:10AB400038A149A15AA10E94D9D36E96EEADFFADAE
:10AB50006E9760837183828393836D857E858F85F5
:10AB600098892B8D3C8D4D8D5E8D0E94D9D36D873C
:10AB70007E878F87988BCE0101960E943119CE0176
:10AB80000196BE016B5F7F4FAE01475F5F4F9E0135
:10AB9000235F3F4F6896ECACFDAC0EAD1FAD6897E0
:10ABA000F8E7CF2ED12CCC0EDD1E0E948B5B2989BD
:10ABB0003A892F5F3F4F3A8B298B49895A896FA178
:10ABC00078A54617570708F4DECE61964EAD5FAD07
:10ABD0006197485F5F4F61962EAD3FAD6197245FEF
:10ABE0003F4F61968EAD9FAD6197DC0114966196E3
:10ABF000BFAFAEAF6197BD016896ECACFDAC0EADDA
:10AC00001FAD6897E8E7CE2ED12CCC0EDD1E0E943A
:10AC10008B5BC35ADF4F0FB6F894DEBF0FBECDBFBC
:10AC2000CF91DF911F910F91FF90EF90DF90CF9028
:10AC3000BF90AF909F908F907F906F905F904F905C
:10AC40003F902F90089580912D1190912E11891B86
:10AC50008F7008956093A0037093A1038093A20363
:10AC60009093A30308950F931F93CF93DF93C0E0B6
:10AC7000D0E08E01035C134FFE01EF5EF34F608165
:10AC80007181828193810E9452D5FE01EF5FF34F63
:10AC900020813181428153810E9492D70E9426D522
:10ACA000F80160837183828393832496C031D10538
:10ACB00001F7DF91CF911F910F910895FC01608101
:10ACC00071818281938120910D0C30910E0C409105
:10ACD0000F0C5091100C0E9492D70E9462D7609383
:10ACE000590C70935A0C80935B0C90935C0C89E523
:10ACF0009CE00E94586808958F929F92AF92BF92F5
:10AD0000CF92DF92EF92FF920F931F93FC018B0182
:10AD10005A01490160817181828193812091010CE6
:10AD20003091020C4091030C5091040C0E9492D778
:10AD30000E9462D73DE4C32E3CE0D32E60934D0CBD
:10AD400070934E0C80934F0C9093500CF8016081DF
:10AD50007181828193812091050C3091060C409184
:10AD6000070C5091080C0E9492D70E9462D724E0F1
:10AD7000E22EF12CEC0CFD1C6093510CF701718359
:10AD800082839383F5016081718182819381209117
:10AD9000090C30910A0C40910B0C50910C0C0E9444
:10ADA00092D70E9462D78601085F1F4F6093550CAF
:10ADB000F801718382839383F401608171818281C0
:10ADC000938120910D0C30910E0C40910F0C5091FD
:10ADD000100C0E9492D70E9462D7F6013C966093B5
:10ADE000590C718382839383C601B701A8019F0127
:10ADF0000E941E6880E090E0A0E0B0E080932F11F8
:10AE000090933011A0933111B0933211809333118C
:10AE100090933411A0933511B0933611809337116C
:10AE200090933811A0933911B0933A1180933B114C
:10AE300090933C11A0933D11B0933E1180933F112C
:10AE400090934011A0934111B09342111F910F9123
:10AE5000FF90EF90DF90CF90BF90AF909F908F903A
:10AE600008958F929F92AF92BF92CF92DF92EF920E
:10AE7000FF920F931F93CF93DF93EC016B01009729
:10AE800009F45CC08FA9882309F058C0EEA0FFA088
:10AE900008A519A5FB01B6A0A7A090A481A4C8018C
:10AEA000B7012B2D3A2D492D582D0E94B2D488235D
:10AEB0000CF044C0C801B701A80197010E9492D7C5
:10AEC0007B018C016AA97BA98CA99DA9905820E0DF
:10AED00030E040E050EC0E9492D72EA53FA548A953
:10AEE00059A90E9492D79B01AC01C801B7010E94E9
:10AEF000D9D30E94FFD77B018C016B2D7A2D892D30
:10AF0000982D9701A8010E94B2D4882324F4EB2C39
:10AF1000FA2C092D182D6B2D7A2D892D982D97013E
:10AF2000A8010E94B2D4882349F0C701D801F601D4
:10AF300086A397A3A0A7B1A781E086ABDF91CF91AD
:10AF40001F910F91FF90EF90DF90CF90BF90AF9047
:10AF50009F908F900895EF92FF920F931F93CF933E
:10AF6000DF93F0902E1100E010E020E030E04DE49F
:10AF7000E42E12C0FE9CE0011124C35AD34FC90134
:10AF8000B801AE010E9431578F2D8F5F803109F4D7
:10AF900080E0F82E98018E0180912D11F81651F75E
:10AFA000C901B80140E050E00E943157DF91CF91D4
:10AFB0001F910F91FF90EF900895AF92BF92CF92A3
:10AFC000DF92EF92FF920F931F93CF93DF93EB01EA
:10AFD0008A016115710509F466C04115510509F42E
:10AFE00062C0DAA4CBA4BCA4ADA46EA17FA188A545
:10AFF00099A52D2D3C2D4B2D5A2D0E94B2D488237E
:10B0000009F451C08FA9882309F043C0F801E6A0D4
:10B01000F7A000A511A56D2D7C2D8B2D9A2DA801D3
:10B0200097010E94C0D61816A4F5C801B701A8015F
:10B0300097010E9492D77B018C016AA97BA98CA9F8
:10B040009DA9905820E030E040E050EC0E9492D75B
:10B050002EA53FA548A959A90E9492D79B01AC01F2
:10B06000C801B7010E94D9D30E94FFD77B018C0190
:10B070006D2D7C2D8B2D9A2D9701A8010E94B2D4A5
:10B08000882324F4ED2CFC2C0B2D1A2DC701D8019C
:10B0900004C08D2D9C2DAB2DBA2D8EA39FA3A8A7E8
:10B0A000B9A781E08EABDF91CF911F910F91FF90F7
:10B0B000EF90DF90CF90BF90AF900895CF92DF9246
:10B0C000EF92FF920F93DF93CF930F920F92CDB732
:10B0D000DEB780912D118FB7F894F0902E118FBFAD
:10B0E00080912D1190E040968F1991098F7090708A
:10B0F000049704F100912D1103500F70CC24DD242E
:10B1000040E050E06DE4E62E13C0802F002309F4E8
:10B1100080E1082F01500E9DC0011124835A934FE6
:10B120009A838983B6010E94DD57A601C980DA801F
:10B130000F1559F70F900F90CF91DF910F91FF905E
:10B14000EF90DF90CF9008956091840790912E1139
:10B1500080912D119817B9F040912E11242F30E0D5
:10B160008DE490E0289FF001299FF00D389FF00DAD
:10B170001124EB55F34F608102C04F5F4F708091F7
:10B180002D114817D1F787E070E00E9462150895ED
:10B1900010922D1110922E1180E1EDE4FCE0DF0100
:10B1A0001D928A95E9F780E090E0A0E0B0E08093FE
:10B1B000331190933411A0933511B09336118093CD
:10B1C000371190933811A0933911B0933A118093AD
:10B1D0003B1190933C11A0933D11B0933E1180938D
:10B1E0003F1190934011A0934111B093421180936D
:10B1F0002F1190933011A0933111B0933211089513
:10B200002F923F924F925F926F927F928F929F9276
:10B21000AF92BF92CF92DF92EF92FF920F931F9364
:10B22000DF93CF93CDB7DEB766970FB6F894DEBF46
:10B230000FBECDBF9E8B8D8B6A017B0148015901EA
:10B24000DC01D8966D917D918D919C91DB970E9448
:10B2500052D5698B7A8B8B8B9C8BA70196010E94B0
:10B2600092D70E949FD40E9426D56D837E838F83C0
:10B27000988769897A898B899C89A50194010E94A4
:10B2800092D70E949FD40E9426D569837A838B83AC
:10B290009C832D813E814F8158852837310541059A
:10B2A000510540F448E750E060E070E04D835E8374
:10B2B0006F83788769817A818B819C81683771057A
:10B2C0008105910540F488E790E0A0E0B0E0898333
:10B2D0009A83AB83BC83AD89BE89AC5BBF4FAD9015
:10B2E000BD90CD90DC901397A454B040BE8BAD8B35
:10B2F0006D817E818F8198850E9452D56D877E8772
:10B300008F87988BC601B5010E9454D51B012C0173
:10B3100020E030E040E050E00E94B2D4882321F4E5
:10B32000E0E070E060E028C069897A898B899C89B7
:10B330009B01AC010E9492D77B018C016D857E85BB
:10B340008F8598899B01AC010E9492D79B01AC012B
:10B35000C801B7010E94D8D37B018C01C201B101A1
:10B36000A20191010E94D9D39B01AC01C801B70190
:10B370000E94B9D4E62F692F2E2F372F482F562F32
:10B38000B901CA010E949FD40E9421D53B014C0102
:10B3900069817A818B819C810E9452D569877A87E5
:10B3A0008B879C8766277727CB016A197B098C09D5
:10B3B0009D090E9454D55B016C0120E030E040E023
:10B3C00050E00E94B2D4882321F4E0E070E060E015
:10B3D00028C069857A858B859C859B01AC010E947C
:10B3E00092D77B018C0169897A898B899C899B0121
:10B3F000AC010E9492D79B01AC01C801B7010E9429
:10B40000D8D37B018C01C601B501A60195010E942C
:10B41000D9D39B01AC01C801B7010E94B9D4E62F72
:10B42000692F2E2F372F482F562FB901CA010E949E
:10B430008FD5ED89FE89A088B188C288D38886011E
:10B440007501E618F708080919090E9421D5A80115
:10B450009701261B370B480B590B57FF71C0C201D0
:10B46000B10120E030E040E050E00E94B2D48823F7
:10B4700021F4E0E070E060E044C0C201B101A2014B
:10B4800091010E94D9D37B018C01C601B5010E94B4
:10B4900052D59B01AC01C801B7010E9492D77B0134
:10B4A0008C016D857E858F8598899B01AC010E94FA
:10B4B00092D79B01AC01C801B7010E94D8D37B0190
:10B4C0008C0169857A858B859C859B01AC010E94E6
:10B4D00092D79B01AC01C801B7010E94D9D37B016F
:10B4E0008C01C201B10120E030E040E850E40E944C
:10B4F00092D79B01AC01C801B7010E94B9D4E62FD5
:10B50000692F2E2F372F482F562FB901CA010E94BD
:10B510009FD40E9421D5AC01CB01DA013C014D0141
:10B5200097FE03C06624772443016A147B048C04CD
:10B530009D0410F03501460120E030E040E050E08D
:10B540009FB7F8946D897E89645B7F4FDB018C9196
:10B55000AC54B040BE8BAD8B882321F5FD01648ACD
:10B56000758A868A978A260D371D481D591D58965B
:10B570002D933D934D935C935B972D813E814F813D
:10B580005885DC962D933D934D935C93DF97A05C9B
:10B59000BF4F29813A814B815C812D933D934D931F
:10B5A0005C9313979FBF66960FB6F894DEBF0FBEED
:10B5B000CDBFCF91DF911F910F91FF90EF90DF9062
:10B5C000CF90BF90AF909F908F907F906F905F9043
:10B5D0004F903F902F9008954F925F927F928F925D
:10B5E0009F92AF92BF92CF92DF92EF92FF920F9312
:10B5F0001F93CF93DF9370902E11C0E0D0E07DE4D5
:10B60000472E512C46C02097B1F18EA9882361F4B2
:10B61000849CF001859CF00D949CF00D1124E35A5C
:10B62000F34F86A9882339F1EAA0FBA00CA11DA144
:10B630006EA17FA188A599A5A80197010E94B9D400
:10B640005B016C01849CF001859CF00D949CF00DD5
:10B650001124E35AF34F66A177A180A591A5A80113
:10B6600097010E94B9D48B019C01CE01B601A501BE
:10B670000E9400591EAA739480E1781609F4772479
:10B68000849CE001859CD00D949CD00D1124C35A5C
:10B69000D34F872C992487FC909480912D1190E0B2
:10B6A0008816990609F0AFCF2097F1F0EAA0FBA029
:10B6B0000CA11DA16EA17FA188A599A5A801970144
:10B6C0000E94B9D45B016C016DEC7CEC8CE49DE3D1
:10B6D000A80197010E94B9D48B019C01CE01B6014B
:10B6E000A5010E9400591EAADF91CF911F910F91D1
:10B6F000FF90EF90DF90CF90BF90AF909F908F9092
:10B700007F905F904F9008950E945E580E94AB57C3
:10B710000E94EC5A08952F923F924F925F926F923F
:10B720007F928F929F92AF92BF92CF92DF92EF92D1
:10B73000FF920F931F93DF93CF93CDB7DEB7CC5912
:10B74000D0400FB6F894DEBF0FBECDBF5C014B01F9
:10B750003A012901C756DF4FE882C959D040C65681
:10B76000DF4FF882CA59D040C556DF4F0883CB5906
:10B77000D040C456DF4F1883CC59D040E796DFAE97
:10B78000CEAEE79780912D118F5F803109F480E074
:10B79000282F332727FD30953CA72BA706C00E94F2
:10B7A0000C760E94151B0E94A0CA80912E1190E079
:10B7B0004BA55CA58417950791F36091010C7091DE
:10B7C000020C8091030C9091040CE5966CAF7DAF58
:10B7D0008EAF9FAFE597D5012D913D914D915C9135
:10B7E0000E9492D70E9462D7CD57DF4F6883C3581B
:10B7F000D040CC57DF4F7883C458D040CB57DF4F71
:10B800008883C558D040CA57DF4F9883C658D04068
:10B810002091050C3091060C4091070C5091080CBA
:10B82000E1962CAF3DAF4EAF5FAFE197CA01B901D2
:10B83000D4012D913D914D915C910E9492D70E942F
:10B8400062D7C957DF4F6883C758D040C857DF4F0A
:10B850007883C858D040C757DF4F8883C958D04035
:10B86000C657DF4F9883CA58D0402091090C3091B9
:10B870000A0C40910B0C50910C0CAD962CAF3DAFC7
:10B880004EAF5FAFAD97CA01B901D3012D913D9184
:10B890004D915C910E9492D70E9462D7C557DF4FAD
:10B8A0006883CB58D040C457DF4F7883CC58D04002
:10B8B000C357DF4F8883CD58D040C257DF4F98839E
:10B8C000CE58D04020910D0C30910E0C40910F0CB1
:10B8D0005091100CA9962CAF3DAF4EAF5FAFA9971A
:10B8E000CA01B901D2012D913D914D915C910E9407
:10B8F00092D70E9462D7C157DF4F6883CF58D0409C
:10B90000C057DF4F7883C059D040CF56DF4F888370
:10B91000C159D040CE56DF4F9883C259D040809154
:10B92000590C90915A0CA0915B0CB0915C0CC157D2
:10B93000DF4F288139814A815B81CF58D040281759
:10B9400039074A075B0709F4B8C0E0918307F0E0C4
:10B95000EE0FFF1FEE0FFF1FEF56FE4E608171814D
:10B96000828193812091A0033091A1034091A20391
:10B970005091A3030E94B2D488230CF033C0C15766
:10B98000DF4F488159816A817B81CF58D0404093F5
:10B99000590C50935A0C60935B0C70935C0CEEEE58
:10B9A000F7E0949108C08091C00085FFFCCF909390
:10B9B000C600319694919923B1F7E2E1F8E09491B1
:10B9C00008C08091C00085FFFCCF9093C6003196DF
:10B9D00094919923B1F78091C00085FFFCCF8AE054
:10B9E0008093C6008091590C90915A0CA0915B0CE9
:10B9F000B0915C0CC157DF4F288139814A815B814E
:10BA0000CF58D040281B390B4A0B5B0BCA01B90138
:10BA100057FF07C090958095709561957F4F8F4F28
:10BA20009F4F0E9454D57B018C01A9966CAD7DADD2
:10BA30008EAD9FADA99720E030E042ED53E40E9427
:10BA400092D79B01AC01C801B7010E94C0D618165D
:10BA50000CF033C0C157DF4F488159816A817B8127
:10BA6000CF58D0404093590C50935A0C60935B0CC4
:10BA700070935C0CEEEEF7E0949108C08091C000EA
:10BA800085FFFCCF9093C600319694919923B1F72E
:10BA9000E4EFF7E0949108C08091C00085FFFCCFEF
:10BAA0009093C600319694919923B1F78091C0008C
:10BAB00085FFFCCF8AE08093C60080912D11682F0E
:10BAC00070E0A5967FAF6EAFA5978DE490E0689F7C
:10BAD000F001699FF00D789FF00D1124E35AF34FA8
:10BAE000E45BFF4F1082EC54F04080914D0C90913C
:10BAF0004E0CA0914F0CB091500CA3968CAF9DAF03
:10BB0000AEAFBFAFA397CD57DF4F288139814A81B0
:10BB10005B81C358D040281B390B4A0B5B0B6F96D7
:10BB20002CAF3DAF4EAF5FAF6F9720833183428321
:10BB3000538357FF0DC0DA01C901B095A0959095C8
:10BB400081959F4FAF4FBF4F80839183A283B38373
:10BB50004091510C5091520C6091530C7091540CC7
:10BB60006B964CAF5DAF6EAF7FAF6B97C957DF4F32
:10BB700088819981AA81BB81C758D040841B950BCD
:10BB8000A60BB70B67968CAF9DAFAEAFBFAF6797F5
:10BB90008DE490E0A596AEADBFADA597A89FF0014E
:10BBA000A99FF00DB89FF00D1124E35AF34F67964B
:10BBB0002CAD3DAD4EAD5FAD679724833583468395
:10BBC000578357FF0DC0DA01C901B095A095909534
:10BBD00081959F4FAF4FBF4F84839583A683B783D3
:10BBE0004091550C5091560C6091570C7091580C27
:10BBF00063964CAF5DAF6EAF7FAF6397C557DF4FB6
:10BC000088819981AA81BB81CB58D040841B950B38
:10BC1000A60BB70B2F968CAF9DAFAEAFBFAF2F97D4
:10BC20008DE490E0A596AEADBFADA597A89FF001BD
:10BC3000A99FF00DB89FF00D1124E35AF34F2F96F2
:10BC40002CAD3DAD4EAD5FAD2F972087318742873C
:10BC5000538757FF0DC0DA01C901B095A0959095A3
:10BC600081959F4FAF4FBF4F80879187A287B38742
:10BC70002090590C30905A0C40905B0C50905C0C0A
:10BC8000C157DF4F488159816A817B81CF58D040AD
:10BC900042195309640975094DA35EA36FA378A7E0
:10BCA000E0918307F0E0EE0FFF1FEE0FFF1FEB5751
:10BCB000FC4F60817181828193812B966CAF7DAF47
:10BCC0008EAF9FAF2B97809181039091820327962F
:10BCD0009FAF8EAF27976DA17EA18FA198A597FFEB
:10BCE00007C090958095709561957F4F8F4F9F4FBE
:10BCF0000E9454D52B962CAD3DAD4EAD5FAD2B972C
:10BD00000E9492D70E9421D52796AEADBFAD27974E
:10BD10009D01442737FD4095542F0E9464D824E6A6
:10BD200030E040E050E00E94CCD88DE490E0A59651
:10BD30006EAD7FADA597689FF001699FF00D789F6C
:10BD4000F00D1124E35AF34FDF011C96248711965E
:10BD50003C93119712964C93129713965C936080C4
:10BD6000718082809380A480B580C680D780E08473
:10BD7000F18402851385C901DA018E159F05A0079C
:10BD8000B10714F4D801C7018A159B05AC05BD05A0
:10BD900014F4D601C5019C01AD0186159705A805CF
:10BDA000B90514F4A40193018DE490E0A596AEAD1D
:10BDB000BFADA597A89FB001A99F700DB89F700D4A
:10BDC0001124635A734FFB01208B318B428B538BB1
:10BDD000263031054105510510F40C94F467E85BF9
:10BDE000FF4F8091840790918507AA2797FDA09522
:10BDF000BA2F80839183A283B383DB0190961C9238
:10BE0000CD57DF4F288139814A815B81C358D040AB
:10BE1000A3968CAD9DADAEADBFADA39728173907E6
:10BE20004A075B0724F481E0DB0190968C93C957A5
:10BE3000DF4F288139814A815B81C758D0406B969A
:10BE40006CAD7DAD8EAD9FAD6B972617370748075C
:10BE5000590794F48DE490E0A596AEADBFADA597DB
:10BE6000A89FF001A99FF00DB89FF00D1124E35A8F
:10BE7000F34F80A1826080A3C557DF4F28813981AD
:10BE80004A815B81CB58D04063966CAD7DAD8EAD61
:10BE90009FAD6397261737074807590794F48DE439
:10BEA00090E0A596AEADBFADA597A89FF001A99F64
:10BEB000F00DB89FF00D1124E35AF34F80A1846078
:10BEC00080A3C157DF4F288139814A815B81CF58D8
:10BED000D040221533054405550594F48DE490E0D7
:10BEE000A5964EAD5FADA597489FF001499FF00D17
:10BEF000589FF00D1124E35AF34F80A1886080A36E
:10BF00008DE490E0A5966EAD7FADA597689FF0019A
:10BF1000699FF00D789FF00D1124E35AF34FE796D7
:10BF2000AEADBFADE7978C9181A320813181428175
:10BF3000538125962CAF3DAF4EAF5FAF25972115AE
:10BF400031054105510509F015988DE490E0A5965D
:10BF50004EAD5FADA597489FF001499FF00D589FEA
:10BF6000F00D1124E35AF34F64807580868097802A
:10BF7000611471048104910409F046988DE490E005
:10BF8000A5966EAD7FADA597689FF001699FF00DF6
:10BF9000789FF00D1124E35AF34FA084B184C2843A
:10BFA000D384A114B104C104D10409F043988DE4F1
:10BFB00090E0A596AEADBFADA597A89FF001A99F53
:10BFC000F00DB89FF00D1124E35AF34F8485958549
:10BFD000A685B7850097A105B10551F0409820903E
:10BFE000210C3090220C4090230C5090240C08C05F
:10BFF0002090390C30903A0C40903B0C50903C0C07
:10C00000C756DF4F6881C959D040C656DF4F788187
:10C01000CA59D040C556DF4F8881CB59D040C4564D
:10C02000DF4F9881CC59D040A20191010E94B2D437
:10C0300087FD16C0C756DF4F8881C959D040C65604
:10C04000DF4F9881CA59D040C556DF4FA881CB59E0
:10C05000D040C456DF4FB881CC59D0401C012D01CF
:10C060006F966CAD7DAD8EAD9FAD6F970E9454D530
:10C07000E5962CAD3DAD4EAD5FADE5970E94B9D4D0
:10C08000C158DF4F6883CF57D040C058DF4F788307
:10C09000C058D040CF57DF4F8883C158D040CE57CB
:10C0A000DF4F9883C258D040AC01CB01DA018983BD
:10C0B0009A83AB83BC8367966CAD7DAD8EAD9FAD2F
:10C0C00067970E9454D5E1962CAD3DAD4EAD5FAD66
:10C0D000E1970E94B9D4EC966FAFEC97ED967FAFE5
:10C0E000ED97EE968FAFEE97EF969FAFEF97AC017F
:10C0F000CB01DA018D839E83AF83B8872F966CAD19
:10C100007DAD8EAD9FAD2F970E9454D5AD962CADD1
:10C110003DAD4EAD5FADAD970E94B9D4E8966FAF1F
:10C12000E897E9967FAFE997EA968FAFEA97EB96A3
:10C130009FAFEB97AC01CB01DA0189879A87AB8778
:10C14000BC876DA17EA18FA198A50E9454D5A99608
:10C150002CAD3DAD4EAD5FADA9970E94B9D42B96E5
:10C160002CAD3DAD4EAD5FAD2B970E9492D77B01BC
:10C170008C012796EEADFFAD2797BF01882777FD8D
:10C180008095982F0E9454D59B01AC01C801B7013E
:10C190000E9492D720E030E048EC52E40E94B9D4EB
:10C1A0009B01AC016D877E878F87988B25966CAD40
:10C1B0007DAD8EAD9FAD25976630710581059105EA
:10C1C0001CF576E06716710481049104ECF486E0B6
:10C1D000A816B104C104D104BCF48DE490E0A59686
:10C1E000AEADBFADA597A89FF001A99FF00DB89F78
:10C1F000F00D1124E35AF34FDA01C901BF7786A786
:10C2000097A7A0ABB1AB5DC0C158DF4F2881CF5716
:10C21000D040C058DF4F3881C058D040CF57DF4F93
:10C220004881C158D040CE57DF4F5881C258D040C6
:10C23000B901CA010E9449D83B014C01EC962FADCF
:10C24000EC97ED963FADED97EE964FADEE97EF96EE
:10C250005FADEF97B901CA010E9449D85B016C013B
:10C26000E8962FADE897E9963FADE997EA964FAD8E
:10C27000EA97EB965FADEB97B901CA010E9449D8E6
:10C280007B018C01C401B301A60195010E94D9D3A1
:10C29000A80197010E94D9D30E94FFD72DE430E076
:10C2A000A5964EAD5FADA597429FF001439FF00D5F
:10C2B000529FF00D1124E35AF34F66A777A780AB86
:10C2C00091AB8DE490E0A5966EAD7FADA597689F8C
:10C2D000F001699FF00D789FF00D1124E35AF34FA0
:10C2E00086A597A5A0A9B1A921968CAF9DAFAEAFA9
:10C2F000BFAF219760E070E080E89FE321962CAD0E
:10C300003DAD4EAD5FAD21970E94B9D49B01AC010C
:10C31000C201B1010E9492D72B013C0180912D11E5
:10C3200090912E11A82FB0E05096A91BB109AF70C3
:10C33000B070BAA7A9A7A230B1050CF451C05D0135
:10C34000CC24B7FCC094DC2CC601B5010E9454D5A6
:10C3500020E030E040E051E40E94B2D488230CF0A9
:10C360003FC060E074E284E799E4A30192010E9477
:10C37000B9D40E9462D77B018C016091ED0B709162
:10C38000EE0B8091EF0B9091F00BE616F706080785
:10C39000190730F56E197F09800B910B660F771F17
:10C3A000881F991FA60195010E94AAD8CA01B90148
:10C3B0000E9452D50E9462D79B01AC012E0D3F1DF9
:10C3C000401F511FCA01B9010E9452D59B01AC0107
:10C3D00060E074E284E799E40E94B9D42B013C0147
:10C3E0008DE490E0A596EEADFFADA597E89F8001A6
:10C3F000E99F100DF89F100D1124035A134F219639
:10C400006CAD7DAD8EAD9FAD2197A30192010E94D1
:10C4100092D7D80192966D937D938D939C93959727
:10C4200050966D917D918D919C9153970E9452D51C
:10C43000A30192010E9492D70E949FD40E9426D508
:10C44000F80160AF71AF82AF93AFCD56DF4F188266
:10C45000C359D040CC56DF4F1882C459D04020E891
:10C46000222E9FE3392E88249924E1E0F0E0EC0F9E
:10C47000FD1FE80DF91DC301B20120813181428108
:10C4800053810E9492D7E1E1F0E0EC0FFD1FE80D2F
:10C49000F91D60837183828393835B016C01E8944F
:10C4A000D7F8F401EF50F44FE080F180028113815E
:10C4B000C601B501A80197010E94C0D61816CCF498
:10C4C000C801B701A60195010E94B9D46B017C0196
:10C4D000CD56DF4F6881C359D040CC56DF4F7881AD
:10C4E000C459D040C101A70196010E94B2D488234B
:10C4F0006CF4CD56DF4F8881C359D040CC56DF4F06
:10C500009881C459D040D1016C017D0124E030E014
:10C51000820E931E30E18316910471F0D701C6019B
:10C52000CD56DF4FC882C359D040CC56DF4F9883D9
:10C53000C459D0401D0199CFC701B60120E030E0B9
:10C5400040E85FE30E94B2D488230CF04CC08E0117
:10C550000F5E1F4F81E2A82EB12CAC0EBD1ED8017C
:10C560006D917D918D919C91A70196010E9492D72A
:10C57000F80161937193819391938F01EA15FB0503
:10C5800071F78DE490E0A5962EAD3FADA597289F5D
:10C590008001299F100D389F100D1124035A134F4D
:10C5A000D80192966D917D918D919C919597A7015F
:10C5B00096010E9492D7F80162A373A384A395A366
:10C5C00060AD71AD82AD93AD0E9452D5A7019601C9
:10C5D0000E9492D70E9426D5D801D8966D937D935C
:10C5E0008D939C93DB978DE490E0A596EEADFFAD27
:10C5F000A597E89F8001E99F100DF89F100D112469
:10C60000035A134FD80150966D917D918D919C9155
:10C6100053970E9452D5F80126A537A540A951A9E4
:10C620000E94B9D41B012C01F80180819181A28163
:10C63000B3810097A105B10549F584819581A68153
:10C64000B7810097A105B10509F580859185A2857F
:10C65000B3850097A105B105C9F4C201B1012091CC
:10C66000290C30912A0C40912B0C50912C0C0E94DB
:10C6700092D70E949FD40C5B1F4F0E9426D5D801F1
:10C680006D937D938D939C93139771C1C201B101FA
:10C690002091250C3091260C4091270C5091280CAC
:10C6A0000E9492D70E949FD40E9426D52DE430E0AC
:10C6B000A596EEADFFADA597E29F6001E39FD00C7C
:10C6C000F29FD00C11242DE53CE0C20ED31EB4E441
:10C6D0006B2E712C6C0C7D1CD3016D937D938D930F
:10C6E0009C93139780903D0C90903E0CA0903F0C33
:10C6F000B090400C0E9452D57B018C01F601608104
:10C700007181828193810E9454D59B01AC01C80143
:10C71000B7010E9492D77B018C01D60150966D9192
:10C720007D918D919C9153970E9452D59B01AC01B4
:10C73000C801B7010E94B9D47B018C01C501B401C5
:10C740000E9452D59B01AC01C801B7010E94C0D61E
:10C7500018162CF4F30180829182A282B382809019
:10C76000410C9090420CA090430CB090440C8DE48E
:10C7700090E0A5962EAD3FADA597289F6001299F1B
:10C78000D00C389FD00C11244DE55CE0C40ED51EB2
:10C79000A4E46A2E712C6C0C7D1CD3016D917D91EB
:10C7A0008D919C910E9452D57B018C01F601648190
:10C7B0007581868197810E9454D59B01AC01C80187
:10C7C000B7010E9492D77B018C01D60150966D91E2
:10C7D0007D918D919C9153970E9452D59B01AC0104
:10C7E000C801B7010E94B9D47B018C01C501B40115
:10C7F0000E9452D59B01AC01C801B7010E94C0D66E
:10C8000018162CF4F30180829182A282B382809068
:10C81000490C90904A0CA0904B0CB0904C0C8DE4BD
:10C8200090E0A5962EAD3FADA597289F6001299F6A
:10C83000D00C389FD00C11244DE55CE0C40ED51E01
:10C84000F4E46F2E712C6C0C7D1CD3016D917D91E5
:10C850008D919C910E9452D57B018C01F6016485DB
:10C860007585868597850E9454D59B01AC01C801CA
:10C87000B7010E9492D77B018C01D60150966D9131
:10C880007D918D919C9153970E9452D59B01AC0153
:10C89000C801B7010E94B9D47B018C01C501B40164
:10C8A0000E9452D59B01AC01C801B7010E94C0D6BD
:10C8B00018162CF4F30180829182A282B3828090B8
:10C8C000450C9090460CA090470CB090480C8DE41D
:10C8D00090E0A5962EAD3FADA597289F6001299FBA
:10C8E000D00C389FD00C11244DE55CE0C40ED51E51
:10C8F000E4E46E2E712C6C0C7D1CD3016D917D9146
:10C900008D919C910E9452D57B018C01F60160852E
:10C910007185828593850E9454D59B01AC01C80125
:10C92000B7010E9492D77B018C01D60150966D9180
:10C930007D918D919C9153970E9452D59B01AC01A2
:10C94000C801B7010E94B9D47B018C01C501B401B3
:10C950000E9452D59B01AC01C801B7010E94C0D60C
:10C9600018162CF4F30180829182A282B3828DE4A6
:10C9700090E0A5962EAD3FADA597289F6001299F19
:10C98000D00C389FD00C11244DE55CE0C40ED51EB0
:10C99000F601EC5BFF4F60817181828193810E947F
:10C9A00052D57B018C01A20191010E94B9D4D6011C
:10C9B000D2966D937D938D939C93D597C801B701C3
:10C9C0002DEB37E346E051E40E9492D70E9421D537
:10C9D000F601648F758F868F978F60902D0C709005
:10C9E0002E0C80902F0C9090300CC401B30120E0ED
:10C9F00030E040E05FE30E9492D75B016C01298D3B
:10CA00003A8D4B8D5C8D29AF3AAF4BAF5CAF409107
:10CA1000310C5091320C6091330C7091340C4DAB51
:10CA20005EAB6FAB78AFCB01BA0120E030E040E005
:10CA30005FE30E9492D77B018C0169AD7AAD8BAD2B
:10CA40009CAD9F77A80197010E94C0D6181644F4A8
:10CA5000C601B501A80197010E94B2D4882314F43D
:10CA6000860175016D8D7E8D8F8D98A169AB7AAB36
:10CA70008BAB9CAB8091350C9091360CA091370C10
:10CA8000B091380C8DA79EA7AFA7B8ABBC01CD0164
:10CA900020E030E040E05FE30E9492D71B012C01D0
:10CAA00069A97AA98BA99CA99F77A20191010E94EB
:10CAB000C0D6181644F4C801B701A20191010E9422
:10CAC000B2D4882314F4170128018DE490E0A596D0
:10CAD000AEADBFADA597A89FF001A99FF00DB89F7F
:10CAE000F00D1124E35AF34F22A133A144A155A123
:10CAF00029A33AA34BA35CA3C201B1010E94B2D403
:10CB000087FD04C029A03AA04BA05CA049A55AA566
:10CB1000423051050CF405C150912F11CB56DF4F17
:10CB20005883C559D04060913011CA56DF4F688391
:10CB3000C659D04070913111C956DF4F7883C7591B
:10CB4000D04080913211C856DF4F8883C859D040F9
:10CB5000652FCA56DF4F7881C659D040C956DF4F7E
:10CB60008881C759D040C856DF4F9881C859D040F6
:10CB700027E137EB41ED58E30E94C0D618160CF0C0
:10CB8000D0C069897A898B899C8920913311309131
:10CB9000341140913511509136110E94D8D39B0128
:10CBA000AC010E9492D77B018C016D897E898F89AF
:10CBB000988D209137113091381140913911509151
:10CBC0003A110E94D8D39B01AC010E9492D79B01DD
:10CBD000AC01C801B7010E94D9D30E94FFD77B01E5
:10CBE0008C01A40193010E94C0D618165CF00F2E90
:10CBF000F0E06F2EF0E07F2EF0E88F2EFFE39F2E07
:10CC0000F02D08C0C401B301A80197010E94B9D456
:10CC10003B014C0169AD7AAD8BAD9CAD20913B11D0
:10CC200030913C1140913D1150913E110E94D8D35A
:10CC30007B018C01E89417F9C801B7012DA93EA921
:10CC40004FA958AD0E94C0D6181694F46DA97EA9BC
:10CC50008FA998ADA80197010E94B9D45B016C011E
:10CC6000C401B301A60195010E94B2D4882314F433
:10CC70006401530169A97AA98BA99CA920913F114C
:10CC80003091401140914111509142110E94D8D3EE
:10CC90007B018C01E89417F9C801B7012DA53EA5C9
:10CCA0004FA558A90E94C0D6181694F46DA57EA56C
:10CCB0008FA598A9A80197010E94B9D47B018C0186
:10CCC000C601B501A80197010E94B2D4882314F4CB
:10CCD0008601750169A17AA18BA19CA1A801970188
:10CCE0000E9492D77B018C01CB56DF4F6881C559DA
:10CCF000D040CA56DF4F7881C659D040C956DF4F61
:10CD00008881C759D040C856DF4F9881C859D04054
:10CD1000A80197010E94B2D487FD19C0D801C701AC
:10CD200002C0D201C101CB56DF4F8883C559D04024
:10CD3000CA56DF4F9883C659D040C956DF4FA883E3
:10CD4000C759D040C856DF4FB883C859D0408DE48A
:10CD500090E0A596AEADBFADA597A89F8001A99F15
:10CD6000100DB89F100D1124035A134FCB56DF4FEF
:10CD70008881C559D040CA56DF4F9881C659D040E6
:10CD8000C956DF4FA881C759D040C856DF4FB88178
:10CD9000C859D040F80182A793A7A4A7B5A762A954
:10CDA00073A984A995A9905820E030E040E050ECA8
:10CDB0000E9492D7D8019E962D913D914D915C9104
:10CDC000D1970E9492D72BE037ED43E25BE30E94BC
:10CDD000D9D30E94FFD7F62EE72ED82EC92ECB56D8
:10CDE000DF4F6881C559D040CA56DF4F7881C65998
:10CDF000D040C956DF4F8881C759D040C856DF4F51
:10CE00009881C859D0402F2D3E2D4D2D5C2D0E946C
:10CE1000B2D487FD14C0CB56DF4FF882C559D0403D
:10CE2000CA56DF4FE882C659D040C956DF4FD88274
:10CE3000C759D040C856DF4FC882C859D0408DE48A
:10CE400090E0A596EEADFFADA597E89F8001E99F24
:10CE5000100DF89F100D1124035A134FCB56DF4FBE
:10CE60008881C559D040CA56DF4F9881C659D040F5
:10CE7000C956DF4FA881C759D040C856DF4FB88187
:10CE8000C859D040F80186A397A3A0A7B1A762A173
:10CE900073A184A195A12F2D3E2D4D2D5C2D0E94B7
:10CEA000B2D418162CF081E0D801D7968C9302C02A
:10CEB000F80117AA8DE490E0A5962EAD3FADA59799
:10CEC000289FF001299FF00D389FF00D1124E35A9F
:10CED000F34F81E086ABA3E3B1E1FE01719680E1FF
:10CEE00001900D928150E1F78DE490E0A5964EAD52
:10CEF0005FADA597489F6001499FD00C589FD00C0B
:10CF000011246DE57CE0C60ED71ED6019296ED90F9
:10CF1000FD900D911C919597E0922F11F092301198
:10CF2000009331111093321196966D917D918D91F0
:10CF30009C919997A80197010E94B9D44B015C017B
:10CF4000C201B101A80197010E94B9D48B019C01D3
:10CF5000C601B501A4010E940059BBA5B0932D11D3
:10CF6000C157DF4F288139814A815B81CF58D0403A
:10CF70002093590C30935A0C40935B0C50935C0CEB
:10CF8000C557DF4F488159816A817B81CB58D0409A
:10CF90004093550C5093560C6093570C7093580C5B
:10CFA000C957DF4F688179818A819B81C758D040FA
:10CFB0006093510C7093520C8093530C9093540CCB
:10CFC000CD57DF4F88819981AA81BB81C358D0405A
:10CFD00080934D0C90934E0CA0934F0CB093500C3B
:10CFE0000E94845B0E941868C456DF4F0FB6F89405
:10CFF000DEBF0FBECDBFCF91DF911F910F91FF908C
:10D00000EF90DF90CF90BF90AF909F908F907F90E8
:10D010006F905F904F903F902F90089510927711EE
:10D020001092791110927B1108958093AE030895A8
:10D03000EFE6F0E080818260808308951F93FC0119
:10D040001FB7F89480819181A281B381809351119F
:10D0500090935211A0935311B0935411FB0180810E
:10D060009181A281B3818093551190935611A09321
:10D070005711B0935811FA0180819181A281B38137
:10D080008093591190935A11A0935B11B0935C1146
:10D09000F90180819181A281B38180935D11909388
:10D0A0005E11A0935F11B09360111FBF1F9108958F
:10D0B000FC012FB7F89480819181A281B381809384
:10D0C0005D1190935E11A0935F11B09360112FBF1B
:10D0D0000895E82F8FB7F894F0E0EE0FFF1FEE0FE2
:10D0E000FF1FEF5AFE4E20813181428153818FBF55
:10D0F000B901CA01089580916F008D7F80936F0000
:10D1000006C080912E118F5F8F7080932E119091A9
:10D110002D1180912E11981751F4109244111092F4
:10D12000431180916F00826080936F000895909109
:10D130002D1180912E11981751F3E3CF9B01882375
:10D1400099F4B901882777FD8095982F2FEF30E06B
:10D1500040E050E00E9464D820ED37E040E050E02D
:10D160000E94CCD88CE214C08130B1F4B901882778
:10D1700077FD8095982F2FEF30E040E050E00E943F
:10D1800064D820ED37E040E050E00E94CCD88DE23A
:10D19000B9010E94621508958230A9F4B901882767
:10D1A00077FD8095982F2FEF30E040E050E00E940F
:10D1B00064D820ED37E040E050E00E94CCD88EE209
:10D1C000B9010E94621508958CE261E00E94421646
:10D1D0008DE261E00E9442168EE261E00E944216FA
:10D1E0006091A4037091A50380E00E949E68609105
:10D1F000A6037091A70381E00E949E686091A80336
:10D200007091A90382E00E949E68E1E2F1E08081D2
:10D21000887F8160808308950E94E468099A3C9A1F
:10D22000399AEAE0F1E080818064808380818460C3
:10D2300080830D9A159A3E9A469A3B9A439A389A59
:10D24000409A8081826080839FB7F894EBE0F1E0A0
:10D250008081826080839FBF0898109A0C98149AEE
:10D260000F98179A0B9A1398159A10927C073D9A6B
:10D270004598469A10927D073A9A4298439A10929E
:10D280007E07EAE0F1E08081806880839FB7F894B0
:10D29000EBE0F1E080818F7780839FBF409AEAE0E6
:10D2A000F1E08081816080839FB7F894EBE0F1E04A
:10D2B00080818E7F80839FBFA1E8B0E08C918F7EBC
:10D2C0008C938C9188608C93E0E8F0E080818D7F76
:10D2D000808380818E7F808380818F738083808133
:10D2E0008F7C80838C91887F82608C9380E090E437
:10D2F000909389008093880010928500109284009A
:10D30000EFE6F0E080818260808381E08093AE036D
:10D310007894089590912D1180912E11981739F0DD
:10D320000E940C760E94151B0E94A0CAF3CF08959C
:10D330000E948A69159A10927C07469A10927D077E
:10D34000439A10927E07409A08951F920F920FB64B
:10D350000F920BB60F921124AF92BF92CF92DF9231
:10D36000EF92FF920F931F932F933F934F935F93EF
:10D370006F937F938F939F93AF93BF93CF93DF93DD
:10D38000EF93FF938091431190914411892B09F001
:10D3900094C190912D1180912E11981719F4E0E00D
:10D3A000F0E014C080912E1190E02DE430E0829FD7
:10D3B000F001839FF00D929FF00D1124E35AF34F7B
:10D3C000E45BFF4F81E08083EC54F040F093441124
:10D3D000E0934311309709F46AC1E45BFF4F81E0A9
:10D3E0008083EC54F04010928311109284111092BB
:10D3F00085111092861160AD71AD2CE96134720710
:10D4000018F060E47CE904C03EE46132730730F058
:10D41000769567957695679584E007C047E2613118
:10D42000740730F07695679582E080937C1107C091
:10D4300080937C116032710510F460E270E06052FC
:10D44000704058E060307507E8F0472F50E0440F17
:10D45000551F440F551F455B574F9A012E5F3F4F95
:10D46000F901859194919C01AA27639FC001629F55
:10D47000810D9A1F06948A1F9A1F1124FA01459163
:10D4800054911EC0CB01969587958C7F855B934FF9
:10D49000FC0145915491FC01329625913491862FDF
:10D4A00090E087709070FC012E9FC0012F9F900D1F
:10D4B0003E9F900D1124B3E096958795BA95E1F7BC
:10D4C000481B590B44365105A8F4EFEEF2E007C0B3
:10D4D0008091C00085FFFCCF31969093C60090816B
:10D4E0009923B1F78FED99E04AE050E00E94F540B2
:10D4F00044E650E0509388114093871180917C114D
:10D500008093891110928A11E0914311F091441196
:10D5100064AD75AD7093821160938111FCE9613443
:10D520007F0718F060E47CE904C02EE461327207E2
:10D5300030F0769567957695679584E007C037E279
:10D540006131730730F07695679582E080937C11A6
:10D5500008C081E080937C116032710510F460E2B4
:10D5600070E06052704048E060307407E8F0472F88
:10D5700050E0440F551F440F551F455B574F9A010C
:10D580002E5F3F4FF901859194919C01AA27639FDB
:10D59000C001629F810D9A1F06948A1F9A1F112451
:10D5A000FA01459154911EC0CB01969587958C7FC9
:10D5B000855B934FFC0145915491FC013296259176
:10D5C0003491862F90E087709070FC012E9FC001EF
:10D5D0002F9F900D3E9F900D112433E096958795D7
:10D5E0003A95E1F7481B590B44365105A8F4EFEE84
:10D5F000F2E007C08091C00085FFFCCF3196909388
:10D60000C60090819923B1F78FED99E04AE050E090
:10D610000E94F54044E650E0CA01A0E0B0E08093EB
:10D620007D1190937E11A0937F11B0938011509340
:10D63000890040938800E0914311F0914411808962
:10D640009189A289B389B695A79597958795B09545
:10D65000A095909581959F4FAF4FBF4F80936111DB
:10D6600090936211A0936311B0936411809365113C
:10D6700090936611A0936711B0936811809369111C
:10D6800090936A11A0936B11B0936C1180936D11FC
:10D6900090936E11A0936F11B0937011109271114D
:10D6A00010927211109273111092741106C080EDD5
:10D6B00097E09093890080938800C0914311D091A6
:10D6C0004411209709F489C488A18093751180FFC3
:10D6D00003C0119A8FEF02C0119881E08093AA03D2
:10D6E0008091751181FF03C044988FEF02C0449A66
:10D6F00081E08093AB038091751180FF36C08091EB
:10D70000AE03882391F120B1217031E0232759F134
:10D7100080917611882339F188819981AA81BB8112
:10D72000181619061A061B06F4F4809151119091EF
:10D730005211A0915311B0915411809345119093BF
:10D740004611A0934711B0934811309377118889FF
:10D750009989AA89BB898093711190937211A093C2
:10D760007311B0937411209376118091751181FF1C
:10D770003AC08091AE038823B1F180B182958F7059
:10D780008095282F217080FF2CC0809178118823EC
:10D7900041F18C819D81AE81BF81181619061A0650
:10D7A0001B06FCF48091551190915611A0915711D0
:10D7B000B09158118093491190934A11A0934B1145
:10D7C000B0934C1181E08093791188899989AA8955
:10D7D000BB898093711190937211A0937311B093D0
:10D7E0007411209378118091751182FF3AC0419A8B
:10D7F0008FEF8093AC038091AE038823B1F120E0DA
:10D8000007992CC021E080917A11882339F188850D
:10D810009985AA85BB85181619061A061B06F4F405
:10D820008091591190915A11A0915B11B0915C11A6
:10D8300080934D1190934E11A0934F11B0935011BE
:10D8400020937B1188899989AA89BB89809371115A
:10D8500090937211A0937311B093741120937A1165
:10D8600004C0419881E08093AC038091751183FFDF
:10D870000AC08FB7F89490910B019F7B90930B0196
:10D880008FBF8FEF09C08FB7F89490910B01906410
:10D8900090930B018FBF81E08093AD0360E070E057
:10D8A00079C18091C00087FF19C04091C600E09106
:10D8B000DB09F091DC0931969F012F7730703197A9
:10D8C0008091DD099091DE092817390739F0E55A72
:10D8D000F64F40833093DC092093DB09288139819E
:10D8E0004A815B818091611190916211A0916311D5
:10D8F000B0916411280F391F4A1F5B1F20936111DB
:10D900003093621140936311509364111216130601
:10D91000140615066CF5139A88899989AA89BB891A
:10D92000281B390B4A0B5B0B20936111309362115A
:10D930004093631150936411209151113091521111
:10D9400040915311509154118091AA03992787FD5A
:10D950009095A92FB92F820F931FA41FB51F8093F5
:10D96000511190935211A0935311B09354111398E5
:10D970002C813D814E815F8180916511909166116E
:10D98000A0916711B0916811280F391F4A1F5B1FC2
:10D99000209365113093661140936711509368117D
:10D9A00012161306140615066CF5459A888999898E
:10D9B000AA89BB89281B390B4A0B5B0B2093651185
:10D9C000309366114093671150936811209155115F
:10D9D0003091561140915711509158118091AB03DD
:10D9E000992787FD9095A92FB92F820F931FA41F08
:10D9F000B51F8093551190935611A0935711B09372
:10DA000058114598288539854A855B85809169112B
:10DA100090916A11A0916B11B0916C11280F391F70
:10DA20004A1F5B1F2093691130936A1140936B1159
:10DA300050936C1112161306140615066CF5429AD3
:10DA400088899989AA89BB89281B390B4A0B5B0BEA
:10DA50002093691130936A1140936B1150936C11AC
:10DA60002091591130915A1140915B1150915C11E4
:10DA70008091AC03992787FD9095A92FB92F820F2C
:10DA8000931FA41FB51F8093591190935A11A0930F
:10DA90005B11B0935C1142982C853D854E855F8566
:10DAA00080916D1190916E11A0916F11B0917011D4
:10DAB000280F391F4A1F5B1F20936D1130936E1181
:10DAC00040936F1150937011121613061406150629
:10DAD000DCF59FB7F89480910B01806880930B016F
:10DAE0009FBF88899989AA89BB89281B390B4A0B52
:10DAF0005B0B20936D1130936E1140936F11509317
:10DB0000701120915D1130915E1140915F11509123
:10DB100060118091AD03992787FD9095A92FB92FAA
:10DB2000820F931FA41FB51F80935D1190935E1108
:10DB3000A0935F11B09360119FB7F89480910B018F
:10DB40008F7780930B019FBF80917111909172111B
:10DB5000A0917311B09174110196A11DB11D809314
:10DB6000711190937211A0937311B093741120915D
:10DB700071113091721140917311509174116F5F56
:10DB80007F4F88899989AA89BB89281739074A074D
:10DB90005B0738F480917C1190E0681779070CF4EA
:10DBA00080CE20917111309172114091731150917A
:10DBB00074118C899D89AE89BF8982179307A40748
:10DBC000B50708F4E3C0E0907D11F0907E1100915C
:10DBD0007F1110918011AC8CBD8CCE8CDF8CA80194
:10DBE0009701C601B501AA27279FB12D389FF001E3
:10DBF000489FF00D479FE00DF11D289FB00DE11DDE
:10DC0000FA1F379FB00DE11DFA1F469FB00DE11DB1
:10DC1000FA1F369FB10DEA1FFA1FB695EA1FFA1FC9
:10DC200011248CAD9DAD8E0F9F1F90938211809318
:10DC3000811128AD39AD4AAD5BADA0E0B0E0281749
:10DC400039074A075B0720F4309382112093811132
:10DC500060918111709182118CE96134780718F01C
:10DC600060E47CE904C09EE46132790730F0769587
:10DC700067957695679584E007C0E7E261317E0796
:10DC800030F07695679582E080937C1108C081E042
:10DC900080937C116032710510F460E270E0605294
:10DCA0007040F8E060307F07E8F0472F50E0440F05
:10DCB000551F440F551F455B574F9A012E5F3F4F2D
:10DCC000F901859194919C01AA27639FC001629FED
:10DCD000810D9A1F06948A1F9A1F1124FA014591FB
:10DCE00054911EC0CB01969587958C7F855B934F91
:10DCF000FC0145915491FC01329625913491862F77
:10DD000090E087709070FC012E9FC0012F9F900DB6
:10DD10003E9F900D1124B3E096958795BA95E1F753
:10DD2000481B590B44365105A8F4EFEEF2E007C04A
:10DD30008091C00085FFFCCF31969093C600908102
:10DD40009923B1F78FED99E04AE050E00E94F54049
:10DD500044E650E050938900409388009A0140E0E7
:10DD600050E080917D1190917E11A0917F11B09132
:10DD70008011820F931FA41FB51F80937D11909374
:10DD80007E11A0937F11B093801102C12091711177
:10DD9000309172114091731150917411888D998D49
:10DDA000AA8DBB8D82179307A407B50708F0E4C0BE
:10DDB00060918311709184118091851190918611E9
:10DDC0002C8D3D8D4E8D5F8DAA27639FB12D749F45
:10DDD000F001849FF00D839FE00DF11D649FB00D55
:10DDE000E11DFA1F739FB00DE11DFA1F829FB00D58
:10DDF000E11DFA1F729FB10DEA1FFA1FB695EA1FC7
:10DE0000FA1F112480918111909182118E179F0722
:10DE100038F4C05CDF4F68817981C054D04003C0C2
:10DE2000BC016E1B7F0BC05CDF4F288139814A81AA
:10DE30005B81CB01A0E0B0E082179307A407B50790
:10DE400008F4B901FCE961347F0718F060E47CE96B
:10DE500004C02EE46132720730F0769567957695AE
:10DE6000679584E007C037E26131730730F076953B
:10DE7000679582E080937C1108C081E080937C11DB
:10DE80006032710510F460E270E06052704048E06A
:10DE900060307407E8F0472F50E0440F551F440FDF
:10DEA000551F455B574F9A012E5F3F4FF9018591F2
:10DEB00094919C01AA27639FC001629F810D9A1FC4
:10DEC00006948A1F9A1F1124FA01459154911EC08D
:10DED000CB01969587958C7F855B934FFC0145918F
:10DEE0005491FC01329625913491862F90E08770F1
:10DEF0009070FC012E9FC0012F9F900D3E9F900DB2
:10DF0000112423E0969587952A95E1F7481B590B34
:10DF100044365105A8F4EFEEF2E007C08091C0004E
:10DF200085FFFCCF31969093C60090819923B1F77D
:10DF30008FED99E04AE050E00E94F54044E650E061
:10DF400050938900409388009A0140E050E080910E
:10DF5000831190918411A0918511B0918611820F47
:10DF6000931FA41FB51F8093831190938411A093D6
:10DF70008511B09386110CC0809187119091881102
:10DF800090938900809388008091891180937C11FF
:10DF9000209171113091721140917311509174114F
:10DFA000E0914311F091441180899189A289B3894C
:10DFB000281739074A075B0780F010924411109226
:10DFC000431190912D1180912E11981731F080916D
:10DFD0002E118F5F8F7080932E11FF91EF91DF9143
:10DFE000CF91BF91AF919F918F917F916F915F91F1
:10DFF0004F913F912F911F910F91FF90EF90DF90E4
:10E00000CF90BF90AF900F900BBE0F900FBE0F90B0
:10E010001F90189580917711882349F48091791188
:10E02000882329F480917B11882309F49CC0EBE4B8
:10E03000F0E1949108C08091C00085FFFCCF9093DF
:10E04000C600319694919923B1F7EDE8F0E19491EF
:10E0500008C08091C00085FFFCCF9093C600319628
:10E0600094919923B1F7809177118823F1F0609111
:10E0700045117091461180914711909148110E946D
:10E0800054D52091010C3091020C4091030C509119
:10E09000040C0E94B9D4AB01BC0189E890E10E9454
:10E0A000D31E89E790E10E946ECA8091791188237E
:10E0B000F1F06091491170914A1180914B1190914A
:10E0C0004C110E9454D52091050C3091060C4091C2
:10E0D000070C5091080C0E94B9D4AB01BC0185E734
:10E0E00090E10E94D31E85E690E10E946ECA809165
:10E0F0007B118823F1F060914D1170914E11809148
:10E100004F11909150110E9454D52091090C3091DB
:10E110000A0C40910B0C50910C0C0E94B9D4AB012D
:10E12000BC0181E690E10E94D31E81E590E10E944E
:10E130006ECAE3E0F3E007C08091C00085FFFCCF2A
:10E1400031969093C60090819923B1F78091C000D9
:10E1500085FFFCCF8AE08093C60010927711109261
:10E16000791110927B11089560E070E08FE793E4DD
:10E170002091B3033091B4034091B5035091B6039D
:10E180000E94B9D46093BD117093BE118093BF11EA
:10E190009093C0110895FC0197FF03C080919B11DB
:10E1A00003C0EE55FE4E808190E008952F923F927D
:10E1B0004F925F926F927F928F929F92AF92BF9297
:10E1C000CF92DF92EF92FF920F931F93CF93DF9343
:10E1D000EC0121E030E0A901440F551F440F551F09
:10E1E000FA01E158FE4E85919491C817D9070CF0B9
:10E1F00059C0B90161507040660F771F660F771FD5
:10E20000CB018F579E4EFC010591149161587E4EB3
:10E21000FB01C590D490FA01EF57FE4EE590F490C3
:10E22000FA01E158FE4EA590B490B801882777FD19
:10E230008095982F0E9454D51B012C01CC19DD0923
:10E24000BE01882777FD8095982F0E9454D53B0109
:10E250004C01E01AF10A0027F7FC0095102FC801C5
:10E26000B7010E9454D59B01AC01C401B3010E94C7
:10E2700092D77B018C01AC18BD08CC24B7FCC094AC
:10E28000DC2CC601B5010E9454D59B01AC01C8012C
:10E29000B7010E94B9D49B01AC01C201B1010E9437
:10E2A000D9D319C0822F8F5F2F5F3F4F21333105A4
:10E2B00009F091CF813329F0E0E070E080E060E088
:10E2C0000CC0E1E4F2E165917491882777FD8095B7
:10E2D000982F0E9454D5E62F692F2E2F372F482FC5
:10E2E000562FB901CA01DF91CF911F910F91FF9075
:10E2F000EF90DF90CF90BF90AF909F908F907F90E6
:10E300006F905F904F903F902F90089510928C11D6
:10E3100010928B111092A211749810928E1110927B
:10E320008D111092A311759810928E1110928D116B
:10E3300010929B11A59808952DEB37E346E05EE31C
:10E340000E9492D708952DEB37E346E05EE30E94EA
:10E35000B9D408952DEB37E346E05EE30E94B9D4CB
:10E3600008952DEB37E346E05EE30E9492D70895CF
:10E37000A5980E94C319882339F5ECE9F0E194913E
:10E3800008C08091C00085FFFCCF9093C6003196F5
:10E3900094919923B1F7E4EBF0E1949108C0809156
:10E3A000C00085FFFCCF9093C600319694919923CD
:10E3B000B1F78091C00085FFFCCF8AE08093C60052
:10E3C00083EA90E10E947DCA0E946A1A08951F9311
:10E3D000182F0E9486710E94C319882309F036C045
:10E3E000ECE9F0E1949108C08091C00085FFFCCF7A
:10E3F0009093C600319694919923B1F78FED99E0EF
:10E40000612F70E04AE050E00E94CB408091C00054
:10E4100085FFFCCF8AE08093C600EBEFF0E194919A
:10E4200008C08091C00085FFFCCF9093C600319654
:10E4300094919923B1F78091C00085FFFCCF8AE0C9
:10E440008093C6008EEE90E10E947DCA0E946A1AF7
:10E450001F9108951F93182F0E9486710E94C3195F
:10E46000882309F036C0ECE9F0E1949108C080916E
:10E47000C00085FFFCCF9093C600319694919923FC
:10E48000B1F78FED99E0612F70E04AE050E00E9413
:10E49000CB408091C00085FFFCCF8AE08093C6000E
:10E4A000E5E3F1E1949108C08091C00085FFFCCFC5
:10E4B0009093C600319694919923B1F78091C00052
:10E4C00085FFFCCF8AE08093C60088E291E10E943C
:10E4D0007DCA0E946A1A1F9108951F920F920FB66B
:10E4E0000F920BB60F9211242F933F934F935F938C
:10E4F0006F937F938F939F93AF93BF93EF93FF930C
:10E500009091C303992391F48091A2118093A71154
:10E51000882311F0749A01C0749880919B118093A4
:10E52000A611882311F0A59A01C0A5988091A71182
:10E53000891708F474988091A611891708F4A59892
:10E540009F5F9F779093C3038091C403843009F445
:10E5500071C0853050F4813021F1813098F08230E3
:10E56000F1F1833009F09FC049C0863009F48DC0B5
:10E57000863008F46EC0873009F48BC0883009F00B
:10E5800092C08FC088E080937B0080E480937C0001
:10E5900080917A00806480937A000E947D9781E068
:10E5A0001BC08091780090917900A0E0B0E02091AC
:10E5B000B4113091B5114091B6115091B711280F97
:10E5C000391F4A1F5B1F2093B4113093B51140933C
:10E5D000B6115093B71182E08093C40364C088E001
:10E5E00080937B0082E480937C0080917A00806439
:10E5F00080937A000E947D9783E0EECF809178002F
:10E6000090917900A0E0B0E02091A8113091A9117B
:10E610004091AA115091AB11280F391F4A1F5B1F5F
:10E620002093A8113093A9114093AA115093AB11D4
:10E6300084E0D2CF88E080937B0081E480937C00EB
:10E6400080917A00806480937A000E947D9785E0B3
:10E65000C3CF8091780090917900A0E0B0E0209144
:10E66000B0113091B1114091B2115091B311280FF6
:10E67000391F4A1F5B1F2093B0113093B111409393
:10E68000B2115093B31186E0A7CF0E947D9787E027
:10E69000A3CF1092C4038091B8118F5F8093B811FB
:10E6A00002C01092C4038091B811803108F466C092
:10E6B0008091A311882381F48091B4119091B511B8
:10E6C0009093901180938F118091A8119091A9112E
:10E6D000909396118093951181E08093A3111092ED
:10E6E000B8111092B4111092B5111092B611109287
:10E6F000B7111092B0111092B1111092B211109284
:10E70000B3111092AC111092AD111092AE11109283
:10E71000AF111092A8111092A9111092AA11109283
:10E72000AB1120918F11309190118091BF03909186
:10E73000C003281739071CF080E00E942A7220913C
:10E740008F11309190118091A4119091A511821791
:10E7500093071CF080E00E94E771209195113091A1
:10E7600096118091C1039091C2032817390734F0A4
:10E7700010928E1110928D110E94B871FF91EF913D
:10E78000BF91AF919F918F917F916F915F914F91C9
:10E790003F912F910F900BBE0F900FBE0F901F90C7
:10E7A0001895EF92FF920F931F93E0909111F090C4
:10E7B0009211009193111091941160918B117091AD
:10E7C0008C11882777FD8095982F0E9454D520E0E2
:10E7D00030E040EA51E40E94D8D39B01AC01C8016B
:10E7E000B7010E94B2D4882394F4C801B7010E94F3
:10E7F00021D570939D1160939C110E948F1460939A
:10E800009E1170939F118093A0119093A1111F915D
:10E810000F91FF90EF9008952F926F927F928F92B9
:10E820009F92AF92BF92CF92DF92EF92FF920F939F
:10E830001F93DF93CF93CDB7DEB729970FB6F89428
:10E84000DEBF0FBECDBF8C01E62E662369F1ECE979
:10E85000F0E1949108C08091C00085FFFCCF9093B7
:10E86000C600319694919923B1F78FED99E06E2D02
:10E8700070E04AE050E00E94CB40E2E6F1E1949182
:10E8800008C08091C00085FFFCCF9093C6003196F0
:10E8900094919923B1F78091C00085FFFCCF8AE065
:10E8A0008093C6000E94AC1AAE2DB0E0FD01EE0FC1
:10E8B000FF1FEC5DFB4F6081718179876887672B53
:10E8C00009F49FC0AA5DBB4F7C917B8322242394D3
:10E8D00079C0222D30E0A901440F551F440F551F68
:10E8E000E885F985E40FF51F8591949108171907BC
:10E8F0000CF067C0C9010197880F991F880F991FF5
:10E90000FC013296A885B985EA0FFB1FC590D4900B
:10E910008A0F9B1FFC01659174917A836983FA01C8
:10E920003296EA0FFB1FE590F490FD01E40FF51F0E
:10E93000A590B490B601882777FD8095982F0E9406
:10E9400054D56C837D838E839F8389819A81081B34
:10E95000190BB801882777FD8095982F0E9454D510
:10E960003B014C01EC18FD080027F7FC0095102F27
:10E97000C801B7010E9454D59B01AC01C401B30189
:10E980000E9492D77B018C01A981BA81AA1ABB0A85
:10E99000CC24B7FCC094DC2CC601B5010E9454D530
:10E9A0009B01AC01C801B7010E94B9D49B01AC0125
:10E9B0006C817D818E819F810E94D9D3E62F692F42
:10E9C00009C02394BB812B1608F483CFE0E070E0EC
:10E9D00080E060E0FB812F1679F5E22DF0E0EE0F8C
:10E9E000FF1FEE0FFF1F329768857985E60FF71F2F
:10E9F00065917491882777FD8095982F0E9454D552
:10EA000019C0B801882777FD8095982F0E9454D5AA
:10EA100020E030E04AEF5EE30E9492D720E030E051
:10EA200040E85DE30E9492D720E030E040E050E013
:10EA30000E94D9D3E62F692F2E2F372F482F562F1C
:10EA4000B901CA0129960FB6F894DEBF0FBECDBF3B
:10EA5000CF91DF911F910F91FF90EF90DF90CF90BA
:10EA6000BF90AF909F908F907F906F902F90089560
:10EA70000F931F93CF93DF9380E090E0A0E0B0E08E
:10EA80008093B9119093BA11A093BB11B093BC11AC
:10EA900060E070E08FE793E42091B3033091B4031A
:10EAA0004091B5035091B6030E94B9D46093BD1153
:10EAB0007093BE118093BF119093C0116C9A6D9AA0
:10EAC0009D9A8091010180618093010187E061E05E
:10EAD00070E00E94C61987ED80937A0010927E0044
:10EAE00010927D0080917D00816080937D008091F7
:10EAF0007D00826080937D0080917D0084608093A2
:10EB00007D0080E888BD80916E00846080936E00F7
:10EB10006AEF70E080E090E00E949D1485E090E054
:10EB20009093C2118093C11109C08091A41190915A
:10EB3000A51140969093A5118093A4118091A411E2
:10EB40009091A51160E00E940C7420E030E040EA52
:10EB500050E40E94B2D487FDE8CF83E191E0909326
:10EB6000C6038093C50309C08091BF039091C00381
:10EB700040979093C0038093BF038091BF0390910F
:10EB8000C00360E00E940C7420E030E849E853E4E0
:10EB90000E94C0D6181644F3C091C103D091C2039D
:10EBA0001C2F0D2FCE010E94D670609720E030E020
:10EBB00046E153E40E94C0D6181694F31093C103A3
:10EBC0000093C203DF91CF911F910F91089580911F
:10EBD0008F119091901160E00E940C7460939111DC
:10EBE0007093921180939311909394118091951149
:10EBF000909196110E94D67060939711709398111E
:10EC00008093991190939A110E9444938FB7F8942E
:10EC10001092A3118FBF08952F923F924F925F924F
:10EC20006F927F928F929F92AF92BF92CF92DF921C
:10EC3000EF92FF920F931F938091A311882309F401
:10EC40001DC20E94E77560909111709092118090A2
:10EC5000931190909411C0908B11D0908C11B601AB
:10EC6000882777FD8095982F0E9454D5A4019301A1
:10EC70000E94D8D37B018C016093C3117093C4119F
:10EC80008093C5119093C61120E030E040E251E43A
:10EC90000E94C0D6181624F481E08093C711E9C001
:10ECA000C801B70120E030E040E251EC0E94B2D44C
:10ECB00087FD02C0CD2821F481E08093C711C4C034
:10ECC0008091C711882371F080E090E0A0E0B0E06F
:10ECD0008093C8119093C911A093CA11B093CB111E
:10ECE0001092C711C801B7012091AF033091B00352
:10ECF0004091B1035091B2030E9492D71B012C01A5
:10ED00006093CC117093CD118093CE119093CF115D
:10ED1000C801B7012091C8113091C9114091CA11A1
:10ED20005091CB110E94D9D35B016C01E090B911D5
:10ED3000F090BA110091BB111091BC11A80197017C
:10ED40000E94B2D487FD12C0E090BD11F090BE11B8
:10ED50000091BF111091C011C601B501A801970122
:10ED60000E94C0D6181614F086017501E092C811F1
:10ED7000F092C9110093CA111093CB11C801B701C9
:10ED80002091B3033091B4034091B5035091B60381
:10ED90000E9492D75B016C016093D0117093D111E6
:10EDA0008093D2119093D311C401B3012091D41157
:10EDB0003091D5114091D6115091D7110E94D8D3DE
:10EDC0002091B7033091B8034091B9035091BA0331
:10EDD0000E9492D720ED3CEC4CE45DE30E9492D778
:10EDE0007B018C016091D8117091D9118091DA1159
:10EDF0009091DB1123E333E343E75FE30E9492D773
:10EE00009B01AC01C801B7010E94D9D37B018C01E1
:10EE10006093D8117093D9118093DA119093DB111C
:10EE2000C201B101A60195010E94D9D3A8019701A1
:10EE30000E94D8D37B018C0120E030E040E050E01C
:10EE40000E94B2D488235CF40F2EF0E0EF2EF0E0A5
:10EE5000FF2EF0E00F2FF0E01F2FF02D14C0C8019F
:10EE6000B70120E030E04FE753E40E94C0D6181607
:10EE700054F40F2EF0E0EF2EF0E0FF2EFFE70F2FFF
:10EE8000F3E41F2FF02D6092D4117092D51180926F
:10EE9000D6119092D7116091C1117091C21188273B
:10EEA00077FD8095982F0E9454D59B01AC01C40139
:10EEB000B3010E94C0D61816DCF46091C5037091AE
:10EEC000C603882777FD8095982F0E9454D59B0113
:10EED000AC01C401B3010E94B2D488234CF4C80130
:10EEE000B7010E9421D5759567956093A21102C064
:10EEF0001092A21180919E1190919F11A091A0114A
:10EF0000B091A1110097A105B10509F461C00E945B
:10EF10008F1420919E1130919F114091A01150911A
:10EF2000A111621B730B840B950B61547C498040CB
:10EF3000904008F44DC060919C1170919D11665FE6
:10EF40007F4F882777FD8095982F0E9454D59B018D
:10EF5000AC016091911170919211809193119091F7
:10EF600094110E94B2D488235CF510928C111092F7
:10EF70008B1189E492E10E946ECAE3E4F2E194917C
:10EF800008C08091C00085FFFCCF9093C6003196E9
:10EF900094919923B1F7E4E0F3E007C08091C000B9
:10EFA00085FFFCCF31969093C60090819923B1F7ED
:10EFB0008091C00085FFFCCF8AE08093C60008C026
:10EFC00010929E1110929F111092A0111092A111F7
:10EFD0000E948F142091DC113091DD114091DE11DF
:10EFE0005091DF11621B730B840B950B68587341B2
:10EFF0008040904008F442C00E948F146093DC115E
:10F000007093DD118093DE119093DF11E0909711E2
:10F01000F09098110091991110919A11C801B701BF
:10F0200020E030E040EA50E40E94C0D618161CF5FB
:10F03000C801B70120E030E046E153E40E94B2D4B9
:10F040008823CCF460918D1170918E11882777FD03
:10F050008095982F0E9454D59B01AC01C801B7013F
:10F060000E94C0D688231CF010929B1107C08FE726
:10F0700080939B1103C010929B11A5981F910F9133
:10F08000FF90EF90DF90CF90BF90AF909F908F90C8
:10F090007F906F905F904F903F902F9008952F92A8
:10F0A0003F924F925F926F927F928F929F92AF9218
:10F0B000BF92CF92DF92EF92FF920F931F93DF9355
:10F0C000CF93CDB7DEB7E6970FB6F894DEBF0FBE8D
:10F0D000CDBF6C8F7D8F8E8F9F8F5EAB4DAB39A375
:10F0E00028A30E948F14698B7A8B8B8B9C8B2DA904
:10F0F0003EA9223031051CF4E3E1F3E019C0E6E259
:10F10000F3E007C08091C00085FFFCCF319690935B
:10F11000C60090819923B1F78091C00085FFFCCF94
:10F1200014C48091C00085FFFCCF31969093C60037
:10F1300090819923B1F78091C00085FFFCCF8AE0D0
:10F140008093C6000E9486714DA95EA957FF74C0C6
:10F150008FE780939B1189899A89AB89BC898D87B8
:10F160009E87AF87B88B89879A87AB87BC8719AA98
:10F170001AAA1BAA1CAA1F8A1E8A91E09D8B1D82B7
:10F180001E821F8218868FE7A82EB12CC12CD12C8D
:10F190000FE7202E312C412C512C20E030E040E0B4
:10F1A00050E029833A834B835C830F2EF0E06F2E6F
:10F1B000F0E47F2EFCE18F2EF6E49F2EF02D4DA97A
:10F1C0005EA94E555E4E5BA34AA3EAE4F3E1549177
:10F1D0005CA3E5E4F3E184918DA3EEE3F3E1949184
:10F1E0009EA3E7E3F3E1A491AFA3E1E3F3E1B491DC
:10F1F000B8A7EBE2F3E1249129A7EDE1F3E1349123
:10F200003AA7E7E1F3E144914BA7E1E1F3E154913F
:10F210005CA7EBE0F3E184918DA7ADA9BEA9AA0F8D
:10F22000BB1FAA0FBB1FAF56BE4EBFA7AEA7E1EDD7
:10F23000F2E1B491B8AB07C0EDA9FEA9EE55FE4EC0
:10F240008FE7808388CF8091A311882309F4A3C21C
:10F250000E94E775EDA9FEA9F7FF0DC0F091971187
:10F26000F9AB209198112AAB309199113BAB4091A9
:10F270009A114CAB11C0AEA5BFA5BC91B9ABEEA520
:10F28000FFA5F181FAABAEA5BFA51296BC91BBABB1
:10F29000EEA5FFA5F381FCAB69817A818B819C810E
:10F2A00029A93AA94BA95CA90E94C0D6181644F016
:10F2B00089A99AA9ABA9BCA989839A83AB83BC838A
:10F2C000C401B30129A93AA94BA95CA90E94B2D4EF
:10F2D00087FD06C089A99AA9ABA9BCA93C014D012B
:10F2E0002D89222309F451C069A97AA98BA99CA967
:10F2F0002C8D3D8D4E8D5F8D0E94C0D618160CF062
:10F300004AC20E948F1429853A854B855C85621B11
:10F31000730B840B950B695873418040904008F43F
:10F320003AC2D601C50182199309A409B5094DA9AC
:10F330005EA957FF07C0B595A795979587958093C8
:10F340009B1107C0B595A79597958795EAA1FBA155
:10F3500080830E948F146D877E878F87988B9B0197
:10F36000AC0189859A85AB85BC85281B390B4A0B76
:10F370005B0B2D833E834F8358872C8D3D8D4E8DA7
:10F380005F8D29833A834B835C8369A97AA98BA912
:10F390009CA92C8D3D8D4E8D5F8D0E94B2D488230B
:10F3A0000CF0F8C10E948F142D853E854F85588939
:10F3B000621B730B840B950B69587341804090401E
:10F3C00008F4E8C10E948F1469877A878B879C872D
:10F3D0004E895F89452B09F4B8C1DC01CB012D852D
:10F3E0003E854F855889821B930BA40BB50B2D814D
:10F3F0003E814F815885280F391F4A1F5B1F288F78
:10F40000398F4A8F5B8F2D813E814F815885281B14
:10F41000390B4A0B5B0BCA01B901A20191010E9491
:10F4200064D8288D398D4A8D5B8D0E94CCD82A0DE9
:10F430003B1D4C1D5D1D24313105410551055CF41A
:10F4400074E1272E312C412C512C64E1A62EB12CD5
:10F45000C12CD12C1FC059016A013CEEA316B10486
:10F46000C104D1042CF05BEEA52EB12CC12CD12C03
:10F4700040E8A416B104C104D1041CF4150126010E
:10F4800009C04EEF242E312C412C512C2A183B0858
:10F490004C085D089CA1EAE4F3E108C08091C0003B
:10F4A00085FFFCCF9093C600319694919923B1F7D4
:10F4B0008FED99E0B601A5012AE030E00E94964068
:10F4C0009DA1E5E4F3E108C08091C00085FFFCCF79
:10F4D0009093C600319694919923B1F78FED99E0FE
:10F4E000B201A1012AE030E00E9496409EA1EEE325
:10F4F000F3E108C08091C00085FFFCCF9093C60067
:10F50000319694919923B1F78FED99E0B401A3015D
:10F5100022E030E00E94A6419FA1E7E3F3E108C0AA
:10F520008091C00085FFFCCF9093C60031969491E6
:10F530009923B1F78FED99E049815A816B817C81E4
:10F5400022E030E00E94A6418091C00085FFFCCF00
:10F550008AE08093C6008E899F8903970CF4F5C0DA
:10F56000C201B1010E9454D520E030E040E850E4EF
:10F570000E9492D77B018C0169817A818B819C8169
:10F58000A40193010E94D8D320ED3FE049E450E468
:10F590000E9492D720E030E040E05FE30E9492D7E3
:10F5A0009B01AC01C801B7010E94B9D47B018C0159
:10F5B000688D798D8A8D9B8D0E9454D520E030E036
:10F5C0004AE754E40E94B9D43B014C0198A5E1E319
:10F5D000F3E108C08091C00085FFFCCF9093C60086
:10F5E000319694919923B1F78FED99E0B801A70175
:10F5F00022E030E00E94A64199A5EBE2F3E108C0C9
:10F600008091C00085FFFCCF9093C6003196949105
:10F610009923B1F78FED99E0B401A30122E030E026
:10F620000E94A6418091C00085FFFCCF8AE08093B4
:10F63000C600C801B7012AE939E949E15FE30E9440
:10F6400092D77B018C019AA5EDE1F3E108C080918E
:10F65000C00085FFFCCF9093C6003196949199230A
:10F66000B1F78091C00085FFFCCF8AE08093C6008F
:10F670009BA5E7E1F3E108C08091C00085FFFCCFC6
:10F680009093C600319694919923B1F78FED99E04C
:10F69000B801A70122E030E00E94A6418091C0009D
:10F6A00085FFFCCF8AE08093C6009CA5E1E1F3E1F1
:10F6B00008C08091C00085FFFCCF9093C6003196B2
:10F6C00094919923B1F7C801B701A80197010E944D
:10F6D000D9D3A40193010E94B9D4AB01BC018FED31
:10F6E00099E022E030E00E94A6418091C00085FFB1
:10F6F000FCCF8AE08093C6009DA5EBE0F3E108C053
:10F700008091C00085FFFCCF9093C6003196949104
:10F710009923B1F7C801B701A40193010E9492D7C0
:10F7200020E030E040E05EE30E9492D7AB01BC01F4
:10F730008FED99E022E030E00E94A6418091C00068
:10F7400085FFFCCF8AE08093C600D201C1018A0DFB
:10F750009B1DAC1DBD1DEDA9FEA9F7FF07C0B5950A
:10F76000A7959795879580939B1107C0B595A79509
:10F7700097958795EAA1FBA180832E893F892F5F0A
:10F780003F4F3F8B2E8B6C8C7D8C8E8C9F8C31E011
:10F790003D8B01C01D8A6C8D7D8D8E8D9F8D20E0EF
:10F7A00030E040EA51E40E94D9D39B01AC0169A941
:10F7B0007AA98BA99CA90E94C0D618169CF4E1EEE8
:10F7C000F2E1949108C08091C00085FFFCCF909336
:10F7D000C600319694919923B1F78091C00085FFBE
:10F7E000FCCFB3C00E948F1429893A894B895C8968
:10F7F000621B730B840B950B615D774080409040DA
:10F8000008F454C04DA95EA957FF11C060919B1127
:10F81000EBEDF2E1949108C08091C00085FFFCCF30
:10F820009093C600319694919923B1F711C0AAA183
:10F83000BBA16C91E5EDF2E1949108C08091C0000C
:10F8400085FFFCCF9093C600319694919923B1F730
:10F85000162F8FED99E049A95AA96BA97CA922E03E
:10F8600030E00E94A64198A9E1EDF2E108C0809144
:10F87000C00085FFFCCF9093C600319694919923E8
:10F88000B1F78FED99E0612F70E04AE050E00E94FF
:10F89000CB408091C00085FFFCCF8AE08093C600FA
:10F8A0000E948F14698B7A8B8B8B9C8B0E948F1498
:10F8B0007B018C010E948F142D853E854F855889D0
:10F8C000E21AF30A040B150B29853A854B855C85F2
:10F8D000E21AF30A040B150BE60EF71E081F191F98
:10F8E00031E8E3163FE4F30632E1030730E01307A3
:10F8F00098F0E4EBF2E1949108C08091C00085FF9C
:10F90000FCCF9093C600319694919923B1F78091E2
:10F91000C00085FFFCCF19C04E895F8988A199A1DD
:10F920008417950774F5E8E5F2E1949108C0809199
:10F93000C00085FFFCCF9093C60031969491992327
:10F94000B1F78091C00085FFFCCF8AE08093C600AC
:10F95000E6960FB6F894DEBF0FBECDBFCF91DF9114
:10F960001F910F91FF90EF90DF90CF90BF90AF90DD
:10F970009F908F907F906F905F904F903F902F90CF
:10F9800008950E94A0CA5FCCFC01128213820895E0
:10F99000FC018381882311F081E082830895FC01BA
:10F9A0008281811112820895CF93DF93DC01FC01E3
:10F9B000EB55FE4F808191810097C9F101979183AA
:10F9C0008083ED01CC5ADF4FFD01ED58FF4F8BE1F5
:10F9D000019009928150E1F7FD01EE5AFF4FAF58B7
:10F9E000BF4F8D919C911197A157B0409183808317
:10F9F000FD01ED58FF4F20E030E0AD014B555E4F6B
:10FA000010C02F5F3F4FEF01DF015F968BE10D903C
:10FA100009928150E1F7858D968D3297918380838D
:10FA2000B196DA018D919C912817390750F3DF9137
:10FA3000CF910895FC0180E294E0918380838781D7
:10FA4000882321F0CF0104960E94C3450895CF92E8
:10FA5000DF92EF92FF920F931F93DF93CF93CDB777
:10FA6000DEB76F970FB6F894DEBF0FBECDBF8C0127
:10FA70006B01095A1F4FD8018C91075510408823FC
:10FA800021F42FE2E22EF12C03C090E5E92EF12CB7
:10FA9000E00EF11E80E294E09A8389831C821B822F
:10FAA00018861D82B7016C5F7F4FCE010596A601B7
:10FAB00021E00E94D04C882391F5EEE5F3E194918A
:10FAC00008C08091C00085FFFCCF9093C60031969E
:10FAD00094919923B1F7E4E6F3E1949108C0809101
:10FAE000C00085FFFCCF9093C60031969491992376
:10FAF000B1F709C08091C00085FFFCCF0894C11CFC
:10FB0000D11C9093C600F6019081992399F78091BA
:10FB1000C00085FFFCCF8AE08093C6005AC0F80180
:10FB2000EB55FE4F208131812A30310508F040C06D
:10FB30002F5F3F4F3183208321503040F90185E012
:10FB4000EE0FFF1F8A95E1F7E21BF30BED58FF4F15
:10FB5000E00FF11F13C0AF01415E5F4FBF018BE1AA
:10FB6000DB010D90BD01DA010D92AD018150C1F7AD
:10FB7000929182913296968F858F7F972150304057
:10FB8000BFEF2E3F3B0739F7D801AD58BF4FF70104
:10FB900034968BE101900D928150E1F70F581F4F81
:10FBA000F70182819381D8018D939C930157104076
:10FBB000D801AC5ABF4FFE0135968BE101900D92F2
:10FBC0008150E1F70E5A1F4F8B819C81F801918380
:10FBD0008083CE0101960E941A7D6F960FB6F8942D
:10FBE000DEBF0FBECDBFCF91DF911F910F91FF9070
:10FBF000EF90DF90CF900895EF92FF920F931F93B5
:10FC00008C013EECE32E31E0F32EE80EF91EC70125
:10FC10000E947345C7010E94C345F80110821182FA
:10FC20001F910F91FF90EF900895CF92DF92EF9286
:10FC3000FF920F931F93CF93DF937C016B01DB0146
:10FC40000D900020E9F78D0101501040061B170BA5
:10FC5000EEECF1E0EE0EFF1ED7011C92E2E3FEEFA8
:10FC6000EE0EFF1ECB016EE470E00E947711EC01F6
:10FC7000009731F4F8013197EC0DFD1D86010EC09F
:10FC800060E270E00E9477118C010F5F1F4FCE0180
:10FC90006AE270E00E947711FC0131978DE0818368
:10FCA0008AE082831382C70186539E4FB8010E9467
:10FCB000D24D8EEC91E0E80EF91ED7018C9188238D
:10FCC00019F1EEE8F3E1949108C08091C00085FF3E
:10FCD000FCCF9093C600319694919923B1F7E5E952
:10FCE000F3E1949108C08091C00085FFFCCF909310
:10FCF000C600319694919923B1F78091C00085FF99
:10FD0000FCCF8AE08093C600DF91CF911F910F91C5
:10FD1000FF90EF90DF90CF900895CF93DF93EC01A9
:10FD20008B81882309F43BC0EDEBF3E1949108C08B
:10FD30008091C00085FFFCCF9093C60031969491CE
:10FD40009923B1F7CD57DD4F488159816A817B8175
:10FD5000C358D2408FED99E02AE030E00E9477400E
:10FD6000EBEBF3E1949108C08091C00085FFFCCFDC
:10FD70009093C600319694919923B1F7C558DD4F01
:10FD8000488159816A817B818FED99E02AE030E0DA
:10FD90000E9477408091C00085FFFCCF12C0EBEA43
:10FDA000F3E1949108C08091C00085FFFCCF90934F
:10FDB000C600319694919923B1F78091C00085FFD8
:10FDC000FCCF8AE08093C600DF91CF9108952F92F7
:10FDD0003F924F925F926F927F928F929F92AF92DB
:10FDE000BF92CF92DF92EF92FF920F931F93DF9318
:10FDF000CF93CDB7DEB7AC970FB6F894DEBF0FBE8A
:10FE0000CDBF5C014B01FC018381882309F438C11B
:10FE1000C50182539E4F0E94C345F50112821A8A82
:10FE20001D8A198A188A80E294E09F878E875EE493
:10FE3000C52ED12CCA0CDB1C2FE230E0A20EB31E63
:10FE4000F601B182A08221ED3FEFA20EB31EF401B4
:10FE500080818F3209F090C0C4016FE270E00E948F
:10FE600077117C010894E11CF11C3E010894611C8F
:10FE7000711C260142E1242E312C2C0E3D1E77C030
:10FE8000C7016FE270E00E9477116C01009709F4DE
:10FE900081C0E816F90608F07DC08C010E191F0913
:10FEA000C301B701A8010E949711060D171DF801A3
:10FEB0001082F30107C08091C00085FFFCCF31960E
:10FEC0009093C60090819923B1F78091C00085FF7F
:10FED000FCCFFAE0F093C600F201608171816115F8
:10FEE000710519F460E070E002C06C5F7F4FC101E2
:10FEF000A30121E00E94D04C882371F5E9EFF3E1E2
:10FF0000949108C08091C00085FFFCCF9093C600FB
:10FF1000319694919923B1F7FE01319607C08091F3
:10FF2000C00085FFFCCF31969093C6009081992345
:10FF3000B1F7E7EFF3E1949108C08091C00085FF2D
:10FF4000FCCF9093C600319694919923B1F780919C
:10FF5000C00085FFFCCF8DC02EE030E02C0F3D1F90
:10FF6000F2013183208376010894E11CF11CE11435
:10FF7000F10409F085CF0BC080E590E0A80EB91E12
:10FF8000F601B182A08220EB3FEFA20EB31ED82C67
:10FF9000092D02C0DE2C0F2D8EE490E0A80EB91EB4
:10FFA000F5018081918122EB3FEFA20EB31E0097F5
:10FFB00019F480E090E001C004966D2D702F0E942E
:10FFC000A24D882339F1E9EEF3E1949108C08091C4
:10FFD000C00085FFFCCF9093C60031969491992381
:10FFE000B1F78D2D902F9C01F90107C08091C000C1
:10FFF00085FFFCCF31969093C60090819923B1F78D
:020000021000EC
:1000000083E892E0A80EB91EF501108211821282D7
:10001000138232C0E1EDF3E1949108C08091C000F9
:1000200085FFFCCF9093C600319694919923B1F748
:100030008D2D902F9C01F90107C08091C00085FF94
:10004000FCCF31969093C60090819923B1F7EFECE5
:10005000F3E1949108C08091C00085FFFCCF90939C
:10006000C600319694919923B1F78091C00085FF25
:10007000FCCF8AE08093C600CE010E960E941A7DC6
:10008000AC960FB6F894DEBF0FBECDBFCF91DF9117
:100090001F910F91FF90EF90DF90CF90BF90AF90A6
:1000A0009F908F907F906F905F904F903F902F9098
:1000B0000895BF92CF92DF92EF92FF920F931F931A
:1000C000CF93DF938C01EB018FE28993EE24E394CD
:1000D000FF2475EAC72E71E0D72EC00ED11E6FE146
:1000E000B62E14C0FB9CC00111248D589F4F800F69
:1000F000911FBE010E94D54502C02196E3948881DC
:10010000882319F08CE88E15C0F7F3942F2D30E07A
:10011000F601808191812817390720F3E7FC07C099
:10012000C80182539E4FBE010E94D54501C018826E
:10013000DF91CF911F910F91FF90EF90DF90CF90C3
:10014000BF9008952F923F924F925F926F927F924D
:100150008F929F92AF92BF92CF92DF92EF92FF92D7
:100160000F931F93DF93CF93CDB7DEB7AD970FB645
:10017000F894DEBF0FBECDBF6C014B014DA7DC0173
:1001800013968C91882309F44AC3E1EDF1E0CE0E79
:10019000DF1ED6018C91EFE2FEEFCE0EDF1E88232C
:1001A00009F419C1222309F0E1C029EE31E0C20EA1
:1001B000D31ED6018C91E7E1FEEFCE0EDF1E882321
:1001C00071F1EEE8F3E1949108C08091C00085FFE1
:1001D000FCCF9093C600319694919923B1F7E1ED4D
:1001E000F4E1949108C08091C00085FFFCCF90930A
:1001F000C600319694919923B1F78FED99E061E0B3
:1002000070E04AE050E00E94CB408091C00085FF42
:10021000FCCF8AE08093C6000E94AC1A00C3EEE5D2
:10022000F3E1949108C08091C00085FFFCCF9093CA
:10023000C600319694919923B1F7E8EBF4E19491DB
:1002400008C08091C00085FFFCCF9093C600319616
:1002500094919923B1F7F40107C08091C00085FF04
:10026000FCCF31969093C60090819923B1F7EDEAC7
:10027000F4E1949108C08091C00085FFFCCF909379
:10028000C600319694919923B1F7C6012EEE31E064
:10029000C20ED31EB6010E9459804BEF5FEFC40E11
:1002A000D51ED6019C91E7E1FEEFCE0EDF1E8DE854
:1002B000989FF0011124E251FE4FEC0DFD1D07C087
:1002C0008091C00085FFFCCF31969093C60090814D
:1002D0009923B1F7E7EAF4E1949108C08091C00056
:1002E00085FFFCCF9093C600319694919923B1F786
:1002F00023E832E0C20ED31ED6014D915D916D917F
:100300007C91EDE7FDEFCE0EDF1E8FED99E02AE048
:1003100030E00E9477408091C00085FFFCCF8AE0EA
:100320008093C600A60147515E4FDA012C91E22F5F
:10033000F0E0EE0FFF1FEE0FFF1FEC0DFD1DE6516D
:10034000FE4F83E892E0C80ED91ED6014D905D9015
:100350006D907C908DE79DEFC80ED91E4082518232
:10036000628273822F5FDA012C932FC0EEE5F3E1F6
:10037000949108C08091C00085FFFCCF9093C60087
:10038000319694919923B1F7E6E9F4E1949108C08C
:100390008091C00085FFFCCF9093C6003196949168
:1003A0009923B1F7F40107C08091C00085FFFCCF0D
:1003B00031969093C60090819923B1F78091C00047
:1003C00085FFFCCF8AE08093C600C60182539E4F12
:1003D0000E94C34539C0E9EEF1E0CE0EDF1ED60122
:1003E0001C92E7E1FEEFCE0EDF1EEEE5F3E1949105
:1003F00008C08091C00085FFFCCF9093C600319665
:1004000094919923B1F7E5E8F4E1949108C08091C3
:10041000C00085FFFCCF9093C6003196949199233C
:10042000B1F7F40107C08091C00085FFFCCF319681
:100430009093C60090819923B1F78091C00085FF09
:10044000FCCF8AE08093C600D60112961C921A8ACD
:100450001D8A198A188A80E294E09F878E87FEE4BD
:10046000AF2EB12CAC0CBD1CEFE2F0E0CE0EDF1EC7
:10047000D501CD92DC92E1EDFFEFCE0EDF1ED4016F
:100480008C918F3209F090C0C4016FE270E00E943D
:1004900077117C010894E11CF11C3E010894611C59
:1004A000711C2501E2E12E2E312C2C0E3D1E77C051
:1004B000C7016FE270E00E9477115C01009709F4B8
:1004C00081C0E816F90608F07DC08C010E191F09DD
:1004D000C301B701A8010E949711060D171DF8016D
:1004E0001082F30107C08091C00085FFFCCF3196D8
:1004F0009093C60090819923B1F78091C00085FF49
:10050000FCCFFAE0F093C600D2016D917C916115A9
:10051000710519F460E070E002C06C5F7F4FC101AB
:10052000A30121E00E94D04C882371F5E1E7F4E1BA
:10053000949108C08091C00085FFFCCF9093C600C5
:10054000319694919923B1F7FE01319607C08091BD
:10055000C00085FFFCCF31969093C600908199230F
:10056000B1F7EFE6F4E1949108C08091C00085FFF7
:10057000FCCF9093C600319694919923B1F7809166
:10058000C00085FFFCCF1BC12EE030E02C0F3D1FCB
:10059000F2013183208375010894E11CF11CE11400
:1005A000F10409F085CF0BC040E550E0C40ED51E24
:1005B000D501CD92DC92E0EBFFEFCE0EDF1E082DD1
:1005C000F92C01C00E2DF601E25BFF4F2DA5222371
:1005D00009F4B1C0608171816115710519F460E0A1
:1005E00070E002C06C5F7F4FC60182539E4F402F68
:1005F0005F2D21E00E94D04C882309F46CC04FEDA0
:1006000051E0C40ED51ED6014D915D916D917C9146
:10061000ECE9F0E0CE0EDF1ED6014D935D936D93B5
:100620007C931397E5E8FDEFCE0EDF1EE1E6F4E1E3
:10063000949108C08091C00085FFFCCF9093C600C4
:10064000319694919923B1F7802F9F2D9C01F90148
:1006500007C08091C00085FFFCCF31969093C60003
:1006600090819923B1F7E9E5F4E1949108C0809174
:10067000C00085FFFCCF9093C600319694919923DA
:10068000B1F78FED99E02AE030E00E947740809149
:10069000C00085FFFCCF8AE08093C60023E832E0EB
:1006A000C20ED31ED6011D921D921D921C9213974D
:1006B000EBE4F4E1949108C08091C00085FFFCCF89
:1006C0009093C600319694919923B1F78091C00020
:1006D00085FFFCCF99C0E7E3F4E1949108C08091D5
:1006E000C00085FFFCCF9093C6003196949199236A
:1006F000B1F7802F9F2D9C01F90107C08091C000A8
:1007000085FFFCCF31969093C60090819923B1F775
:10071000E5E3F4E1949108C08091C00085FFFCCF2F
:100720009093C600319694919923B1F78091C000BF
:1007300085FFFCCF44C0608171816115710519F49A
:1007400060E070E002C06C5F7F4FC60182539E4F35
:10075000402F5F2D26E50E94D04C882309F033C03E
:10076000E1E2F4E1949108C08091C00085FFFCCFE4
:100770009093C600319694919923B1F7802F9F2DC5
:100780009C01F90107C08091C00085FFFCCF319624
:100790009093C60090819923B1F7EFE1F4E1949131
:1007A00008C08091C00085FFFCCF9093C6003196B1
:1007B00094919923B1F78091C00085FFFCCF8AE026
:1007C0008093C60028C081E0F6018083EDE0F4E16B
:1007D000949108C08091C00085FFFCCF9093C60023
:1007E000319694919923B1F7F40107C08091C0002C
:1007F00085FFFCCF31969093C60090819923B1F785
:100800008091C00085FFFCCF8AE08093C600802FD6
:100810009F2D0E9491CACE010E960E941A7DAD9620
:100820000FB6F894DEBF0FBECDBFCF91DF911F9101
:100830000F91FF90EF90DF90CF90BF90AF909F907F
:100840008F907F906F905F904F903F902F90089582
:10085000EF92FF920F931F93CF93DF93EC010E94CF
:100860008A698E0107511E4FD8018C919EECE92EAA
:1008700091E0F92EEC0EFD1E8823A1F1C7010E9424
:10088000C345F8016081615060838DE8689FB001C5
:10089000112462517E4F6C0F7D1FCE0141E021E09B
:1008A0000E94A280D801EC91F0E0EE0FFF1FEE0F46
:1008B000FF1FEC0FFD1FE651FE4F40815181628109
:1008C0007381CD57DD4F488359836A837B83C35837
:1008D000D240C7010E94A9448B81882369F081E03E
:1008E0008A830AC00E947B68C7010E94C3451A829E
:1008F00082E593E10E94583EDF91CF911F910F91C5
:10090000FF90EF900895FC0181E08183CF0140E0EA
:1009100021E00E94A2800895EF92FF920F931F930F
:10092000CF93DF938C01FC01138286A9882321F0E9
:10093000C801C3960E94C34527EAE22E21E0F22EA9
:10094000E00EF11EC70160E045E30E946D4388237D
:1009500009F5EEE5F3E1949108C08091C00085FFB0
:10096000FCCF9093C600319694919923B1F7E2E4BD
:10097000F5E1949108C08091C00085FFFCCF909371
:10098000C600319694919923B1F78091C00085FFFC
:10099000FCCF7DC0E801C455DE4FCE01B70141E078
:1009A0000E94674E882341F5CE01B70140E00E94C6
:1009B000674E882309F5EEE8F3E1949108C0809131
:1009C000C00085FFFCCF9093C60031969491992387
:1009D000B1F7EFE2F5E1949108C08091C00085FF86
:1009E000FCCF9093C600319694919923B1F78091F2
:1009F000C00085FFFCCF4BC0C801C396BE010E945A
:100A0000C448882309F5EEE8F3E1949108C0809189
:100A1000C00085FFFCCF9093C60031969491992336
:100A2000B1F7EFE1F5E1949108C08091C00085FF36
:100A3000FCCF9093C600319694919923B1F78091A1
:100A4000C00085FFFCCF23C081E0F8018383EEE581
:100A5000F3E1949108C08091C00085FFFCCF909392
:100A6000C600319694919923B1F7E4E1F5E19491B0
:100A700008C08091C00085FFFCCF9093C6003196DE
:100A800094919923B1F78091C00085FFFCCF8AE053
:100A90008093C600D801AC5ABF4FF801F3968BE1A2
:100AA00001900D928150E1F7F80181A992A90E5AA7
:100AB0001F4FF8019183808302551040C8018F9623
:100AC000025B1F4FF80191838083DF91CF911F91CB
:100AD0000F91FF90EF9008952F923F924F925F9267
:100AE0006F927F929F92AF92BF92CF92DF92EF92DE
:100AF000FF920F931F93DF93CF93CDB7DEB7CC5503
:100B0000D0400FB6F894DEBF0FBECDBF6C01662398
:100B100011F527E832E0C20ED31ED6018C91E9E729
:100B2000FDEFCE0EDF1E882309F4E2C02FE732E08E
:100B3000C20ED31ED601ED90FD900D911C91E1E8FF
:100B4000FDEFCE0EDF1E0E948F14E616F706080793
:100B5000190708F4CDC027E832E0C20ED31ED60133
:100B60001C92E9E7FDEFCE0EDF1ED60113968C91A5
:100B7000882341F4C6010E948C84F6018381882376
:100B800009F4B6C000D000D0EDB7FEB731967E01B3
:100B90000894E11CF11CADB7BEB71296FC92EE9220
:100BA000119785E893E193838283D6019D968D9179
:100BB0009C919E97958384830E94A6118701EDB72F
:100BC000FEB736960FB6F894FEBF0FBEEDBF5701C5
:100BD00008C0D8018C9190E00E94F5D8F80181936B
:100BE0008F01F50101900020E9F73197EA19FB091F
:100BF000802F8E198E176CF363E3A62EB12CAC0CEC
:100C0000BD1CC50140E050E060E070E00E94A944D6
:100C100099245DE3E52EF12CEC0EFD1E2E010894C7
:100C2000411C511C4FE1642E712C6C0E7D1E3EE761
:100C3000232E33E1332E42C0D8018C9190E00E94E4
:100C4000F5D8F80181938F01F70101900020E9F7B1
:100C50003197EE19FF09802F8E198E176CF32796A6
:100C60008FAD27978E3751F1C701B20145E050E0B3
:100C70000E948911009711F500D000D0EDB7FEB7A2
:100C80003196ADB7BEB712967C926E9211973382B1
:100C90002282558244820E94A611EDB7FEB7369695
:100CA0000FB6F894FEBF0FBEEDBFC3010E94D13E48
:100CB0008AE793E10E94583E99249394C501B701B5
:100CC00040E050E00E94E047181614F48701BCCFC2
:100CD000992041F48FEF9FEFD6019E969C938E93BF
:100CE0009D9706C0F60185A596A5019696A785A7AE
:100CF000C45ADF4F0FB6F894DEBF0FBECDBFCF9101
:100D0000DF911F910F91FF90EF90DF90CF90BF90F8
:100D1000AF909F907F906F905F904F903F902F90FB
:100D200008952F923F924F925F926F927F928F928F
:100D30009F92AF92BF92CF92DF92EF92FF920F936A
:100D40001F93DF93CF93CDB7DEB7CF58D0400FB608
:100D5000F894DEBF0FBECDBF8C013B016A0184E079
:100D600090E0C80ED91EF8017196C757DF4FF9837E
:100D7000E883C958D040C8010496CA57DF4F998309
:100D80008883C658D040C857DF4F1882C858D04013
:100D9000B6E6EB2EF12CEC0EFD1EF7013B96C55787
:100DA000DF4FF983E883CB58D040A8E88A2EA2E031
:100DB0009A2E800E911EF9E8AF2EF2E0BF2EA00E03
:100DC000B11EEEE02E2E312C2C0E3D1E77E4472E68
:100DD000512C4C0E5D1EC2010496C357DF4F998300
:100DE0008883CD58D040EEE5F3E19491C157DF4FB1
:100DF0009883CF58D04049C1F7018385282F30E030
:100E0000A901487150704031510509F04CC1F401FD
:100E10009081913009F447C1923009F444C1F7013F
:100E2000DE0111969081903239F08E2F8E19883024
:100E300011F48EE28D939D933196C557DF4F8881D3
:100E40009981CB58D040E817F90761F71C921E86AC
:100E5000F3018081882329F4C10160E573E00E94D9
:100E60006C11C101B3010E946C11C101BE016F5F21
:100E70007F4F0E946C11C10160E573E00E946C110C
:100E80001CA61FA61BA61AA680E294E099A788A715
:100E9000CE018C96B601AE014F5F5F4F21E00E94FC
:100EA000D04C882309F03EC0F40180818823D1F51D
:100EB000C157DF4F9881CF58D040EEE5F3E108C02D
:100EC0008091C00085FFFCCF9093C600319694912D
:100ED0009923B1F7E2E5F3E007C08091C00085FFF8
:100EE000FCCF31969093C60090819923B1F7809101
:100EF000C00085FFFCCFFAE0F093C600FE013196FA
:100F000007C08091C00085FFFCCF31969093C6004A
:100F100090819923B1F78091C00085FFFCCF8AE0D2
:100F20008093C600C357DF4FA881B981CD58D04008
:100F3000FE01BC968BE101900D928150E1F78AA5EC
:100F40009BA5F2019383828380E294E09183808366
:100F5000C801B101A2010E949186C2010E941A7DBE
:100F6000CE0188960E941A7D90C0953E09F48DC0EE
:100F70009E3209F48AC09F3509F487C0F80191892F
:100F8000992331F09E3209F480C09F3509F47DC069
:100F900023FD7BC080E04031510509F481E0F80178
:100FA00084A7882349F4F7018085873409F06DC050
:100FB00081858E3709F469C0CA57DF4FA881B9818E
:100FC000C658D040F7018081803241F08E2F8E19B3
:100FD000883011F48EE28D9380818D933196C557C0
:100FE000DF4F88819981CB58D040E817F90759F72E
:100FF0001C92F4018081882329F5F30107C08091B8
:10100000C00085FFFCCF31969093C6009081992354
:10101000B1F7CA57DF4FE881F981C658D04007C001
:101020008091C00085FFFCCF31969093C6009081DF
:101030009923B1F78091C00085FFFCCFFAE0F093CF
:10104000C60023C0813039F4F50180819181019679
:10105000918380831AC08230C1F4C857DF4FF88172
:10106000C858D0402F2F30E0F5018081918128179A
:101070003907F1F0C857DF4FF881C858D040FF5FFB
:10108000C857DF4FF883C858D040C601B701C757CB
:10109000DF4F48815981C958D0400E94E047181657
:1010A0000CF4AACE05C0F7019081992309F05DCF19
:1010B000C157DF4F0FB6F894DEBF0FBECDBFCF9143
:1010C000DF911F910F91FF90EF90DF90CF90BF9035
:1010D000AF909F908F907F906F905F904F903F90D8
:1010E0002F900895EF92FF920F931F93DF93CF936A
:1010F000CDB7DEB76F970FB6F894DEBF0FBECDBF8A
:101100007C018C01025B1F4F805B9F4FF801918334
:10111000808328E832E0E20EF31E21E0F7012193FC
:101120007F011182108227E73DEFE20EF31E049645
:1011300040E050E060E070E00E94A944F8012081A6
:101140003181DE011596F90134968BE101900D9203
:101150008150E1F7F901828193819C838B8380E246
:1011600094E09A838983C70165E673E08E010F5F7F
:101170001F4FA8010E949186C8010E941A7DF701A5
:10118000E757FD4F808191816F960FB6F894DEBFCF
:101190000FBECDBFCF91DF911F910F91FF90EF90C8
:1011A0000895EF92FF920F931F93DF93CF93CDB7E4
:1011B000DEB76F970FB6F894DEBF0FBECDBF7C01D0
:1011C0008C01025B1F4F805B9F4FF80191838083EE
:1011D00028E832E0E20EF31E22E0F701208328E740
:1011E0003DEFE20EF31EF701E757FD4F60831182DA
:1011F000049640E050E060E070E00E94A944F801ED
:1012000020813181DE011596F90134968BE1019040
:101210000D928150E1F7F901828193819C838B8348
:1012200080E294E09A838983C70165E673E08E01CA
:101230000F5F1F4FA8010E949186C8010E941A7D6E
:101240006F960FB6F894DEBF0FBECDBFCF91DF9182
:101250001F910F91FF90EF900895EF92FF920F93DF
:101260001F93DF93CF93CDB7DEB76F970FB6F89488
:10127000DEBF0FBECDBF7C0188E892E0E80EF91E0C
:10128000F701108288E79DEFE80EF91E87010D5CDB
:101290001F4FC80140E050E060E070E00E94A944A8
:1012A000DE011596F8018BE101900D928150E1F776
:1012B000F70181A992A99C838B8380E294E09A83B1
:1012C0008983C70165E673E08E010F5F1F4FA80198
:1012D0000E949186C8010E941A7D6F960FB6F894FD
:1012E000DEBF0FBECDBFCF91DF911F910F91FF9059
:1012F000EF9008950F931F93CF93DF93DC01D39664
:101300001C92D397D6961C92D697D2961C921E9278
:10131000D19780E294E0D0969C938E939F97AC5A9D
:10132000BF4F1C9213961C92A755B040FD01E05B85
:10133000FF4FAE5ABF4F11961C921E92A255B0405D
:1013400091838083ED01C159DF4FFE0120E030E041
:10135000482F148217821382128240839183215E68
:101360003F4F7F9681E02633380799F7A855BE4F47
:1013700089E18C9313961C9258961C921B961C9292
:1013800013961C92A15DB140FD01E653FE4FA4539C
:10139000BE4F11961C921E9240839183A155BF4F60
:1013A0001D921D921D921C92139718961D921D92CC
:1013B0001D921C921397A358B24012961C9212973A
:1013C00013961C9213971C9211961C9211978D01E3
:1013D00001581D4FF8011082118212821382AB5501
:1013E000BE4F11961C921E92AC5BBF4F1C92FE0129
:1013F000C90111920197E9F7A256BF4F81E08C9382
:10140000A758B2409E961C921E929D970E948F14E0
:1014100068577C4E8F4F9F4FF801608371838283A2
:101420009383DF91CF911F910F910895DF93CF9315
:10143000CDB7DEB72A970FB6F894DEBF0FBECDBF8B
:101440008091660390916703A0916803B09169034E
:101450008B839C83AD83BE83FE01339624E630E00C
:101460008081F999FECF1FBA32BD21BD80BD0FB674
:10147000F894FA9AF99A0FBE2F5F3F4F283631053C
:1014800011F03196EDCFE1E0FCE08081F999FECFDB
:101490001FBA32BD21BD80BD0FB6F894FA9AF99AF1
:1014A0000FBE2F5F3F4F2837310511F03196EDCF3A
:1014B000E1EFFBE08081F999FECF1FBA32BD21BD7B
:1014C00080BD0FB6F894FA9AF99A0FBE2F5F3F4F7E
:1014D0002838310511F03196EDCFE1E1FCE0808153
:1014E000F999FECF1FBA32BD21BD80BD0FB6F89469
:1014F000FA9AF99A0FBE2F5F3F4F2839310511F044
:101500003196EDCFE5E2FCE08081F999FECF1FBA7C
:1015100032BD21BD80BD0FB6F894FA9AF99A0FBE7C
:101520002F5F3F4F2C39310511F03196EDCFE9E2B5
:10153000FCE08081F999FECF1FBA32BD21BD80BD8C
:101540000FB6F894FA9AF99A0FBE2F5F3F4F203AE0
:10155000310511F03196EDCFE1E2FCE08081F9999F
:10156000FECF1FBA32BD21BD80BD0FB6F894FA9AE6
:10157000F99A0FBE2F5F3F4F243A310511F0319693
:10158000EDCFE9E3FCE08081F999FECF1FBA32BDCF
:1015900021BD80BD0FB6F894FA9AF99A0FBE2F5F5D
:1015A0003F4F283A310511F03196EDCFEDEEFBE0DB
:1015B0008081F999FECF1FBA32BD21BD80BD0FB623
:1015C000F894FA9AF99A0FBE2F5F3F4F2C3A3105E3
:1015D00011F03196EDCFEDE2FCE08081F999FECF7C
:1015E0001FBA32BD21BD80BD0FB6F894FA9AF99AA0
:1015F0000FBE2F5F3F4F203B310511F03196EDCFED
:10160000E1E3FCE08081F999FECF1FBA32BD21BD34
:1016100080BD0FB6F894FA9AF99A0FBE2F5F3F4F2C
:10162000243B310511F03196EDCFE5E3FCE08081FC
:10163000F999FECF1FBA32BD21BD80BD0FB6F89417
:10164000FA9AF99A0FBE2F5F3F4F283B310511F0F0
:101650003196EDCFE4E6F7E08081F999FECF1FBA2D
:1016600032BD21BD80BD0FB6F894FA9AF99A0FBE2B
:101670002F5F3F4F243C310511F03196EDCFE8EE5E
:10168000F1E18081F999FECF1FBA32BD21BD80BD45
:101690000FB6F894FA9AF99A0FBE2F5F3F4F263C87
:1016A000310511F03196EDCFEAEEF1E18081F99943
:1016B000FECF1FBA32BD21BD80BD0FB6F894FA9A95
:1016C000F99A0FBE2F5F3F4F283C310511F031963C
:1016D000EDCFECEEF1E18081F999FECF1FBA32BD7A
:1016E00021BD80BD0FB6F894FA9AF99A0FBE2F5F0C
:1016F0003F4F2A3C310511F03196EDCFEEEEF1E18E
:101700008081F999FECF1FBA32BD21BD80BD0FB6D1
:10171000F894FA9AF99A0FBE2F5F3F4F2C3C31058F
:1017200011F03196EDCFE0EFF1E18081F999FECF34
:101730001FBA32BD21BD80BD0FB6F894FA9AF99A4E
:101740000FBE2F5F3F4F2E3C310511F03196EDCF8C
:10175000E2EFF1E18081F999FECF1FBA32BD21BDE0
:1017600080BD0FB6F894FA9AF99A0FBE2F5F3F4FDB
:10177000203D310511F03196EDCFEFE7F7E08081A4
:10178000F999FECF1FBA32BD21BD80BD0FB6F894C6
:10179000FA9AF99A0FBE2F5F3F4F243D310511F0A1
:1017A0003196EDCFEFEAF3E08081F999FECF1FBAD1
:1017B00032BD21BD80BD0FB6F894FA9AF99A0FBEDA
:1017C0002F5F3F4F283D310511F03196EDCFE3EB10
:1017D000F3E08081F999FECF1FBA32BD21BD80BDF3
:1017E0000FB6F894FA9AF99A0FBE2F5F3F4F2C3D2F
:1017F000310511F03196EDCFE7EBF3E08081F999F7
:10180000FECF1FBA32BD21BD80BD0FB6F894FA9A43
:10181000F99A0FBE2F5F3F4F203E310511F03196F0
:10182000EDCF80E290E09A838983FE01319680813A
:10183000F999FECF1FBA32BD21BD80BD0FB6F89415
:10184000FA9AF99A0FBE213E310521F0319621EE28
:1018500030E0EDCF80916A0390916B03A0916C030F
:10186000B0916D038F839887A987BA87FE01379659
:1018700084E690E02081F999FECF1FBA92BD81BD28
:1018800020BD0FB6F894FA9AF99A0FBE87369105E3
:1018900019F001963196EECFEFE4F5E1949108C08E
:1018A0008091C00085FFFCCF9093C6003196949143
:1018B0009923B1F7E9E5F7E1949108C08091C00060
:1018C00085FFFCCF9093C600319694919923B1F790
:1018D0008091C00085FFFCCF8AE08093C6002A96E5
:1018E0000FB6F894DEBF0FBECDBFCF91DF91089544
:1018F000DF93CF93CDB7DEB7E0970FB6F894DEBF96
:101900000FBECDBFDE011196E7E4F4E080E1019067
:101910000D928150E1F7DE015196E7E3F4E080E1BA
:1019200001900D928150E1F7DE019196E7E2F4E03B
:1019300080E101900D928150E1F789819A81AB811C
:10194000BC818093010C9093020CA093030CB09384
:10195000040C89899A89AB89BC898093F10B909397
:10196000F20BA093F30BB093F40B89A19AA1ABA156
:10197000BCA18093110C9093120CA093130CB09304
:10198000140C8D819E81AF81B8858093050C909356
:10199000060CA093070CB093080C8D899E89AF8923
:1019A000B88D8093F50B9093F60BA093F70BB09343
:1019B000F80B8DA19EA1AFA1B8A58093150C9093B3
:1019C000160CA093170CB093180C89859A85AB85DB
:1019D000BC858093090C90930A0CA0930B0CB093D8
:1019E0000C0C898D9A8DAB8DBC8D8093F90B9093E7
:1019F000FA0BA093FB0BB093FC0B89A59AA5ABA5A2
:101A0000BCA58093190C90931A0CA0931B0CB09357
:101A10001C0C8D859E85AF85B88980930D0C9093A5
:101A20000E0CA0930F0CB093100C8D8D9E8DAF8D6E
:101A3000B8A18093FD0B9093FE0BA093FF0BB09386
:101A4000000C8DA59EA5AFA5B8A980931D0C909301
:101A50001E0CA0931F0CB093200C0E94335680E004
:101A600090E0AAE7B5E48093250C9093260CA09310
:101A7000270CB093280C80E090E8ABE3B5E48093AA
:101A8000290C90932A0CA0932B0CB0932C0C20E0E3
:101A900030E040E050E02093210C3093220C409342
:101AA000230C5093240C80E29EE4A0E0B0E08093ED
:101AB000ED0B9093EE0BA093EF0BB093F00B2093F4
:101AC000390C30933A0C40933B0C50933C0C80E023
:101AD00090E0A0EAB1E480932D0C90932E0CA0939B
:101AE0002F0CB093300C8DEC9CECACECBEE38093EF
:101AF000310C9093320CA093330CB093340C80E0F3
:101B000090E0A0EAB0E48093350C9093360CA0935B
:101B1000370CB093380C20936C0730936D074093CB
:101B20006E0750936F0720936807309369074093BF
:101B30006A0750936B0720936407309365074093BF
:101B400066075093670782ED90E09093E9118093C8
:101B5000E81186E490E09093EB118093EA111092E3
:101B6000ED111092EC118AEF90E09093EF118093B9
:101B7000EE1184E690E09093F1118093F0111092B1
:101B8000F3111092F2118AE999E9A1EBB1E4809383
:101B9000AF039093B003A093B103B093B20361E796
:101BA0007DE38AE89FE30E949C716093B303709386
:101BB000B4038093B5039093B60360E070E084EEC5
:101BC00092E40E94AA716093B7037093B803809364
:101BD000B9039093BA030E94B47080E090E0A0E84B
:101BE000BFE38093BB039093BC03A093BD03B0936A
:101BF000BE03EFE4F5E1949108C08091C00085FF39
:101C0000FCCF9093C600319694919923B1F7E5E506
